:020000022000DC
:1070000000F003206D7302005573020057730200F5
:10701000597302005B7302005D7302000000000000
:107020000000000000000000000000005F7302008C
:1070300061730200000000006373020065730200C8
:1070400067730200677302006773020067730200D0
:107050006773020067730200C9C50300677302000B
:107060006773020067730200159A030067730200DA
:1070700067730200677302006773020067730200A0
:1070800067730200392F0400F9EA020067730200F7
:107090009D2F04006773020061C90300677302003B
:1070A0006773020067730200677302006773020070
:1070B0006773020067730200000000000000000018
:1070C0006773020067730200677302006773020050
:1070D0006773020067730200677302006773020040
:1070E000677302006773020067730200000000000C
:1070F00000000000677302000000000067730200D8
:10710000000000000000000000000000000000007F
:10711000000000000000000000000000000000006F
:10712000000000000000000000000000000000005F
:10713000000000000000000000000000000000004F
:10714000000000000000000000000000000000003F
:10715000000000000000000000000000000000002F
:10716000000000000000000000000000000000001F
:10717000000000000000000000000000000000000F
:1071800000000000000000000000000000000000FF
:1071900000000000000000000000000000000000EF
:1071A00000000000000000000000000000000000DF
:1071B00000000000000000000000000000000000CF
:1071C00000000000000000000000000000000000BF
:1071D00000000000000000000000000000000000AF
:1071E000000000000000000000000000000000009F
:1071F000000000000000000000000000000000008F
:10720000344935480A1A02D0072291438D46334942
:1072100033480A1A06D00722914381F309880222D3
:1072200082F314882F483049304A00F042F8304841
:107230003049314A00F03DF830483149314A00F0D8
:1072400038F831483149324A00F033F83148324990
:10725000324A00F02EF832483249334A00F029F819
:1072600032483349334A00F024F833483349002286
:1072700000F02AF832483349002200F025F832485D
:107280003249091A082902DB0022026041601F48C6
:107290001F49884205D00268043003B4904703BCFC
:1072A000F7E700208646EC4600200021284A904758
:1072B000FEE7884207D0521A05D0037801300B70E0
:1072C0000131013AF9D17047884202D00270013091
:1072D000FAE7704700F0032000E8032000F00320E5
:1072E00000F003206C650400002E00207C2E00209E
:1072F000A0730200A0730200E43404006C65040073
:10730000002E0020002E00209C3804009C38040031
:107310009C3804009C3804009C3804009C3804000D
:107320009C3804009C3804006C650400E865040087
:107330007C2E00207C2E00207C2E00200C5D002066
:107340000C5D00200C5D00200C5D00200C61002015
:1073500005810200FEE7FEE7FEE7FEE7FEE7FEE747
:10736000FEE7FEE7FEE7FEE700F002B8FFF7FCBF2E
:1073700008484FF00701884385460748804707487B
:10738000016841F470010160BFF34F8FBFF36F8F4D
:10739000FFF736BF00F0032055CA030088ED00E078
:1073A00041DF70470B781BBB124B1B6813F4804FF7
:1073B0001ED0114B1B68032B1ADD10B584B00F4B88
:1073C000D3F804354A685088097B526914786CB93F
:1073D00092F90D20039202910190094A0092E12254
:1073E0000849042008F0C0FB04B010BD0022F1E7FA
:1073F000704700BF242E0020202E002000100140E6
:10740000D4380400CB38040030B5C7B0724B1B68C9
:1074100013F4804F03D0714B1B68032B2FDC6E4B92
:107420001B6813F4804F03D06C4B1B68032B32DCBA
:10743000694B1B6813F4804F03D0684B1B68032B08
:107440003ADC654B1B6813F4804F03D0634B1B6819
:10745000032B5DDC604B1B6813F4804F03D05F4B44
:107460001B68032B7FDC5C4B1B6813F4804F04D03C
:107470005A4B1B68032B00F3A28047B030BD584B1A
:10748000D3F80435574A009240F2032256490420AB
:1074900008F06AFBC3E7524BD3F80435534A11781E
:1074A000527802920191524A00924FF401724E4971
:1074B000042008F059FBBBE700230F2B12D84B4ADE
:1074C0001A4492F830204B490C6810095900255C89
:1074D00005A800F8135002F00F020131A25C4254DB
:1074E0000133EAE705AA00238DF8343003F1804325
:1074F00003F58833D3F8043502923F4A01923F4A9C
:10750000009240F206223849042008F02DFB98E74B
:1075100000230F2B11D8354A1A44127C35490C68C8
:1075200010095900255C05A800F8135002F00F025D
:107530000131A25C42540133EBE705AA00238DF828
:10754000343003F1804303F58833D3F804350292D5
:107550002B4A0192294A009240F207222249042034
:1075600008F002FB76E700230F2B12D81F4A1A44BB
:1075700092F820201F490C6810095900255C05A8C5
:1075800000F8135002F00F020131A25C42540133A3
:10759000EAE705AA00238DF8343003F1804303F5B0
:1075A0008833D3F804350292164A0192134A0092A6
:1075B0004FF402720C49042008F0D6FA53E7084B46
:1075C000D3F80435104A009240F2092206490420FB
:1075D00008F0CAFA51E700BF242E0020202E002018
:1075E000001001400C390400CB380400982E002014
:1075F00028390400282E002058390400643904007A
:107600006C390400783904008439040000B585B071
:107610000390124B1B6813F4804F03D0104B1B6870
:10762000042B0BDCBDF80E30012B12D140220021BF
:107630000C481BF0CBFE05B05DF804FB0A4BD3F8F9
:1076400004350A4A009290220949052008F08CFA74
:10765000E8E7784602F0C6FCE8E700BF242E0020E9
:10766000202E0020982E002000100140CC3904006C
:10767000CB38040000B583B00378142B1BD01D2B2E
:107680000AD11C4B1B6813F4804F03D01A4B1B68A4
:10769000042B04DCFFF7B8FE03B05DF804FB174BC6
:1076A000D3F80435164A00924FF4A172154905200B
:1076B00008F05AFAEEE7C388102BEDD10D4B1B688A
:1076C00013F4804F03D00C4B1B68032B05DC4022C6
:1076D00000210D481BF07AFEDEE7084BD3F8043595
:1076E0000A4A00924FF4A6720649042008F03CFAB8
:1076F000EDE700BF242E0020202E002000100140C6
:10770000E8390400CB380400982E0020083A040021
:10771000F0B585B003900C46154B1B6813F4804FF1
:1077200003D0144B1B68042B12DCBDF80E30012B68
:1077300019D1114E06F1400735460FCD206061602A
:10774000A260E3602E461034BD42F5D105B0F0BD15
:107750000A4BD3F804350A4A0092872209490520CA
:1077600008F002FAE1E7784602F03CFCE1E700BFEE
:10777000242E0020202E0020982E002000100140F2
:107780004C3A0400CB380400F0B585B003900D46A8
:10779000154B1B6813F4804F03D0144B1B68042B4C
:1077A00013DCBDF80E30012B1AD12C46104F40359A
:1077B0003E4620686168A268E3680FC61034374609
:1077C000AC42F5D1002005B0F0BD0A4BD3F804352A
:1077D000094A00927C220949052008F0C5F9E0E732
:1077E000784602F0FFFBE0E7242E0020202E002048
:1077F000982E002000100140643A0400CB380400A9
:1078000000B583B0194B1B6813F4804F03D0184B9D
:107810001B68032B12DC174B4FF6FF725A809A80BD
:107820001A80154817F0C4FCA0B9144A0021144866
:107830001BF09CF8A0B903B05DF804FB114BD3F822
:107840000435114A00924FF4D5721049042008F013
:107850008BF9E0E70E4A4FF4D97115F0F3F9E4E73C
:107860000B4A40F2B31115F0EDF9E4E7242E0020A5
:10787000202E00207C2E002095780200A5730200A7
:10788000842E0020001001407C3A0400CB38040014
:107890009C38040070B582B004460D4616460D4B68
:1078A0001B6813F4804F03D00B4B1B68032B06DCC3
:1078B00032462946204601F0E3FE02B070BD074B78
:1078C000D3F80435064A0092FD220649042008F048
:1078D0004BF9EDE7242E0020202E0020001001405F
:1078E0009C3A0400CB38040000B583B0234B1B68DE
:1078F00013F4804F03D0224B1B68032B1ADC1F4B61
:107900001B6813F4804F03D01D4B1B68032B1FDC37
:107910001A4B1B6813F4804F03D0194B1B68032BC1
:1079200021DC0021174B19700E2002F03DF903B045
:107930005DF804FB144BD3F80435144A52780192D5
:10794000134A0092BF221349042008F00DF9D6E72C
:107950000D4BD3F80435104A0092C0220D49042083
:1079600008F002F9D4E7084BD3F804350B4A00922B
:10797000C1220849042008F0F7F8D2E7242E00209D
:10798000202E0020942E002000100140982E002070
:10799000B43A0400CB380400D83A0400043B040095
:1079A00000B583B00E4B1B6813F4804F03D00D4B12
:1079B0001B68032B08DC00210B4B19700D2002F013
:1079C000F3F803B05DF804FB084BD3F80435084A1C
:1079D0000092D2220749042008F0C6F8EBE700BF66
:1079E000242E0020202E0020942E00200010014084
:1079F0003C3B0400CB38040000B583B00F4B1B6840
:107A000013F4804F03D00E4B1B68032B0ADC00F0ED
:107A1000CDFC00F073FC01210D2002F0C5F803B08D
:107A20005DF804FB074BD3F80435074A00924FF486
:107A300083720649042008F097F8E8E7242E002016
:107A4000202E0020001001406C3B0400CB380400C5
:107A500000B583B0254B1B78002B31D1244B5A78CD
:107A60001B789A4229D2234B1B6813F4804F03D012
:107A7000214B1B68032B14DC1D48C36801930023B2
:107A8000009300F120020221408801F051FE012103
:107A90000E2002F089F8154B01221A7003B05DF830
:107AA00004FB164BD3F80435154A009240F2271216
:107AB0001449042008F058F8DEE7FFF79DFFEAE7D5
:107AC0000C4B1B6813F4804FE8D00B4B1B68032B47
:107AD000E4DD0A4BD3F804350B4A009240F237122A
:107AE0000849042008F040F8D8E700BF942E002091
:107AF000982E0020242E0020202E0020001001406F
:107B0000903B0400CB380400C43B040008B5094B8B
:107B10001B7823B9084B5A781B789A4200D308BDCA
:107B2000013B054A1370FFF767FF024B01221A70F1
:107B3000F5E700BF942E0020982E002008B500F035
:107B40000FFC024B18680AF084FF08BD943D040046
:107B500000B583B00F4B1B6813F4804F03D00E4B5E
:107B60001B68032B09DC0322C8210F2002F088F8D0
:107B70000BF006FF03B05DF804FB084BD3F80435A7
:107B8000074A00924FF4B2720649042007F0ECFF56
:107B9000E9E700BF242E0020202E00200010014025
:107BA000F43B0400CB38040010B582B0441C214BD8
:107BB0001B6813F4804F03D01F4B1B68032B1ADC88
:107BC000022C29D0042C2AD0012C21D0194B1B685F
:107BD00013F4804F1ED0184B1B68032B1ADD174B74
:107BE000D3F80435164A00924FF4CB72154904209D
:107BF00007F0BAFF0EE0114BD3F804350194124A96
:107C000000924FF4BC720F49042007F0ADFFD7E794
:107C1000FFF71EFF02B010BDFFF778FFFAE70BF089
:107C20005CFE10B9FFF794FFF4E7FFF787FF0BF056
:107C300048FEF7E7242E0020202E002000100140EF
:107C40009C3D0400CB380400103C040000B583B018
:107C50003138032814D90D4B1B6813F4804F11D011
:107C60000B4B1B68032B0DDD0A4BD3F804350A4A76
:107C700000924FF4D2720949042007F075FF01E029
:107C8000FFF792FF03B05DF804FB00BF242E002035
:107C9000202E0020001001409C3D0400CB38040041
:107CA00000B583B00649074B18680AF0A1FE10B969
:107CB00003B05DF804FB784602F094F9F8E700BFE2
:107CC000982E0020783D040000B583B0154B1B684A
:107CD00013F4804F03D0144B1B68032B14DC0021DA
:107CE0000E2001F061FF01210D2001F05DFF0F4A20
:107CF000537801335370FFF7D3FF00F057FB00F0C8
:107D0000FDFA03B05DF804FB094BD3F80435074ACC
:107D100052780192074A0092B2220749042007F0E4
:107D200023FFDCE7242E0020202E0020982E0020A8
:107D300000100140243C0400CB38040000B583B09F
:107D4000104B1B6813F4804F03D00F4B1B68032BA1
:107D50000CDC00210D2001F027FF01210E2001F095
:107D600023FFFFF79DFF03B05DF804FB074BD3F83B
:107D70000435074A0092C8220649042007F0F4FEA1
:107D8000E7E700BF242E0020202E00200010014035
:107D90004C3C0400CB38040008B5FFF781FF08BD58
:107DA00010B582B004460F4B1B6813F4804F03D00C
:107DB0000D4B1B68032B04DC2378232B0ED002B061
:107DC00010BD0A4BD3F8043502780192084A00929C
:107DD000F1220849042007F0C7FEEDE7002005F076
:107DE0002FFDECE7242E0020202E00200010014063
:107DF000683C0400CB38040000B583B064212148FE
:107E000001F0F4FD204B1B6813F4804F03D01F4B8F
:107E10001B68032B17DC0BF050FD00BB1A4B1B68D3
:107E200013F4804F03D0194B1B68032B1DDC00217A
:107E30000F2001F00FFF0222C8210F2001F020FFC8
:107E400003B05DF804FB124BD3F80435114A0092DD
:107E500040F20F221049042007F086FEDBE70F4AAC
:107E600040F2112114F0EEFED8E7094BD3F80435A7
:107E70000B4A009240F217220749042007F074FED3
:107E8000D5E700BF4D7C0200242E0020202E0020CC
:107E900000100140843C0400CB3804009C380400EE
:107EA0009C3D040008B5124B998818890DF0DEFD41
:107EB00058B90F4B998818890DF08AFE58B90C4BA8
:107EC00018881AF071F960B908BD0A4A40F25B11CE
:107ED00014F0B8FEEDE7074A4FF4AE7114F0B2FEAD
:107EE000EDE7044A40F25F1114F0ACFEECE700BF8E
:107EF0007C2E00209C38040030B593B02022002155
:107F00000DEB02001BF062FA01238DF820300723ED
:107F10008DF8233006238DF82830454B0C93454BC4
:107F20001093454805F026FC0DF1470108A80BF019
:107F3000D9FC044660B30B2829D1404B1B6813F4CD
:107F4000804F03D03E4B1B68032B14DC3B4B1B685C
:107F500013F4804F1CD03A4B1B68032B18DD394BB0
:107F6000D3F80435384A009240F2C712374904204A
:107F700007F0FAFD0CE0334BD3F80435344A009295
:107F80004FF4E3723149042007F0EEFDDEE710B94B
:107F90003CB113B030BD2F4A4FF4E67114F052FEDD
:107FA000F6E702AC2C4D0FCD0FC495E8030084E832
:107FB000030002A800F072FD9DF84730FBB91F4B8B
:107FC0001B6813F4804F03D01D4B1B68032B0ADC86
:107FD00000F08CFDFFF766FFFFF7DEFE1F4920482B
:107FE00001F048FCD5E7174BD3F804351D4A009241
:107FF0004FF4F0721549042007F0B6FDE8E70F4B87
:108000001B6813F4804F03D00D4B1B68032B02DC5D
:1080100000F0D0FCE2E70B4BD3F80435124A009293
:108020004FF4F4720949042007F09EFDF0E700BF09
:10803000A17D020001780200002E0020242E0020E5
:10804000202E002000100140C03C0400CB3804006A
:10805000903C04009C3804007C3D0400E978020058
:10806000C97C0200FC3C0400343D040000B583B030
:108070001C4A04214FF4C04007F05AFD1A4B1B68FC
:1080800013F4804F03D0194B1B68032B11DC1AF03B
:1080900089FFD0B901F026FE154801F057FED0B98E
:1080A00001F094FEFFF728FF01F01AFC03B05DF821
:1080B00004FB104BD3F804350F4A009240F2F31240
:1080C0000E49042007F050FDE1E70D4A40F2F5119A
:1080D00014F0B8FDDEE70A4A40F2F91114F0B2FDDF
:1080E000DEE700BF05FB0200242E0020202E00202A
:1080F000A97B020000100140483D0400CB38040079
:108100009C38040008B5FFF7B1FFFFF775FEFFF7D5
:1081100047F9FCE7184B1B781BB1174B01221A706B
:10812000704700B587B0154A03AB07CA03C323F8ED
:10813000022B120C1A70124B009303AB114A124916
:10814000124815F0DDF868B9114816F0D5FD014662
:108150000E4815F001F950B9074B01221A7007B00B
:108160005DF804FB0B4A962114F06CFDECE7094A1C
:10817000972114F067FDEFE754320020E843040034
:10818000218402001C2F00205832002004310020DE
:108190003C2F0020D03E040038B52F4B5C68E568CA
:1081A00029462E481BF045F930B9A37903F2013076
:1081B0000133A371608038BD294629481BF039F985
:1081C00028B9637903F2012001336371F2E729468C
:1081D00024481BF02EF928B9E37903F2014001335A
:1081E000E371E7E7294620481BF023F938B9237AE1
:1081F00003EB430000F2015001332372DAE7294612
:108200001A481BF016F938B9637A03EB430000F201
:10821000016001336372CDE7294615481BF009F967
:1082200038B9A37A03EB430000F201700133A37263
:10823000C0E729460F481BF0FCF828B9E37A03F69B
:1082400001000133E372B5E7237903F140008000B8
:1082500001332371AEE700BF3C320020143F04001D
:10826000343F0400503F0400803F0400A83F040056
:10827000D03F0400FC3F040070B58AB005460023DF
:108280000393049305930693079308938DF8243082
:10829000154E3389ADF81C30FFF77EFFADF8220094
:1082A00003AC736853F8100F59689A68DB680FC401
:1082B0000E490F4815F066F858B90123009303AB37
:1082C000094A927A29460B4815F060F830B90AB08D
:1082D00070BD094A8C2114F0B5FCEEE7064A8D21E9
:1082E00014F0B0FCF3E700BF3C3200201C2F00204C
:1082F0005832002004310020D03E040000B583B085
:10830000104B1B6813F4804F03D00F4B1B68032BDB
:1083100006DC0E4815F0E8F870B903B05DF804FB10
:108320000B4BD3F804350B4A00924FF4A3720A4961
:10833000042007F019FCECE7084A40F2471114F05A
:1083400081FCEAE7242E0020202E00202184020058
:10835000001001401C400400FF3E0400D03E040019
:1083600000B583B00C4B1B6813F4804F03D00B4B4C
:108370001B68032B04DC15F0BFF803B05DF804FBA9
:10838000074BD3F80435074A00924FF4A67206490A
:10839000042007F0E9FBEEE7242E0020202E002029
:1083A0000010014040400400FF3E040000B583B0CF
:1083B000134B5B685B78282B0AD0124B02221A7091
:1083C000114B01221A70FFF7A5FE03B05DF804FB04
:1083D000FFF7C6FF0D4B1B6813F4804FF5D00C4B15
:1083E0001B68032BF1DD0B4BD3F804350A4A0092CE
:1083F0004FF49D720949042007F0B6FBE5E700BF82
:108400003C3200209832002038320020242E0020F8
:10841000202E0020001001406C400400FF3E0400AC
:1084200070B5C8B0044603780A2B10D8DFE813F003
:108430000B008102BD000F000F000F000F0059025A
:108440000F00F70175019B4B1B78012B01D048B041
:1084500070BD994B1B6813F4804F03D0974B1B687A
:10846000032B5BDCE269137843B9934B1B6813F46D
:10847000804F03D0914B1B68032B51DC637D002B95
:10848000E5D08D4B1B6813F4804F03D08B4B1B68DA
:10849000032B7ADC8A4D6E6804F1160001F000FAB5
:1084A000F0606B68DB68002BD1D0FFF759FF824B7F
:1084B0001B6813F4804F03D0804B1B68032B66DCD2
:1084C0007C4B03221A70201DFFF7D6FEBFE7E2188F
:1084D00012797C490D68100959002E5C07A800F834
:1084E000136002F00F020131AA5C425401330F2BDA
:1084F000EDD907AA00238DF83C3003F1804303F542
:108500008833D3F8043502926F4A01926F4A009281
:10851000A8226F49042007F027FBA3E70023E6E722
:108520006C4BD3F8043592F90D2001926A4A0092FF
:10853000AB226749042007F017FB9FE7E218927D02
:1085400060490D68100959002E5C07A800F81360F7
:1085500002F00F020131AA5C42540133032BEDD922
:1085600007AA00238DF8243003F1804303F58833F4
:10857000D3F804350292594A0192544A0092B1222A
:108580005349042007F0F0FA84E70023E6E7514B53
:10859000D3F804356A68D2680192514A0092B72232
:1085A0004B49042007F0E0FA8AE7434B1B6813F4B9
:1085B000804F03D0414B1B68032B28DC3D4B1B78BD
:1085C000032B35D0022B7FF442AF3D4C6268137809
:1085D00001331370E368984723699847364B1B684B
:1085E00013F4804F04D0354B1B68032B00F38280BB
:1085F000334B5A685088D368019300240094234673
:108600002032022101F094F82A4B1C701FE7314BF5
:10861000D3F80435334A12780292264A127801922E
:10862000314A0092C0222A49042007F09DFAC5E78A
:108630002C4B1B78EBB1204B1B6813F4804F03D0FD
:108640001E4B1B68032B09DC1A4B01221A70254AAA
:108650001378013B1370FFF751FEF8E61D4BD3F87A
:108660000435224A0092C5221949042007F07CFAF9
:10867000EAE7114B1B6813F4804F03D00F4B1B68C4
:10868000002B06DC0B4B00221A700D4B5B699847E0
:10869000DDE6104BD3F80435227A09494968498848
:1086A00002910192124A0092CC220949012007F05E
:1086B0005BFAE7E738320020242E0020202E00202D
:1086C0003C320020282E0020C840040064390400F9
:1086D000FF3E040000100140D0400400DC400400D4
:1086E000E840040098320020144104005C4104007A
:1086F000804104009A4BD3F8043562685188994848
:10870000008803900291D2680192974A0092D82281
:108710009649042007F028FA6AE7954B1B6813F482
:10872000804F03D0934B1B68032B4EDC924B0222ED
:108730001A708F4B1B6813F4804F03D08D4B1B684E
:10874000032B4DDCE3688D49D88A0FF03BFB0028F2
:1087500051D1E0688A4B19688A4BA2684988C08A5F
:1087600010F06AF800284BD1864B188816F096FD59
:1087700000284AD1814B1988824B188816F044FD95
:10878000002847D17A4B1B6813F4804F3FF45FAE4B
:10879000784B1B68032B7FF75AAE714BD3F8043527
:1087A000E268D28A76490968498876480088049048
:1087B00003917249098802910192734A0092FB2247
:1087C0006A49042007F0D0F941E6654BD3F8043537
:1087D0006E4A0092E9226549042007F0C5F9A5E731
:1087E0005F4BD3F804356A4A0092EE225F490420B9
:1087F00007F0BAF9A6E7674AEF2114F023FAA8E7D1
:10880000644AF12114F01EFAAEE7624AF72114F02F
:1088100019FAAFE75F4AF82114F014FAB2E7027AC6
:10882000504B1A80102300220121406814F0DDFD16
:1088300000283FF40CAE4E4B1B6813F4804F03D05E
:108840004C4B1B68002B13DC534B1B784BB3484B32
:108850001B6813F4804F03D0464B1B68032B14DCBA
:10886000454B01221A704C4A1378013B1370EEE518
:108870003B4BD3F804350190484A009240F20F1266
:108880003A49012007F070F9DEE7354BD3F804359B
:10889000434A00924FF489723449042007F064F986
:1088A000DEE7334B1B6813F4804F03D0314B1B685A
:1088B000032B06DC304B00221A70314B5B69984762
:1088C000C5E5274BD3F804352D4A526852880192EA
:1088D000344A00924FF48C722449042007F044F982
:1088E000E8E707AD304B0FCB85E80F001022294693
:1088F000606814F083FDB0B91D4B1B6813F4804F02
:108900003FF4A5AD1B4B1B68032B7FF7A0AD144BA9
:10891000D3F80435254A009240F227121349042067
:1089200007F022F993E51B4A4FF4937114F08AF98A
:10893000E2E70F4B1B6813F4804F3FF488AD0D4BFB
:108940001B68032B7FF783AD054BD3F80435184A1A
:1089500000924FF496720549042007F005F976E578
:10896000001001409A320020C4410400FF3E040080
:10897000242E0020202E002038320020162F002028
:108980003C320020182F00204C420400004204001A
:1089900024420400D03E040098320020904204009B
:1089A000C0420400D0420400804304003843040065
:1089B0006043040030B589B00123069306A90DF188
:1089C00016000FF02BFF60BB069B012B2FD12C4C08
:1089D0002568BDF816000FF0BBFB688023685A8835
:1089E0004FF6FF739A4226D0254B1B6806AA191D25
:1089F000588810F069F910BB07A80FF0D5F9204B83
:108A00001968BDF81C000FF0A3FFF0B91D4B1B68DF
:108A100013F4804F03D01C4B1B68032B1BDC09B0E5
:108A200030BD1A4A4FF4AC7114F00CF9CCE778461B
:108A300001F0D8FACBE7784601F0D4FAD4E7134A2C
:108A40004FF4AE7114F0FEF8D6E7104A4FF4B0714F
:108A500014F0F8F8DAE70E4BD3F80435084A126838
:108A6000518890881288039202900191094A0092DD
:108A70004FF4B1720849042007F076F8CFE700BF41
:108A80003C320020242E0020202E0020D03E040066
:108A90000010014094430400FF3E040038B5044632
:108AA000C36883B1636993B12369A3B10C4D0FCC43
:108AB0000FC594E8030085E803000023094A1370FA
:108AC000094A137038BD784601F08CFAEAE7784617
:108AD00001F088FAE8E7784601F084FAE6E700BF9B
:108AE0003C320020543200203832002010B584B0CF
:108AF000324BDB68039303A80FF022F9002835D12D
:108B00002F4C60681021084405F054FA6068102169
:108B1000203005F04FFA60681021303005F04AFA35
:108B2000616822680232103100200FF003FC18BB8C
:108B3000244B1B6813F4804F03D0234B1B68032B7B
:108B400020DC1F4B19685A680B1D20324988002011
:108B50000FF01AFF30BB1A4A136852683032598836
:108B600001200FF069FE18BB04B010BD174A4FF486
:108B7000BB7114F067F8C3E7144A4FF4BF7114F0E7
:108B800061F8D5E7124BD3F804350D4A12685288C4
:108B90000192104A009240F27F120F49042006F021
:108BA000E3FFCEE7094A4FF4C07114F04BF8D2E767
:108BB000064A40F2831114F045F8D5E7E843040073
:108BC0003C320020242E0020202E0020D03E040025
:108BD00000100140D4430400FF3E040082B04FF671
:108BE000FF73ADF800300B4B1B685B88ADF80230AB
:108BF000009B0020DAB262F30700C3F3072262F39E
:108C00000F20C3F3074262F317401B0E63F31F608C
:108C100002B070470C2E002010F0010F02D04CF271
:108C2000050070474CF20400704710F0010F02D0AD
:108C30004CF2030070474CF20200704741F20323EC
:108C4000984264D015D941F2103398426BD8B0F5F0
:108C5000985F3AD3A0F59850102821D8DFE800F0AB
:108C60005B431E4F51555320202020202020204BB5
:108C70004D0041F20703984218D8B0F5805F09D340
:108C8000A0F5805007280FD8DFE800F00C47292B0B
:108C9000330E2F3102283CD12648704726487047B2
:108CA00026487047264870472448704741F2011310
:108CB000984234D041F20213984201D121487047C2
:108CC000B0F5885F2DD12048704741F204239842C7
:108CD0002BD041F20523984229D11C4870471C48EB
:108CE00070471C4870471C4870471C4870471C4818
:108CF00070471C4870471C4870471C4870471C4808
:108D000070471C4870471C4870471C4870471C48F7
:108D100070470A4870471B4870471B4870471B48FC
:108D20007047064870470548704719487047034820
:108D3000704700BF6844040008440400F045040084
:108D4000B0450400A045040000460400104604009D
:108D5000384404005044040090440400B04404002B
:108D6000CC440400F04404001845040028450400E5
:108D700040450400544504006C4504008C45040043
:108D8000F84304007844040020440400C84504006B
:108D9000DC45040070B5054614460E4601B122B10B
:108DA000044B5D801E705C6070BD784601F01AF95E
:108DB000F6E700BFA432002010B584B0424B5A88B9
:108DC00082420ED148F21F03984240D035D848F273
:108DD000030398423DD048F2190398421AD10C7807
:108DE00046E03A4B1B6813F4804F03D0384B1B68A6
:108DF000002B02DC022004B010BD364BD3F8043542
:108E000002900192344A0092F3223449012006F084
:108E1000ABFEEFE702282AD02C4B1B6813F4804FDF
:108E200003D02B4B1B68002B15DC2D4A4FF48971A6
:108E3000052013F007FFFF241AE048F225039842AB
:108E40002FD048F23E039842E6D10C7810E00C781F
:108E50000EE00C780CE01F4BD3F80435214A009249
:108E600040F211121D49012006F07EFEDDE7FF24CD
:108E7000154B18780028BED0144B1B6813F4804F94
:108E800003D0134B1B68032B0DDC00230E4A127812
:108E90009A4215D90C4A5268D25CA24212D00133D0
:108EA000F4E7FF24E4E70B4BD3F8043501940E4AB2
:108EB00000924FF48D720949042006F055FEE4E754
:108EC000012098E7002096E7A4320020242E0020FD
:108ED000202E0020001001405C4604004F46040094
:108EE0002046040088460400A846040030B583B03C
:108EF0000446084A012148F23E00FFF74BFF064BAB
:108F00001D88FFF76BFE02462946204616F0B8FA88
:108F100003B030BD984A04009C32002070B504466E
:108F200015461E460180104604F0A6FA2071E58021
:108F3000104B1B88A3810023A3732822E27326749D
:108F400001256574A374FFF749FEE074C0F307239D
:108F50002375C0F307436375C0F30760A075064A25
:108F6000294648F21900FFF715FF204616F012FABD
:108F700070BD00BF9C320020904A040030B585B01F
:108F80000446084601AD002301930293ADF8061094
:108F900004F072FA8DF80400074A012148F21F001C
:108FA000FFF7F8FEFFF71AFE034695E80600204695
:108FB00016F00AFA05B030BD944A040010B50A4B09
:108FC0001B7863B1084C2378013B04F8043B04F0A0
:108FD000B7FE06490144204604F07EFE10BD7846E7
:108FE00001F000F8EEE700BFBC320020404B4C001F
:108FF00008B5034804F058FE024B034A1A6008BD46
:10900000C03200200C2E00205C4C040008B5FFF795
:10901000EFFF024B1B68984708BD00BFB03200202D
:10902000F0B58BB0914B1A681378013B482B00F2D6
:109030004982DFE813F0BD00490073009800C700C3
:10904000C700C700C700C700C700C700C700C700E8
:10905000C700C700C700C700C700C700C700C700D8
:10906000C700C700C700C700C700C700EA003D012E
:109070007901B30117023D017901B30117023D01E6
:109080007901B30117023D01B3013D01B3013D0177
:10909000B3013D01B3013D01B301E5013D01B30160
:1090A0003D01B3013D01B3013D01B3017901170257
:1090B0003D01B3013D01B3017901170279011702A6
:1090C0003D01B3013D01B301694B1B6813F4804FAF
:1090D00003D0684B1B68032B14DC002016F0F4F857
:1090E0000446002211460220FFF754FE44B116F058
:1090F000D1F9614B1B78002B00F0EB81FFF75EFF8D
:109100000BB0F0BD5D4BD3F804355D4A00924FF4CF
:10911000D7725C49042006F027FDDEE7544B1B683C
:1091200013F4804F03D0534B1B68032B0BDC01213E
:10913000022016F071F904460022114648F225007B
:10914000FFF728FED2E74D4BD3F8043501220292F7
:10915000022201924C4A009240F2B712494904207F
:1091600006F002FDE3E7424B1B6813F4804F03D087
:10917000404B1B68032B0FDC444B1A68444B198887
:10918000444B188816F0C4F80446434A022148F2BA
:109190000300FFF7FFFDA9E7384BD3F804353F4A3A
:1091A00000924FF4E1723749042006F0DDFCE3E75A
:1091B0003B490B8801330B8004322C4B1A60FFF7BC
:1091C0002FFF9DE72A4B1B6813F4804F03D0294BD8
:1091D0001B68032B05DC324B1888FFF787FE04461B
:1091E00084E7264BD3F804455088FFF727FD2C4B26
:1091F0001B88029301902B4B009323464FF4F67289
:109200002049042006F0B0FCE5E700230493059311
:109210000693079308930993234B1B780122204957
:10922000098804A8FFF77AFE0446114B1B6813F463
:10923000804F3FF45BAF0F4B1B68032B7FF756AF9C
:109240000E4BD3F80455094B1B685888FFF7F6FC02
:10925000012302930190154B00932B4640F2FF121D
:109260000849042006F080FC40E700BF0C2E0020D7
:10927000242E0020202E0020BC32002000100140AF
:10928000C44604004F460400E0460400D8320020E3
:109290009C320020AC3200209C4A0400104704009D
:1092A0009E320020204704008C4A04004C470400F2
:1092B0000023049305930693079308930993864B21
:1092C0001C88864B1888FFF7A7FC02464FF0000366
:1092D000214604A8FFF722FE0446814B1B6813F4C5
:1092E000804F3FF403AF7F4B1B68032B7FF7FEAE2D
:1092F0007D4BD3F80465794B1888FFF78DFC054644
:109300007A4B1B685888FFF799FC734B1B880393B3
:1093100002900195764B0093334640F22522754921
:10932000042006F021FCE1E6002304930593069354
:10933000079308930993684B1C882046FFF775FC38
:1093400002464FF00003214604A8FFF7E7FD04465C
:10935000634B1B6813F4804F3FF4C8AE614B1B682E
:10936000032B7FF7C3AE604BD3F804755A4B1E88AE
:109370003046FFF75AFC05465C4B1B685888FFF7E0
:109380005DFC039602900195594B00933B464FF4C8
:1093900010725849042006F0E7FBA7E64E4B1C88E4
:1093A0004E4B1888FFF741FC01462046FFF7E6FDCB
:1093B00004464B4B1B6813F4804F3FF497AE494B68
:1093C0001B68032B7FF792AE474BD3F80465434BE2
:1093D0001888FFF72AFC0546444B1B685888FFF79E
:1093E0002DFC3D4B1B88039302900195424B00934B
:1093F000334640F25A223F49042006F0B5FB75E699
:10940000354B1C88354B1888FFF706FC0146204673
:10941000FFF7B4FD0446324B1B6813F4804F3FF452
:1094200065AE304B1B68032B7FF760AE2E4BD3F835
:1094300004652A4B1888FFF7EFFB05462B4B1B688A
:109440005888FFF7FBFB244B1B8803930290019580
:10945000294B0093334640F265222649042006F04A
:1094600083FB43E61C4B1C882046FFF7D5FB0146D7
:109470002046FFF783FD0446194B1B6813F4804F09
:109480003FF434AE174B1B68032B7FF72FAE164B00
:10949000D3F80475104B1E883046FFF7BDFB054618
:1094A000124B1B685888FFF7C9FB03960290019581
:1094B000114B00933B4640F275220E49042006F002
:1094C00053FB13E60D4A40F27D21052013F0BAFB51
:1094D0000DE6FFF79BFD13E69E320020A032002030
:1094E000242E0020202E0020001001400C2E0020F1
:1094F0007C4704004F460400C44704002046040093
:1095000008B5FFF78DFD08BD08B5FFF771FD024BEB
:109510001B68984708BD00BFB432002000B583B077
:109520001C4B1B681A789AB14A2A11D041680088EE
:10953000FFF742FC28BB174A1368191D1160164A31
:10954000032111701B794A2B18D0FFF769FD1AE02F
:10955000124B1B6813F4804F15D0114B1B68012B65
:1095600011DD104BD3F8043501920F4A009240F2FE
:10957000AB220E49022006F0F7FA04E0FFF7C4FF21
:1095800001E0012802D003B05DF804FBFFF73EFDC7
:10959000F9E700BF0C2E0020BC320020242E002052
:1095A000202E0020001001400C4804004F4604000B
:1095B00000B589B04FF6FF73ADF81E30ADF81C3022
:1095C00001238DF81430ADF816000DF11E0105A829
:1095D0000EF08AFDE8B907A9BDF816000FF0B8F93A
:1095E000E8B9BDF81C0015F059FEF0B9BDF81E1021
:1095F000BDF81C0015F008FEE8B91B4B1B6813F4FE
:10960000804F03D0194B1B68032B1ADC09B05DF89F
:1096100004FB174A40F29D2113F014FBDBE7144AC8
:1096200040F29E2113F00EFBDBE7114A40F2A1212C
:1096300013F008FBDAE70E4A40F2A22113F002FB16
:10964000DBE70C4BD3F80435BDF81E200292BDF8C1
:109650001C200192084A009240F2A32207490420EC
:1096600006F082FAD2E700BF242E0020202E002030
:109670002046040000100140404804004F4604000A
:1096800030B583B0002837D1224B1B6813F4804FCC
:1096900003D0214B1B68032B13DC204B1B8843B3E7
:1096A0001C4B1B6813F4804F03D01B4B1B68032B10
:1096B00013DC1A4A1388013B1380FFF7B1FC03B097
:1096C00030BD174BD3F80435164A009240F2D3222E
:1096D0001549042006F048FADFE7114BD3F80435AA
:1096E000124A009240F2D7220F49042006F03CFAB9
:1096F000DFE7FFF78BFCE2E70C4615460228DED1D8
:1097000021B129462046FFF709FFD8E7784600F047
:1097100069FCF6E7242E0020202E0020B83200201D
:1097200000100140784804004F460400A44804009B
:1097300030B583B0079D3E4C2468247804BB3D4C73
:1097400020803D4C20803D4801803D493D48C86017
:10975000032008703C490A603C4A1380BDF8182079
:109760003B4B1A800024324B1C600E2C23D8394B03
:1097700053F83410284619F05CFEB0B10134F4E718
:10978000354B1B6813F4804F27D0344B1B68002BDC
:1097900023DD334BD3F80435324A009240F2EF22F6
:1097A0003149012006F0E0F917E02A4B03EBC4042D
:1097B00062681F4B1A601E4B1B6883B1264B1B68E7
:1097C00013F4804F03D0254B1B68032B20DC194B6F
:1097D0001888FFF7EDFEFFF723FC03B030BD1E4BEA
:1097E0001B6813F4804F03D01C4B1B68002B03DC59
:1097F000784600F0F7FBE1E7194BD3F804351B4A34
:10980000009240F207321849012006F0ADF9EFE767
:10981000134BD3F80435074A12880192144A009278
:1098200040F20B321049042006F09EF9CFE700BF4A
:109830000C2E0020A03200209E320020B8320020E2
:10984000BC32002001950200D83200209C3200205A
:10985000AC320020D04E0400242E0020202E002008
:1098600000100140B04804004F460400E4480400E2
:109870001049040038B50C46054628B144B1064BE2
:109880001D60064B1C6038BD784600F0ABFBF5E769
:10989000784600F0A7FBF2E7B4320020B032002097
:1098A00070B584B0064600240E2C12D80B4B53F82A
:1098B0003450284619F0E4FD6A4681B2284605F086
:1098C0001BFA04226946304619F024FD10B1013418
:1098D000EAE70025284604B070BD00BFD04E040062
:1098E00070B598B0002401E00134E4B20E2C27D802
:1098F0002F4B53F83450284619F0C2FD14AA81B2F8
:10990000284605F0F9F9149A18AB03EB840343F8E1
:109910004C2C284B1B6813F4804FE5D0264B1B685A
:10992000062BE1DD254BD3F8043502920195244A3C
:10993000009240F235322349072006F015F9D3E7AB
:1099400000252DE00134E4B20E2C28D818AB03EB2F
:10995000850353F84C2C18AB03EB840353F84C3CB1
:109960009A42EFD1134B1B6813F4804FEAD0124B8D
:109970001B68002BE6DD114BD3F8043503920C4A2B
:1099800052F83400029052F8352001920E4A0092AB
:1099900040F23F320B49012006F0E6F8D2E73546A7
:1099A0000D2D03D86E1CF6B23446CDE718B070BD4D
:1099B000D04E0400242E0020202E00200010014054
:1099C0002C4904004F4604005049040008B5064BDA
:1099D0001B681BB906E0044B1B68984711F06EF931
:1099E0000028F8DA08BD00BFDC32002010B50C46B4
:1099F000144B1860144A0121144819F00DFBA0B94A
:109A0000610CE00341F26F7200238B4208BF824277
:109A100010D24FF47A72002319F076FB014600222F
:109A20000B4819F00FFB38B910BD0A4A4A2113F050
:109A300009F9E5E70521F2E7064A4B2113F002F99F
:109A4000F2E700BFDC320020CD9902002050040074
:109A5000E0320020E84F040070B582B005460024D3
:109A60000FE0831B19E02A464FF0A043D3F81035CE
:109A7000D34013F0010F19D104F062F9284B18609C
:109A80000134032C4AD8274B1B5DAB42F8D1244B41
:109A90001E6804F055F9331AE3D4234A9342EBD9F4
:109AA0001F2DE0D905F01F02204BDFE71C4B1E687D
:109AB00004F046F9331A10D41D4A93421AD81D4BAC
:109AC0001B6813F4804F03D01B4B1B68032B06DC71
:109AD0001A4B1B6820469847CEE7831BECE7184BD0
:109AE000D3F80435174A009260221749042006F083
:109AF0003BF8EDE70F4B1B6813F4804FE8D00E4B9B
:109B00001B68032BE4DD0E4BD3F804350F4A00929B
:109B100063220D49042006F027F8D9E702B070BD92
:109B20002C33002084500400A08601000003005064
:109B30007F841E00242E0020202E002028330020A9
:109B4000001001405C5004004E5004006C500400B2
:109B50001F280CD900F01F00064BD3F8043523FA58
:109B600000F010F0010F0CBF0120002070474FF0F3
:109B7000A043F2E70003005070B5054600242646D6
:109B800006E0084B185DFFF7E3FFA04006430134F1
:109B9000032C04D80123A3402B42F8D0F1E7304630
:109BA00070BD00BF8850040008B511B112F016FC5A
:109BB00008BD12F003FCFBE770B5054600240BE07E
:109BC000094B1E5D3046FFF7C3FF80F00101C9B2AB
:109BD0003046FFF7E9FF0134032C04D80123A340EA
:109BE0002B42F8D0ECE770BD8850040010B5144B40
:109BF0001B684BB1134B1868FFF7DEFF104B1C6856
:109C0000013C1C6024B110BD002013F00DF8F1E7F9
:109C10000D4819F039FA09E00C4B1968E14001F0E0
:109C200001010B4B185DFFF7BFFF0134032CEAD88D
:109C30000123A340034A12681342F6D0ECE700BFA9
:109C4000003300200433002008330020303300208C
:109C50008850040070B505460E46002405E03146E4
:109C6000064B185DFFF7A0FF0134032C04D8012335
:109C7000A3402B42F8D0F2E770BD00BF885004002B
:109C80003AB338B50C461346132900D838BD114AEB
:109C900010605B00013B104A1360FFF76DFF0F4B34
:109CA00018600025610CE0034FF47A72002310F570
:109CB000FA70694119F028FA01462A46084819F055
:109CC000C1F90028E2D10121024B1868FFF7C2FF59
:109CD000DCE77047043300200033002030330020DD
:109CE0000833002010B582B012F0E4FA40B100242D
:109CF000ADF804408DF8064001238DF8053009E0E9
:109D000012F088FA0028F2D012F08EFFEFE712F07E
:109D10008BFF0134032C07D801A9094B185D12F001
:109D2000D3FA0028F5D0F2E7064A0121064819F0D7
:109D300073F908B902B010BD12F076FFFAE700BF60
:109D400088500400ED9B02008050040060B310B501
:109D500082B0164A106012F0ADFA40B1144B1B6885
:109D6000ADF804301B0C8DF8063000240EE012F024
:109D700051FA0028F2D012F057FFEFE712F054FF2B
:109D800001210C4B185D12F0B3FB0134032C08D8F1
:109D9000094A01A9074B185D12F030FB0028EFD0EB
:109DA000ECE7002002B010BD0E20704728330020E1
:109DB0007C50040084500400599A020060DF704710
:109DC00069DF704708B503F0DDFC08BD10B588B049
:109DD00012F06EFD00282DD1234B0793079A0692AF
:109DE00000230393049305938DF80C3003A90120FD
:109DF000FFF7E6FF08BB002304930593F8230393C2
:109E0000069A03A9A120FFF7DBFFC8B906A8FFF750
:109E1000D5FF0446069A079B9A4208D0134B1B684D
:109E200013F4804F03D0124B1B68012B0BDCB4B929
:109E300008B010BD12F0F8FECEE712F0F5FEDAE73A
:109E400012F0F2FEE2E70B4BD3F8043501920A4A16
:109E50000092AB220949022005F086FEE7E7204682
:109E600012F0E2FEE4E700BF002E0020242E0020C6
:109E7000202E002000100140D0500400B6500400F5
:109E80000620704700B587B044F20103984262D0C3
:109E90001BD8012836D041F20103984276D1474BB6
:109EA0001B6813F4804F36D0454B1B68002B32DD06
:109EB000444BD3F8043502920191434A0092632245
:109EC0004249012005F050FE25E044F20203984289
:109ED0005CD13A4B1B6813F4804F1CD0384B1B6885
:109EE000002B18DD374BD3F8043510680390526807
:109EF00002920191364A009269223449012005F00C
:109F000033FE08E02D4B1B6813F4804F03D02C4B1D
:109F10001B68002B12DC4FF0A0434FF4F032C3F863
:109F20001825C3F80C25EFF3108372B64DF6AD6C0F
:109F3000284B1B78002B3ED030BFF9E7214BD3F8DC
:109F4000043502920191244A009260221F490120A7
:109F500005F00AFEDFE7194B1B6813F4804FDAD0D7
:109F6000174B1B68002BD6DD164BD3F80435106851
:109F7000049050680390029192680192174A0092EF
:109F800073221249012005F0EFFDC4E70B4B1B685B
:109F900013F4804FBFD00A4B1B68002BBBDD094B6D
:109FA000D3F8043501910E4A00927B220749012023
:109FB00005F0DAFDAFE707B05DF804FB242E0020C2
:109FC000202E00200010014064510400365104008E
:109FD00088510400102E002048510400A8510400AC
:109FE000CC51040000B583B0014600230093054B1B
:109FF00001936A4644F20200FFF744FF03B05DF8A4
:10A0000004FB00BF483A040010B40346044C006847
:10A0100059689A68DB680FC45DF8044B704700BF4D
:10A02000343300200D4B0E4A92E8030083E803000E
:10A0300003F108020B4903C982E8030093F90620E3
:10A0400002F00F0242F040029A7193F9082002F0E8
:10A050003F0242F080021A72704700BF3433002082
:10A0600060000010A4000010004870473433002046
:10A0700000231F2B09D8074901EBC30000224280AF
:10A08000426001F833200133F3E7034B00221A60EA
:10A09000704700BF443300204434002030B40546EC
:10A0A0000F4B1B6800240AE01F230E4A12F83300EE
:10A0B000A0B102EBC3025288AA4207D001341F2C80
:10A0C0000BD85A1E002BEFD01346EEE7054A02EBE1
:10A0D000C30252688A42F1D100E0002030BC7047D0
:10A0E000443400204433002030B40A4A13680A4C38
:10A0F00004EBC30568806960012104F833100B4448
:10A100001360202B01D030BC7047134600221A6028
:10A11000F9E700BF4434002044330020F0B4144673
:10A120001D46002300E00133072B0ED81A01084911
:10A130008A5A8242F7D101EB0312D2E90267AF4299
:10A1400008BFA642EFD1012000E00020F0BC70471C
:10A150004834002030B4C1698269C3880D0A0C06F6
:10A16000C2F30C01994216D25B1A1344A3F50053B3
:10A17000E41845F10005094A1368591C116003F001
:10A180000703808A064A190102EB03135052C3E900
:10A19000024530BC70475B1A1344E9E7C83400201D
:10A1A00048340020C37D002B42D0C3780A7802F0E7
:10A1B000800203F07F0313430B7002780B7803F0E7
:10A1C0007F0343EAC2130B700378002B41D030B4F5
:10A1D0008378082B14BF002201224B7803F07F0301
:10A1E00043EAC2134B70C58803F08003C5F386149D
:10A1F00023434B708A7802F0030242EA8502D2B20E
:10A200008A70057A02F0FC02C5F3C10422438A7009
:10A21000CB7803F01F0343EA4513DBB2CB70427ADD
:10A2200003F0E00302F01F021343CB7030BC704711
:10A23000C3780A7802F0BF029B0103F04003134386
:10A240000B70027903F0C00302F03F0213430B705E
:10A25000B3E770470023032B31D810B402E0013379
:10A26000032B28D8C3EBC302164C04EB021292F85E
:10A270004820012AF3D1C3EBC30204EB0212948AF3
:10A28000C2899442EBD1C3EBC3020E4C04EB021221
:10A29000D2888A42E3D1C3EBC30204EB0212B2F8C4
:10A2A000582012B1848AA242D9D1C3EBC303054816
:10A2B00000EB031000E000205DF8044B7047002025
:10A2C000704700BFF4340020002300E00133032B6B
:10A2D00016D8C3EBC3020B4901EB021292F84820D7
:10A2E000022AF3D1C3EBC30201EB0212918A828AE4
:10A2F0009142EBD1C3EBC303024800EB031070475C
:10A3000000207047F434002008B90420704708206A
:10A31000704730B403460C460978C1700021416291
:10A32000A1680B2903D8217BF9B1012100E00121AB
:10A3300019700020987029B1A1680731C908013946
:10A34000597218720121D97503F10C0561692069F0
:10A3500085E80300E1899982A1691962217F9975D5
:10A36000216AD9629A6230BC70470021E0E70000A0
:10A370000021164B1B688B4226D90023144A02EB9E
:10A38000C10252689A421DD910B4114A52F83120C4
:10A3900002EBC30412F8332082420DD001330C4A81
:10A3A00002EBC10252689A42EFD80131074B1B6899
:10A3B0008B4205D90023F2E760685DF8044B7047D3
:10A3C0000020FAE70131D4E700207047CC340020A8
:10A3D000D034002070B58CB006460D4614462C22B1
:10A3E000002101A818F0F2FF0F238DF80430ADF81A
:10A3F00008604FF0000365F300038DF80A308DF814
:10A400000B4001A801F0F6F90CB070BD30B58DB06D
:10A4100005460C462C22002101A818F0D7FF102376
:10A420008DF8043002958DF80C4001A801F0E2F996
:10A430000DB030BD00B58DB010B913F1020F06D1CB
:10A44000074B186804F088FA0DB05DF804FB012191
:10A450008DF804100293039201A801F0CBF9EFE705
:10A46000D8340020F8B5069C002960D01E460F465F
:10A4700015685168D2F808C0D368E5602161C4F856
:10A4800014C0A36115695169E561216200236370FD
:10A490000278D20922705AB30423BB4249D8E17D25
:10A4A00041B3037803F07F03E3700023A3709AB1F4
:10A4B00043789B0103F4FE53827843EA9203E380DE
:10A4C0008378DB0003F01803C27843EA5213237247
:10A4D000C37803F01F036372002363623378032B96
:10A4E00021D83278144B53F82230E3620020F8BDB3
:10A4F0000123D2E70178C1F38011E170017801F006
:10A500003F01217142B190F90130002B02DB04239D
:10A51000A370CCE70823FBE70421A1700B44BB42E6
:10A52000C5D90920E3E77846FFF75CFDD9E70920A4
:10A53000DDE70920DBE700BF6053040070B50C467F
:10A540001D4603789BB104263244A26000F10C033F
:10A550002360836A6360C36AE36000232374204638
:10A5600004F062FD10B963691E442E6070BD0126BF
:10A57000EAE72DE9F0418EB00D4616461C468046AE
:10A5800000282DD0002D2FD0002C31D0636A02334B
:10A59000059304F10C00E378002B2DD00121A27863
:10A5A00001AF3B46082A14BF0022012204F019FB28
:10A5B0000697CDF81C80B2B2ADF820200B9515445B
:10A5C0000C95A3788DF83430237B022B16D0002312
:10A5D000ADF8283005A804F0FCFA0EB0BDE8F08113
:10A5E0007846FFF7FFFCCDE77846FFF7FBFCCBE7AB
:10A5F0007846FFF7F7FCC9E70221D0E723692BB1C2
:10A60000236909931023ADF82830E3E77846FFF774
:10A61000E9FCF5E72DE9F04188B004460D46C37D1D
:10A62000002B3CD0082605FB06F8637AAB4238D0F5
:10A63000257201AB324602A92046FFF77FFF07468D
:10A6400048BB4DB994F8533033B9A369C3F30C0335
:10A65000E380012384F85330E37D7BB994F85230D2
:10A6600063B91DBBE06EB4F84A10A27823468A1A7B
:10A670000146FFF77EFF012384F8523007992046F8
:10A68000FFF790FDE16E32464144019818F075FEE7
:10A6900002A804F0EFFC384608B0BDE8F0810C26B3
:10A6A000C1E7B4F84A60A6EB0806C1E77846FFF7B1
:10A6B00099FCD7E770B505460E4609B100230B603B
:10A6C00095F85040002104E0631C85F850300134B7
:10A6D000E4B26B7AA34210D3EA6C0123A3401A427E
:10A6E000F5D121462846FFF795FF014628B9002EEF
:10A6F000EAD0336801333360E6E7084670BDF0B551
:10A7000089B004460E46154683789A18C37D63B116
:10A710000B239A4221D801AB02A92046FFF70EFF76
:10A72000074620B1384609B0F0BD0F23F1E707997D
:10A730002046FFF737FDE37D43B12A4631460198B5
:10A7400018F01BFE02A804F095FCEBE723462A460E
:10A7500001993046FFF70DFFF4E70927E2E7000013
:10A7600010B5044690F84830012B0CD103F0E8FAFC
:10A77000237B012B0BD0094BD968014404F1300035
:10A7800003F0AAFA10BD7846FFF72CFCEEE7A17D96
:10A79000024BDA681B6903FB0121EEE7DC34002081
:10A7A00030B583B0002403E02846FFF7D9FF013419
:10A7B000032C18D8C4EBC4030C4A02EB031393F820
:10A7C0004830012BF3D100230193C4EBC40502EB05
:10A7D000051501A92846FFF76DFF0428E4D0019B69
:10A7E000002BE4D0E0E703B030BD00BFF43400201C
:10A7F00038B5044690F84830022B09D1064B1D6845
:10A8000003F09EFA411904F1300003F065FA38BDF7
:10A810007846FFF7E7FBF1E7DC34002038B5044663
:10A8200090F84830022B10D10A4B5D7D5A689B6826
:10A8300003FB052503F084FA411904F1500003F0ED
:10A840004BFA012384F8683038BD7846FFF7CAFB1D
:10A85000EAE700BFDC34002010B50446808A02F02D
:10A860000BFE01281CD1237BE3B194F91620002AAA
:10A870001ADBE27D4AB1022B18D094F90330002B89
:10A8800016DBA378B3B900200BE0E2780AB9012BFC
:10A8900012D1237893B9A378042B11D1002000E0C2
:10A8A000102010BD1020FCE70720FAE71020F8E781
:10A8B0000720F6E70720F4E70720F2E70020F0E79B
:10A8C0000720EEE738B5044603784BB1C388C26968
:10A8D0008169808A06F08AFC054645B9284638BD5C
:10A8E000C2698169808A06F07BFC0546F5E7E1696B
:10A8F000002201F00101A08AFFF76CFDEEE70000E5
:10A900002DE9F04780460E4617464B1EDBB2012B61
:10A910000FD8B7F5C07F10D80024032C1AD8C4EB89
:10A92000C403314A02EB031393F848304BB10134AE
:10A93000F3E77846FFF756FBEBE77846FFF752FB65
:10A94000EAE7C4EBC40502EB0515384608F08DFFB5
:10A95000E86600E000255DB3EB6E002B42D0434675
:10A960002C4608F1300ED3F800C058689968DA68B0
:10A97000C4F800C06060A160E26010331034734519
:10A98000F1D10023EB64A5F84A70012E13D06FF0CB
:10A990000103AB62002385F86830144BAB652D666C
:10A9A000134BAB632D64012002F018FA85F8486060
:10A9B0002846BDE8F0870F4B1B7D85F851300023FA
:10A9C00085F8523085F8533085F85030D8F8282073
:10A9D0006A65A5F858306FF00103AB62064BAB63B4
:10A9E0002D64E0E71D46E3E7F4340020FFB30200E6
:10A9F00049AD0200DC34002095AD020000B585B001
:10AA000000228DF80F20A0B10B46024602320A60E8
:10AA10000DF10F01184604F0E0F89DF80F3043B136
:10AA20000C4B1B6813F0040F03D00B4B1B68032B5C
:10AA300004DC9DF80F0005B05DF804FB074BD3F86C
:10AA40000435074A009240F215420649042005F0F9
:10AA50008BF8EEE7242E0020202E0020001001406D
:10AA6000185204000C5204002DE9F04391B0054641
:10AA70000E4614461F46D0F8188003784BB1C388A1
:10AA8000C8F30C029A4230D29B1A4344A3F50053F8
:10AA9000AB6105F10C00EB7853B30121AA780DF1FD
:10AAA00030094B46082A14BF0022012204F099F80D
:10AAB000C5F81880CDF810900596AB78E21A92B2DE
:10AAC000ADF8182032440A9209978DF82C300023F3
:10AAD000ADF82030EB78002B40D02B7B022B09D037
:10AAE00000236B620193029324E09B1A4344CFE757
:10AAF0000221D3E71023ADF820302B690793EFE74D
:10AB00000134012C14D810AB03EB840353F83C0C34
:10AB100070B103A9FFF772FF0028F1D010AB03EB6F
:10AB2000840454F83C3C6B62002011B0BDE8F08313
:10AB3000019B3BB102AB01AA2979286A0EF078F992
:10AB40000024DEE72B7B022B2CD105F10C01E889D8
:10AB50000EF028FA0028C0D10520E6E72B7B012B58
:10AB600001D00520E1E7EB89ADF80430AB8AADF800
:10AB700006300024012C13D82946002341F8243F35
:10AB800010AB03EB440333F83C0C0EF076F903A949
:10AB9000686AFFF733FF08B90134EBE70020C4E728
:10ABA0000520C2E70520C0E770B5F0B00E46144698
:10ABB0001D4610AB0A4601462046FFF755FF50B12F
:10ABC000214B1B6813F0040F03D0204B1B68052B8F
:10ABD0002DDC70B070BD2046FFF774FE0028F8D160
:10ABE00003AB01228DF80C20A28AADF80E200022C2
:10ABF00004928DF8142010AA0692A178711AADF86B
:10AC00001C1008AA93E8030082E803000AAB21693C
:10AC1000E06883E80300A37D8DF83830236A0C9345
:10AC2000636A0D930F9505A800F0E4FDD1E7084B8A
:10AC3000D3F80435074A009240F203720649062011
:10AC400004F092FFC5E700BF242E0020202E002034
:10AC5000001001402C5204000C52040010B50446B0
:10AC6000C06E08F006FE04F1300003F01DF894F801
:10AC70004830022B0AD070220021204618F0A6FB93
:10AC8000002084F8480002F0A9F810BD04F150003B
:10AC900003F00AF8EFE710B58CB0044690F848309E
:10ACA000012B0FD101238DF80430636D029303F063
:10ACB00047F8039001A800F09DFD2046FFF7CEFF66
:10ACC0000CB010BD7846FFF78DF9EBE730B585B0D5
:10ACD0000D460446A8B194F84830022B15D02946F9
:10ACE000606DFFF793FB2046FFF7B8FF114B1B6821
:10ACF00013F0040F03D0104B1B68032B09DC05B0C5
:10AD000030BD7846FFF76EF9E5E72046FFF722FAF7
:10AD1000E5E70A4BD3F8043594F8482002950192F0
:10AD2000074A009240F2F3120649042004F01CFF87
:10AD3000E5E700BF242E0020202E00200010014057
:10AD4000585204000C52040008B508460021FFF7D1
:10AD5000BDFF08BD08B5037B012B02D0FFF79BFFA9
:10AD600008BD0121FFF7B2FFFAE7000008B590F82F
:10AD7000513053B1013B80F85130002380F85030FE
:10AD8000034B186803F0E8FD08BDFFF7E3FFFBE79E
:10AD9000D834002010B50C4691F84830012B03D16F
:10ADA0002046FFF7E3FF10BD7846FFF71BF9F7E7F2
:10ADB000062976D1F0B585B015460678B20102F4C1
:10ADC000FE5241788478C3781B0443EA0463047913
:10ADD00043EA042344791C4376B242EA91012846AF
:10ADE000FFF738FA0746E0B1002E2FDBC289A98AA7
:10ADF0008A422BD02B4B1B6813F0040F3ED02A4BFA
:10AE00001B68012B3ADD294BD3F8043502910192DE
:10AE1000274A009240F27D622649022004F0A4FEF7
:10AE20002CE0204B1B6813F0040F27D01E4B1B682F
:10AE3000012B23DD1D4BD3F804351F4A009240F24D
:10AE400079621C49022004F08FFE17E0002E17DB08
:10AE5000FD6C2543FD64BCB13B78D3B17B7A5A1CB1
:10AE600001239340013B9D4217D0002187F85010E9
:10AE70003846FFF71FFC3846FFF772FC05B0F0BDFF
:10AE8000AB8AA7F85830E3E703213846FFF71EFFE7
:10AE9000F4E77846FFF7A6F8E0E73846FFF7FBFE51
:10AEA000ECE77047242E0020202E002000100140E7
:10AEB000AC5204000C5204007C5204002DE9F04115
:10AEC0008AB007460E4614461D461046FFF7FAFCA8
:10AED00050B994F80380B8F1000F08D12B462246F0
:10AEE00031463846FFF764FF0AB0BDE8F0814046BE
:10AEF000FFF73EFA02460028F6D08DF80480236A58
:10AF00000793A38AADF8123005AB2169E06883E8A6
:10AF10000300A37D8DF820300297039623788DF8E7
:10AF20001030E36A0993294601A89047DCE710B581
:10AF3000547814F0010F03D0D47D14B1FFF7BEFF95
:10AF400010BDFFF731FEFBE708B501390130FFF70F
:10AF5000EEFF08BDF0B5C7B00F4616468278324402
:10AF6000C37D2BB14FF4807393427CD3002303E065
:10AF70004FF4C073F8E70133032B1AD8C3EBC304B3
:10AF80003B4D05EB041494F848100129F3D1C3EBB1
:10AF9000C30105EB01118C8A818A8C42EBD1C3EB92
:10AFA000C30105EB0111CC89C1898C42E3D108258D
:10AFB00052E00121FFF7A4FC0446002855D0324698
:10AFC0003946C06E18F0D9F90023459345A92046AB
:10AFD000FFF770FB054608B1042840D1459B0BBB29
:10AFE000244B1B6813F0040F35D0234B1B68032B35
:10AFF00031DDB4F84A70802F28BF80270023BB4280
:10B0000014D2E26ED25C1D490D68100959002E5C05
:10B0100004A800F8136002F00F020131AA5C425448
:10B020000133ECE72046FFF79BFBD9E704AA002396
:10B0300002F8173003F1804303F58833D3F8043561
:10B0400002920F4A01920F4A00924FF4AC620E49ED
:10B05000042004F089FD0025284647B0F0BD2046B5
:10B06000FFF7FCFDF8E70925F6E70425F4E700BF44
:10B07000F4340020242E0020202E0020282E002032
:10B08000F0520400643904000C52040070B5044608
:10B090000D461646FFF7E0FB30B923782BB1324658
:10B0A00029462046FFF756FF70BD32462946204606
:10B0B000FFF725FBF8E7000038B504460D46CB69DD
:10B0C0005B780371CB691B7883F00103C370CB6994
:10B0D00043628B8A0B2B07D8CB7A002B35D10B7BA5
:10B0E000012B02D0002300E001232370002B31D07C
:10B0F000287B02282BD0FFF707F9A070AB8A034406
:10B100000B33174A82FB03235B10013B637200235E
:10B1100023720023E37504F10C0395E8030083E830
:10B120000300AB6923622B89A382AB7AA3752B6AD8
:10B13000A362DF23E36228460DF062FF20B12B7883
:10B14000012B0AD0FF23E36238BD0123CDE7054B75
:10B15000987DD0E70423A370DBE72023F3E700BF4B
:10B16000ABAAAA2ADC34002010B54FF4E07200210B
:10B17000134818F02BF906F005F80024114B1C6059
:10B1800080222146104818F021F9104B104A1A600D
:10B19000104A5A604CF250329A600F49D9601A61D5
:10B1A00004221A759C7508225A750C4803F0B4FBEA
:10B1B0000B4B18600B4B1C600B4806F0DDFA10BD02
:10B1C000F4340020C834002048340020DC3400204F
:10B1D00080969800F049020020A10700F1B3020018
:10B1E000D8340020CC34002035A4020008B505F086
:10B1F000E9FF08BD98B110B58CB00446036983B16E
:10B20000C36983B1836983B101466846FFF754FF80
:10B21000A28A21696846FFF739FF0CB010BD0E20E5
:10B2200070470E20F9E70E20F7E70E20F5E7000043
:10B2300058B310B590B00A46044643683BB38369DF
:10B240003BB3014604A8FFF764F8134B1B6813F0E7
:10B25000040F03D0114B1B68062B06DCA268616843
:10B2600004A8FFF713FF10B010BD0D4BD3F8043541
:10B270002278A169029101920A4A009240F60502E1
:10B280000949072004F070FCE8E70E2070470E2003
:10B29000E9E70E20E7E700BF242E0020202E002043
:10B2A00000100140005304000C520400037B012BEA
:10B2B00001D00020704730B591B004460D46334BA5
:10B2C0001B6813F0040F03D0314B1B68032B41DCC8
:10B2D00004A900230593CDF81730E288C2F3861045
:10B2E00092008DF811202A0E8DF812202A0C8DF86C
:10B2F00013202A0A8DF814208DF815506278022A3E
:10B300000CBF80221A4642EA00028DF810204FF04E
:10B31000060209924FF001028DF82C20A28AADF8A6
:10B320002E200C938DF81C300891226A0D928DF816
:10B330002830E36A0F9319D0E389ADF82A30A37D52
:10B34000F3B98DF838306FF0010107A8FFF770FFEF
:10B3500011B030BD0F4BD3F804350F4A009240F2C4
:10B3600063220E49042004F0FFFBB1E70DF10E014A
:10B3700003A80DF033FEBDF80C30ADF82A30DEE73F
:10B38000074B5B7D8DF83830DDE700BF242E0020B1
:10B39000202E0020001001402C5304000C52040009
:10B3A000DC34002090F84830022B00D0704710B5F4
:10B3B000044690F86830022B00D010BDC16CFFF736
:10B3C00075FF0028F9D1002384F86830F5E7000004
:10B3D00010B5002407E0C4EBC4021301034818446D
:10B3E000FFF7E0FF0134032CF5D910BDF434002041
:10B3F00008B5FFF7D5F9FFF7EBFF012008BD10B541
:10B400000C4691F84830022B06D1022384F86830AC
:10B410002046FFF7C7FF10BD7846FEF7E3FDF4E7CF
:10B42000F0B583B00446C5698269C3882F0A2E0629
:10B43000C2F30C05AB4232D95B1B1344A3F5005396
:10B44000F61847F1000732463B46A08AFEF766FE33
:10B45000002840F08B802046FEF736FF054648B3B3
:10B46000D0F81CC08269C3884FEA1C214FEA0C60E7
:10B47000C2F30C0C9C4515D2A3EB0C031344A3F5AB
:10B480000053C01841F10001B94208BFB0420DD3CA
:10B490008F4208BF864230D3284603B0F0BD5B1B05
:10B4A0001344CDE7A3EB0C031344EAE70521284638
:10B4B000FFF70CFCE388E269A169A08A05F068FF48
:10B4C000E8B9627A531CE17D99B3082202FB03F2CA
:10B4D00089B34FF48073934230D302212046FFF7A3
:10B4E0000FFA05460028D7D100212046FFF7DEFEDF
:10B4F00002210020FEF78AFFCEE70025CCE7E38893
:10B50000E269A169A08A05F0BBFF60B1237863B14D
:10B51000617A4B1C0121994001392046FFF7C6FE94
:10B520002046FFF7CFF90025B6E77846FEF75AFD2B
:10B53000EEE70C22CAE74FF4C073CCE70C4B1B6854
:10B5400013F0040F03D00B4B1B68002B01DC00250C
:10B55000A2E7094BD3F804350192084A009240F261
:10B560007F320749012004F0FFFAF0E7002593E756
:10B57000242E0020202E0020001001403C53040007
:10B580000C5204002DE9F04182B007460E461446E5
:10B5900098461046FFF744FF002846D00546404B2A
:10B5A0001B6813F0040F03D03E4B1B68032B3FDCDA
:10B5B0002846FFF71DF92B7B012B47D0EB6C217A36
:10B5C00001228A40134230D11A43EA64043E237AAE
:10B5D000E27D002A42D04FF0080C0CFB03FC697A94
:10B5E0008B423ED0002A41D00823B34240D1AA6901
:10B5F000A3699A4209D205F10C0E0C340FCCAEE8C7
:10B600000F0094E803008EE80300E86E3246391D0F
:10B61000604417F0B2FEEC6C2B7873B36B7A5A1C53
:10B6200001239340013B9C422BD002B0BDE8F08146
:10B630001D4BD3F80435227A01921C4A009240F245
:10B64000A3321B49042004F08FFAB1E795F8683063
:10B65000002BB3D12846FFF7E1F8AFE74FF00C0C11
:10B66000BBE70CEB0603A5F84A30C0E70C23BCE7A8
:10B6700004212846FFF72AFBD7E77846FEF7B2FCFD
:10B68000CCE7E96C2846FFF711FE43462A46B5F899
:10B690004A10E86EFFF74BFC2846FFF7DFFAC4E7D5
:10B6A000242E0020202E00200010014050530400C2
:10B6B0000C5204002DE9F04190B000284CD00F4608
:10B6C00014461E468046002A48D004AB00933346F9
:10B6D000FEF7C8FE054618B1284610B0BDE8F08157
:10B6E00004A8FFF7B9F805460028F5D10023029316
:10B6F000039302A960880DF055FC28B19DF8113024
:10B7000043F001038DF811302269E168208905F0CA
:10B71000F7FD38B19DF8113003F0FE038DF81130BC
:10B72000002BD9D09DF81130002BD5D013F0010F8C
:10B7300001D0039B08939DF8103033B1334604AA1F
:10B7400039464046FFF71EFFC6E7334604AA39468E
:10B750004046FFF7F9FBBFE70E25BDE70E25BBE727
:10B76000F8B508B30E460546164B1F68F7B93C46B8
:10B77000B4420FD205EBC4035B68D3B115F83400B3
:10B7800015F93430002B16DBB8B1FEF7F1FDB0B976
:10B790000134EDE70C4B43F8375003EBC7035E6011
:10B7A0007B1C084A136002E00E2700E0042738469D
:10B7B000F8BD0E27FBE70B27F9E70F27F7E70F2761
:10B7C000F5E700BFCC340020D0340020084B1968C6
:10B7D00061B110B504E0064804F031F9214624B106
:10B7E0000C680B79002BF9D0F5E710BD704700BF4E
:10B7F000B836002038B5054630B1104B1C68C4B1CE
:10B800000F4B01221A7004E07846FEF7EBFBF4E7D9
:10B8100024683CB12379002BFAD154F8043C284623
:10B820009847F5E7064B1B78022B03D0044B002208
:10B830001A7038BDFFF7CAFFF8E700BFB83600201E
:10B84000B436002010B5044630B100232372211D08
:10B85000034804F0C9F810BD7846FEF7C3FBF4E7CF
:10B86000B836002010B5044658B10A4B1B78013B8E
:10B87000DBB2012B09D8074B02221A700123237275
:10B8800010BD7846FEF7AEFBEFE7211D024804F03D
:10B89000D6F8F5E7B4360020B83600200A88836869
:10B8A0009B5A07339BB223F0030313449BB20288D5
:10B8B000043A934200D900230B80704710B582B040
:10B8C00004468368C91AADF806100DF10601FFF7AA
:10B8D000E5FFBDF80630A068184402B010BD00882E
:10B8E000043880B2704743888268D018D15201234F
:10B8F0008370704782680023937043808380704711
:10B90000073189B221F0030189B2428883889A42C3
:10B9100004D29B1A99421EDC0020704710B59A424F
:10B920000FD90488A41AA14217D98B4217D3032C2C
:10B9300003D98368134404229A7000234380184675
:10B9400004E0826813449B780BB1042010BDFFF71C
:10B95000D1FF0020FAE7042070470020F6E704201A
:10B96000F4E738B504460D468368828813448B4259
:10B9700002D07846FEF736FB0023AB70211D20462F
:10B98000FFF78CFFA288A36813449B78042B00D098
:10B9900038BD0023A380FBE710B50C4683684288BE
:10B9A00013448B4202D07846FEF71CFB0023A370A1
:10B9B00010BD70B5054614460E46002944D0002D32
:10B9C00046D0B6F1005F08D94FF08053D3F80C3160
:10B9D00003F50023B6EB832F0ED3B6F5000F08D97D
:10B9E0004FF08053D3F80C3103F50053B6EB832F9F
:10B9F00002D37846FEF7F6FA631E3344B3F1005FD4
:10BA000008D94FF08052D2F80C2102F50022B3EB96
:10BA1000822F0ED3B3F5000F08D94FF08052D2F821
:10BA20000C2102F50052B3EB822F02D37846FEF7C9
:10BA3000D9FA042C10D92C8000236B80AB80AE6027
:10BA4000043C3480B37070BD7846FEF7CBFAB6E79D
:10BA50007846FEF7C7FAB4E77846FEF7C3FAEAE796
:10BA600038B50446A0B16288A36813449B78012BC3
:10BA700012D0EFF3108572B6A388A16819448B78B1
:10BA8000032B0DD02046FFF735FF05B962B638BD50
:10BA90007846FEF7A7FAE6E77846FEF7A3FAE8E766
:10BAA0002046FFF70BFFA368C31A6380002383704F
:10BAB000EBE72DE9F0410E4614460546D0B1EEB154
:10BAC0006A88AB6813449B78012B1BD024B32846AB
:10BAD000FFF705FFA04221D3EFF3108872B621468D
:10BAE0002846FFF70DFF074680B1B8F1000F16D1C9
:10BAF00062B614E07846FEF775FAE0E77846FEF79E
:10BB000071FADDE77846FEF76DFADFE72146284651
:10BB1000FFF7E9FE3060E8E7092700E0092738462B
:10BB2000BDE8F081F8B50C4615460646E0B1FCB11B
:10BB3000A378012B20D12388AB4221D325B3EFF387
:10BB4000108772B625800223A370F1183046FFF7E4
:10BB5000A5FE7388B288934203D0B26813440022D2
:10BB60009A7007B962B6F8BD7846FEF73BFADEE791
:10BB70007846FEF737FADBE77846FEF733FADAE77E
:10BB80007846FEF72FFAD9E77846FEF72BFAD6E784
:10BB900070B50C46054690B1ACB1EFF3108672B6A5
:10BBA000AA88AB6813449A78042A10D09A78022A9B
:10BBB00015D0032A18D0052006B962B670BD7846A4
:10BBC000FEF710FAE8E77846FEF70CFAE5E7291DDC
:10BBD0002846FFF763FEAA88AB681344E6E7032212
:10BBE0009A7023600020E7E77846FEF7FBF9002013
:10BBF000E2E738B5044680B1EFF3108572B6A0884D
:10BC0000A16801448B78042B0BD08878022814BFDC
:10BC10000020012005B962B638BD7846FEF7E2F98A
:10BC2000EAE72046FFF74AFE0146EEE738B505464B
:10BC300078B1EFF3108472B6A888A96801448878B7
:10BC4000C31EDBB2012B08D82846FFF737FE01469A
:10BC5000F5E77846FEF7C6F9EBE7022814BF0020A7
:10BC6000012004B962B638BD70B50C46064678B1FD
:10BC700094B1EFF3108572B6A378012B10D0032B8B
:10BC800013D121463046FFF76CFE05B962B670BD90
:10BC90007846FEF7A7F9EBE77846FEF7A3F9E8E761
:10BCA00021463046FFF778FEEFE77846FEF79AF92F
:10BCB000EBE710B5EFF3108472B6838881681944FE
:10BCC0008B78042B06D08878B0FA80F0400904B94C
:10BCD00062B610BDFFF7F2FD0146F4E7024B002209
:10BCE0001A769A6002207047BC36002008B5064BD1
:10BCF000986800221A605A609A60DA601A615A6184
:10BD00009A6104F0F9FE08BDBC36002000B585B08C
:10BD10000A4BDB6802228DF8002001934FF4805318
:10BD20000293074A6946012001F0BCFA18B90120C4
:10BD300005B05DF804FB0020FAE700BFBC36002028
:10BD4000DA36002000B585B00A4B1B6802228DF858
:10BD5000002001934FF480530293074A6946012063
:10BD600001F0A0FA18B9012005B05DF804FB00202D
:10BD7000FAE700BFDC360020DA360020164BDA681E
:10BD8000137951795B1A03F57F2303F6FF7302EBF6
:10BD900003339A4205D002F580520F4BDA6003203C
:10BDA000704700B585B00D4B1B6801208DF8000071
:10BDB00001930B4B0393042302930A4A694601F053
:10BDC00071FA18B1002005B05DF804FB024B0122A6
:10BDD0001A760220F7E700BFBC360020DC360020D0
:10BDE000E0360020DA36002000B585B00C4BDA686A
:10BDF0000C4B1B68043301208DF800000192039363
:10BE000040F6FC730293084A694601F04BFA28B9E0
:10BE10000120034B187605B05DF804FB0020FAE71B
:10BE2000BC360020DC360020DA36002000B585B0B4
:10BE30000A4B1B6801208DF800000193084B039307
:10BE400004230293074A694601F02CFA18B901202D
:10BE500005B05DF804FB0020FAE700BFDC360020E7
:10BE6000C8360020DA36002010B584B0104BDA68EE
:10BE70001478104B1B68043301208DF800000193E7
:10BE8000039202940C4A694601F00CFA70B9094B0E
:10BE90001B6804F0FC041C440434054B5C61D96845
:10BEA0000A780A441A61012004B010BD0020FBE7A3
:10BEB000BC360020DC360020DA36002008B500232E
:10BEC0000A2B09D8064A52F82320824201D00133B6
:10BED000F6E7044A536002E07846FEF783F808BDAF
:10BEE000E0530400BC36002010B5214BDB6853B191
:10BEF0001F4B1B7E5BB91E4B5B680A2B26D978460D
:10BF0000FEF770F822E07846FEF76CF8F0E7784626
:10BF1000FEF768F8EFE7164A5368013353600A2BBF
:10BF200021D97846FEF75EF81DE0114B00225A60D9
:10BF300019E00F4B1B7E1BB10D4B02221A7012E051
:10BF4000FFF7D4FE0FE00A4B1B7E83B9084B5A68FB
:10BF5000084B53F82230984704460228E9D00328BA
:10BF6000E3D00128D7D0012CEDD0032CEBD010BDAD
:10BF7000BC360020E0530400104B1B681B685A1E9F
:10BF800012F1030F18D8C3F30B020AB10020704757
:10BF900010B50B4AD3600023137653760124147036
:10BFA00093600848FFF78AFF0749204601F068F9C7
:10BFB000FFF79AFF204610BD00207047DC360020B6
:10BFC000BC3600200DBD0200CDBF020008B50B78C5
:10BFD000032B06D00B4B1B78012B06D0022B0BD06A
:10BFE00008BD084B00221A76F4E7064B1B7E002B97
:10BFF000F6D1FFF779FFF3E70B78032BF0D1FFF7CA
:10C0000075FEEDE7BC36002000B585B0174BDB6848
:10C0100018784FF6FF7203F58051184405F062FB63
:10C02000E0B10246114BD9680B780B44984217D007
:10C030000E4B5B7E83B10E4B01208DF80000019208
:10C040000393042302930B4A694601F02BF948B984
:10C050000120064B187606E0074BEDE7012002E0D1
:10C06000012000E0002005B05DF804FBBC36002094
:10C0700010560400DA3600200C56040008B5104BA8
:10C08000DB681878002203F58051184405F02AFB7C
:10C0900008B1012008BD0A4BDA68137951795B1A9F
:10C0A00003F57F2303F6FF7302EB03339A4205D0B7
:10C0B00002F58052024BDA600320EBE70220E9E749
:10C0C000BC360020F0B585B0514BDE68727933790B
:10C0D000591E8A4214D006F580510D780D444D4901
:10C0E0000968081D0F7907449B1A06EB03366B8815
:10C0F000013B9BB247F6FE62934260D92C461AE0A0
:10C100000120434B58767EE07846FDF76BFF15E043
:10C1100024F47F6424F00F0404F5805423781C4435
:10C12000A64247D9A54247D26388013B9BB247F656
:10C13000FE62934211D92388002BE5D0238804EBBB
:10C14000830323F47F6222F00F029342E0D06288DF
:10C15000B2F5FE4FDCD01C46E2E725462FE07846DC
:10C16000FDF740FF15E024F47F6424F00F0404F58C
:10C17000805423781C44A64220D9A5423BD2638830
:10C18000013B9BB247F6FE62934211D92388002BF4
:10C19000E5D0238804EB830323F47F6222F00F02AF
:10C1A0009342E0D06288B2F5FE4FDCD01C46E2E755
:10C1B000254604E0002502E0002500E00025E5B169
:10C1C000144B19686A8801F58051384605F08AFADF
:10C1D000074690B101200E4B18768DF800000195AE
:10C1E0000D4B0393042302930C4A694601F05AF85D
:10C1F00058B92C46CAE70025E1E7B5FA85F56D097F
:10C20000034B5D76012005B0F0BD0020FBE700BFC9
:10C21000BC360020DC36002008560400DA36002048
:10C220002DE9F04186B0644B1B692BB1624B5B6911
:10C2300033B14FF0000846E07846FDF7D3FEF5E74E
:10C240007846FDF7CFFEF4E77846FDF7CBFE15E024
:10C2500025F47F6525F00F0505F580552B781D44E5
:10C26000AF421CD9AC421ED26B88013B9BB247F651
:10C27000FE62934211D92B88002BE5D02B8805EB69
:10C28000830323F47F6222F00F029342E0D06A8896
:10C29000B2F5FE4FDCD01D46E2E72C4600E000245C
:10C2A0001CB100943AE00024FAE700230093019BBC
:10C2B000002B5CD14FF00108002C77D0628847F644
:10C2C000FF739A4272D0B8F1000F73D13A4B5A699A
:10C2D00022F47F6626F00F06B61A06F580561C6912
:10C2E000DF683B797A799B1A07EB033700230193C8
:10C2F0006388013B9BB247F6FE629342D1D9254643
:10C30000B9E77846FDF76EFE23E024F47F6424F05D
:10C310000F0404F58054237823441C46A742C6D951
:10C320002388019A02EB83029642C0D9009B6340A6
:10C3300023F47F6323F00F03002BB8D16388013B04
:10C340009BB247F6FE618B42B1D801922388002B45
:10C35000D7D0238804EB830323F47F6222F00F02FB
:10C360009342D2D06288B2F5FE4FD6D1CDE7124AC1
:10C37000526901208DF808000392009A05920493F7
:10C380000E4A02A900F08EFF70B90B49019B23F001
:10C3900003024B6913444B6114B1074B1C618BE7DB
:10C3A0007846FDF71FFEF8E7002000E0012006B008
:10C3B000BDE8F0810120FAE7BC360020DA36002023
:10C3C00000B585B0274B00221A7040F6F8731B6841
:10C3D000B3F1FF3F09D0B3F1FF3F0CD07BB1B3F114
:10C3E000FF3F37D0A3F580520FE01F4A1268B2F129
:10C3F000FF3FF0D103E01C4A1268002AEFD14FF052
:10C4000080514B690A6902FB03F2A2F58052174B77
:10C410001A60174B1B6813F4801F16D0154B1B684E
:10C42000062B12DD144BD3F8043540F6F871096879
:10C43000B1F1FF3F13D002920191104A009240F2F5
:10C4400076220F49072003F08FFBFFF795FD05B01B
:10C450005DF804FB044B1A68A2F58052D5E7024947
:10C460000968E8E7D836002014100010DC360020F8
:10C47000242E0020202E002000100140AC53040088
:10C480009453040010B50446B0B1104B1B78BBB1F7
:10C490000E4BD968E3685879A3EB0032914211D36F
:10C4A0001A79121A02F57F2202F6FF7203EB0233A9
:10C4B000994209D8012004E07846FDF793FDE4E7AE
:10C4C000002010BD0020FCE70020FAE7BC36002069
:10C4D000024B1878003818BF01207047BC36002086
:10C4E00010B50446124B1B78BBB92378032B18D127
:10C4F0000F4B9C60E268DA600E4B1B78ABB10A22EE
:10C500000B4B5A6000221A76012018705A760A499D
:10C5100000F0B6FEFFF7E8FC10BD7846FDF762FDBF
:10C52000E3E77846FDF75EFDE2E70022E8E700BFBB
:10C53000BC360020D8360020CDBF0200014B186861
:10C54000704700BFDC36002010B5044680B1636838
:10C550001BB123680BB1A36813B97846FDF742FD00
:10C56000A3685A1E134207D10023E360236110BD64
:10C570007846FDF737FDEAE77846FDF733FDF3E748
:10C58000F8B500B30F4604468368F3B1EFF31085A6
:10C5900072B60369C268934211D001684268866826
:10C5A000013E334003FB021117B1384616F0E5FE99
:10C5B00023690133236155B962B62846F8BD05B930
:10C5C00062B60525F9E70E25F7E70925F5E7002509
:10C5D000F3E700000246C0F30B0040BB49B310B4C0
:10C5E00001F6FF710C0B144B0221C3F80415124B1A
:10C5F000D3F80034002BFAD001460AE00E4BC3F802
:10C6000008250D4BD3F80034002BFAD002F58052E8
:10C610000131A142F2D3084B0022C3F80425064B96
:10C62000D3F80034002BFAD05DF8044B704710208B
:10C6300070470920704700BF00E0014010F0030F71
:10C640002FD110B4044611F0030F2CD16AB312F0AD
:10C65000030F2CD19008174B0122C3F80425154B6A
:10C66000D3F80034002BFAD002E004340431104631
:10C67000421E50B10B68B3F1FF3FF6D023600D4B63
:10C68000D3F80034002BFAD0EFE70A4B0022C3F8AE
:10C690000425084BD3F80034002BFAD05DF8044B86
:10C6A0007047102070471020F8E70920F6E70920AE
:10C6B000F4E700BF00E00140094B1B7813F0040FC2
:10C6C00002D00378122B00D07047064B1A68064B35
:10C6D0005A60034B1A786FF382021A70F4E700BFB6
:10C6E00088370020783700201437002010B582B03A
:10C6F00001900C46000C012810D12368094A1360F0
:10C7000009490B7843F001030B705B0883F00103C8
:10C7100003F001031371002002B010BD7846FDF74D
:10C7200061FCEAE7783700208837002010B582B036
:10C7300001900C46000C02280FD12268094B1A60A8
:10C7400022791A71002058719871D871064A1378AD
:10C7500043F00203137002B010BD7846FDF742FCAF
:10C76000EBE700BF703700208837002010B582B09B
:10C7700001900C46000C032806D1054B1868206078
:10C780001B79237102B010BD7846FDF72BFCF4E74E
:10C790007837002010B582B001900C46000C0328B9
:10C7A0000CD1084B2068186022791A71064A137858
:10C7B00043F001031370002002B010BD7846FDF76E
:10C7C00011FCEEE7783700208837002010B582B0E2
:10C7D00001900C46000C042805D1054B03CB2060CA
:10C7E000616002B010BD7846FDF7FCFBF5E700BFC5
:10C7F0007037002010B582B001900C46000C042860
:10C800000BD1084B2068616803C3074A137843F0D3
:10C8100002031370002002B010BD7846FDF7E2FB62
:10C82000EFE700BF703700208837002000B583B0E5
:10C830000190000C032806D1054B00221A601A71E2
:10C8400003B05DF804FB7846FDF7CCFBF4E700BFCE
:10C850007837002000B583B00190000C042806D181
:10C86000054B00221A605A6003B05DF804FB78465D
:10C87000FDF7B8FBF4E700BF7037002000B585B0C6
:10C88000184B1B7813F0400F0FD0164B1B7813F08A
:10C89000040F07D1144B5B6803F500530193B3F108
:10C8A000807F06D905B05DF804FB7846FDF79AFB5A
:10C8B000EBE70E4B1B788DF808300A4A137843F0EB
:10C8C000040313700023ADF80C300323ADF80E30D1
:10C8D00001A9039806F08CF80028E3D07846FDF70C
:10C8E00081FBDFE7883700201437002089370020DC
:10C8F00000B585B00022ADF809200F4B9968019171
:10C900001B7B8DF808300D490B780133DBB20B70BF
:10C910008DF80B30ADF80C200423ADF80E300DEB84
:10C920000301039806F064F810B905B05DF804FB44
:10C930007846FDF757FBF8E71437002089370020C9
:10C9400000B585B00F4B9A6801921A7B8DF80820CC
:10C950001B8AADF809300C4B1B788DF80B30002387
:10C96000ADF80C300423ADF80E300DEB0301039845
:10C9700006F03EF810B905B05DF804FB7846FDF707
:10C9800031FBF8E7143700208937002000B58DB05F
:10C990000B4B1B7B012B0ED0094A926804928DF839
:10C9A0000830039002238DF8043001A8FEF722FF1F
:10C9B0000DB05DF804FB024A9268013A0492EEE77A
:10C9C0001437002008B51D481D4B036000F0D2FE4F
:10C9D0001C4B1B7813F0200F2AD103F00303032B09
:10C9E00014D1194B1968194A916019791173B3F868
:10C9F00005001082DB79164A1370164A12799342A9
:10CA000017D0B1B9114B00221A6007E00F4B00227A
:10CA10001A609A601A731A82FFF76AFF0B4B1A6842
:10CA20005A60084A137843F040031370FFF726FF5B
:10CA300008BD084B1A68054B1A60EFE76437002001
:10CA4000B9C6020088370020703700201437002054
:10CA5000893700207837002010B582B00024ADF867
:10CA600000400123ADF80230009805F0F2FFADF868
:10CA700004400223ADF80630019805F0EAFF02B049
:10CA800010BD000008B5002006F00AF8084B00228F
:10CA90001A605A609A60DA601A61064A137803F0E5
:10CAA000DF0343F040031370FFF7E8FE08BD00BF4B
:10CAB000143700208837002038B50C4D00242C6036
:10CAC0006C60AC60EC602C6101F03AF9084B586086
:10CAD000084A9A60084ADA601C615C61074B1A7860
:10CAE00064F3C3021A706C6038BD00BF14370020B5
:10CAF000F036002059CC02000087930388370020CD
:10CB000008B50C4B1B7813F0100F00D008BD0A4875
:10CB10000A4B036000F02EFEFFF754FFFFF79CFF67
:10CB2000074801F091F8034A137843F0100313709B
:10CB3000ECE700BF8837002008370020B1CD0200A5
:10CB4000F0360020034B1878800880F0010000F0D8
:10CB5000010070478837002010B501F065FE174BC3
:10CB60001B7B1BBB154B9B7B2BBB144B1A8A41F2C7
:10CB700082639A4206D8124B1B7813F0080F05D037
:10CB8000012300E001231BB9082410E00023FAE789
:10CB90000A4B01221A7300241C829A6801329A609F
:10CBA000FFF7A6FE2046FFF7F1FE00E0082401F0A3
:10CBB0007FFE204610BD0824F9E700BF143700208F
:10CBC0008837002010B501F02FFE214B5B7BABB105
:10CBD0001F4B9B7B03BB1E4B1A8A41F282639A4216
:10CBE00006D81C4B1B7813F0080F05D0012300E07A
:10CBF00001239BB1012302E00023FAE700231C4636
:10CC00000BB3134B00225A731B7B4BB1012B0ED07D
:10CC10007846FDF7E7F916E00023F0E70023EEE79A
:10CC2000FFF79AFF78B17846FDF7DCF90BE0084B87
:10CC300000201860586018731882FFF7A7FEFFF7EE
:10CC400057FEFFF71BFE01F033FE204610BD00BF6C
:10CC5000143700208837002008B52C4B1B7BDBB134
:10CC6000012B2ED07846FDF7BDF9284A138A0133EF
:10CC70009BB21382264AA2FB03121209C2EB0212D4
:10CC8000A3EB42039BB2002B3DD0204B5B8A13B138
:10CC9000013B1E4A538208BD1C4B1A8A41F2826333
:10CCA0009A4206D81B4B1B7813F0080F07D00123BC
:10CCB00000E00123002BD8D0FFF784FFE5E7002335
:10CCC000F8E7124B1B8A41F28262934206D8114A5E
:10CCD000127812F0080F14D0012200E00122002A7D
:10CCE000C3D042F2B012934202D9084B01225A73C8
:10CCF000FFF768FF0028C8D1044B5B7B012BB4D140
:10CD0000C3E70022EBE7FFF71BFEBEE71437002066
:10CD1000898888888837002010B5244B1B7B002B1E
:10CD200035D10446214B5B8A2BBB1AB91F4B9B683C
:10CD30008B4205D3FAB11D4B9B6801338B421AD24B
:10CD40001A4B9B682A338B4223D3184B9B7B03BB24
:10CD5000164B996000221A605A601A8242F60651F8
:10CD600059825A731A73FFF7C3FDFFF787FD2046F8
:10CD7000FFF70CFE0DE062B10C4B9B6801338B4258
:10CD800007D10A4B01225A73FFF71CFF01E0012B68
:10CD900000D010BD002AFCD1044B9B688B42F8D117
:10CDA000024B01225A73FFF70DFFF2E71437002000
:10CDB0000378042B00D0704743681B78002BFAD00F
:10CDC00010B58468027E437E012A14BF002201222E
:10CDD000416904F11000FFF79FFF10BD08B538B19D
:10CDE0000D4B01229A730D4A13680133136008BD7D
:10CDF0000A4B1B685BB1094A1368013B1360002BA7
:10CE0000F5D1054B00229A73FFF7DCFEEFE7784679
:10CE1000FDF7E8F8EFE700BF14370020E436002004
:10CE200000B58DB0ADF808008DF8102003910323F4
:10CE30008DF8043001A8FEF7DDFC0DB05DF804FBB1
:10CE4000014B9868704700BF14370020054B1B7BCF
:10CE5000012B02D0034B98687047024B9868013849
:10CE6000704700BF143700201D4B1B7813F0400F94
:10CE700034D070B504460D461A4B1A685B689A4266
:10CE800028D2184B1B7B012B17D0174B9A4216D276
:10CE9000144B1A685B68403B9A4218D2EFF3108635
:10CEA00072B6104A1368591C11602B60FFF7CEFF51
:10CEB000206006B962B6002070BD0C4BE6E7094B56
:10CEC00001225A73FFF77EFE0028E7D1E0E7FFF763
:10CED000D5FCE3E7FFF7D2FC0F20EDE70F2070470A
:10CEE0008837002014370020FFFF7F0000E0FF009C
:10CEF000044B9B68584010F0010F00D0013B1846CE
:10CF0000704700BF14370020014B187B704700BFEB
:10CF1000143700202DE9F041002624E02449BC23E9
:10CF200003FB04F3CA5A0132CA520221284602F016
:10CF30005BFC01370221284602F026FC014679B14C
:10CF40001B4ABC2303FB0423D3F80880B8F1000F6D
:10CF5000E4D0BC2303FB04F3D25A3046C047DDE7DC
:10CF600097B90136F6B2022E1FD83446BC2303FB14
:10CF700006F308330E4D1D4404350221284602F005
:10CF800003FC01460027DAE7284602F095FC082852
:10CF9000E7D1074BBC2202FB0434A368002BE0D08E
:10CFA0000022044930469847DBE70120BDE8F081C4
:10CFB000943700201C54040008B508238373102301
:10CFC000437300F11C0343610323037300F118034F
:10CFD00003610C3002F042FC08BD000008B5037884
:10CFE000012B06D0022B06D07846FCF7FBFF002071
:10CFF00002E0292000E0014808BD00BF084C010004
:10D0000008B50378012B07D0022B15D07846FCF722
:10D01000E9FF4FF4FA730AE08368591A21F0030319
:10D0200003EB9103DB0003EB910303F5FA7307486D
:10D03000984228BF184608BD8368591A090B044B4B
:10D0400003FB01F303F5FA73F1E700BF608501000C
:10D05000084C010038B5044601210C3002F094FB65
:10D06000054678B1084BC4F89C300023C4F8A030C2
:10D070006168FFF7C5FFC4F8A800C4F8AC400123FD
:10D0800084F8B830284638BDA9D1020010B504464E
:10D09000FFF7E0FF20B104F19C000CF045FD00B962
:10D0A00010BD7846FCF79EFFFAE70000F8B505468C
:10D0B0000C46164617680378012B19D11249A1FBBB
:10D0C000043149098B00AC68E41BB4EB810F00D339
:10D0D0001C468CB1686827F00307E968224639448A
:10D0E0003844FFF7ABFA58B933681C443460F8BDD4
:10D0F0007846FCF777FFE1E77846FCF773FFE9E74E
:10D100007846FCF76FFFEFE77D0CCEC7F8B5064613
:10D110000C46154617680378022B17D1114BA3FB59
:10D1200004231B0C1A03B468E41BB4EB033F00D3C5
:10D1300014467CB1706827F0030721463844FFF796
:10D1400049FA58B92B681C442C60F8BD7846FCF7A6
:10D1500049FFE3E77846FCF745FFEBE77846FCF745
:10D1600041FFEFE7EB0661C538B505460C461146B1
:10D170002378012B06D0022B0FD07846FCF732FF24
:10D18000002304E0021D2046FFF790FFA3686868B3
:10D19000984214BF0020012038BD021D2046FFF731
:10D1A000B5FFA368F3E700002DE9F8430F46D1F877
:10D1B000A850254B1B786BB90446A5F5FA7501F10B
:10D1C0000C080121404602F0DFFA064648B14FF054
:10D1D000000924E00CF0E4FC002387F8B830BDE837
:10D1E000F8837846FCF7FEFEF1E70CF0D9FC01214C
:10D1F000404602F0F9FA00237B6087F8B830134B01
:10D20000186801F0A9FB3846FFF740FFE7E7A4EBF9
:10D2100000093046FFF7E2FE4844A8420DD8A5EBCE
:10D22000090231463846FFF79FFF0028DDD101F0A3
:10D23000CDF9B0EB0409ECD5E9E70CF0B1FC3846C8
:10D24000FFF724FFCBE700BF903700208C3700208A
:10D2500010B5084801F060FB074B1860002406E099
:10D26000064BBC2000FB0430FFF7A6FE0134022C65
:10D27000F6D910BD15CF02008C370020943700205E
:10D2800038B504460D46022805D80548BC2303FBE3
:10D290000404A56038BD7846FCF7A4FEF5E700BF9E
:10D2A000943700202DE9F84305460C46174602281E
:10D2B00016D8CCB12378012B1AD0022B3ED163684B
:10D2C000C3F30B03002B31D1A368C3F30B03002B73
:10D2D00030D1A368002B34D17846FCF783FE30E0D0
:10D2E0007846FCF77FFEE4E77846FCF77BFEE1E753
:10D2F000636813F0030F0DD1E36813F0030F0DD132
:10D30000A36813F0030F0DD1A368D3B97846FCF7D7
:10D3100069FE16E07846FCF765FEEDE77846FCF717
:10D3200061FEEDE77846FCF75DFEEDE77846FCF739
:10D3300059FEC9E77846FCF755FECAE77846FCF780
:10D3400051FEEFF3108872B6BC2606FB05F606F117
:10D3500008032A4E1E4404360021304602F014FA17
:10D36000814678B30021304602F03EFA20686168B9
:10D37000A268E368C9F80000C9F80410C9F80820D9
:10D38000C9F80C302FB11D4ABC2303FB05235B8871
:10D390003B801A4ABC2303FB05235A8801325A807A
:10D3A00093F8B83083B9164B1B7813B10024A1460B
:10D3B0000CE0124BBC2000FB0530FFF74BFE814612
:10D3C000002403E0042401E00024A146B8F1000F8A
:10D3D00000D162B6B9F1000F09D0BC2000FB05F006
:10D3E0009830064D284404300CF09EFB10B92046BE
:10D3F000BDE8F8837846FCF7F5FDF8E794370020A0
:10D400009037002038B50446EFF3108572B610B996
:10D41000164B1B6873B18CB1144A13680133136047
:10D42000124B1B68003B18BF0123114A137005B94A
:10D4300062B638BD7846FCF7D5FDECE70B4B1C68AF
:10D44000013C1C6034B1EBE7BC2000FB0420FFF77B
:10D450001DFE0134022CE3D8064ABC2303FB04233F
:10D4600093F8B830002BF4D1EEE700BFC8390020A4
:10D47000903700209437002018B1830B024AD05C0B
:10D4800070470020704700BF2C54040012DF704723
:10D4900000B583B001F098FE40B10C4B1B6813F04F
:10D4A000400F03D00A4B1B68012B02DC03B05DF870
:10D4B00004FB084BD3F804350190074A009275220B
:10D4C0000649022002F050FBF0E700BF242E0020A6
:10D4D000202E002000100140605404005454040029
:10D4E00000B58DB0114B1B78022B06D07846FCF7A7
:10D4F00079FD01200DB05DF804FBFFF723FB18B99F
:10D500000B48FEF79FF9F4E70DF082F8074B032272
:10D510001A702C22002101A815F058FF1D238DF848
:10D52000043001A8FEF766F9E3E700BFD039002018
:10D53000142E002008B50378122B00D008BD044833
:10D54000FEF790F9034B186801F006FAF6E700BF02
:10D55000142E0020CC39002070B58AB00DF09AF856
:10D5600048B3064600238DF8103005AC05460FCDB4
:10D570000FC42B682360727D052A04D9337D03F024
:10D580000F03072B1ED1174B1A688AB104AB039304
:10D59000337DC3F303038DF80430737D062B1BD951
:10D5A000063B8DF8053006F11D03029301A8904754
:10D5B00030460DF04FF80DF089F880F00100C0B250
:10D5C0000AB070BD307D04AB063A06F11D0100F0D3
:10D5D0000F000BF087FDD6E700238DF8053002938E
:10D5E000E4E700BFD439002070B582B0314B1B781E
:10D5F000002B54D10446002855D0067A0F2E01D0B6
:10D60000062E52D106F030F9E06870B1FCF7FCFC50
:10D610000DF10700FFF73AFF0546002840D19DF8BD
:10D620000730012B04D002253AE0FCF7FBFCEFE7C2
:10D63000FCF71EFD00F0F0FA304601F09DF8E078AE
:10D6400000F014F900F09CFE0CF012FA1A480DF0EC
:10D65000D9F80BF0EFFE0BF027FDFFF7F9FD05F011
:10D660008BF900F0E9FC06F0BFF805F05DFE2046FE
:10D6700001F0C4FCFDF778FD04F0D4FBFCF700FCDE
:10D6800008B1062813D10D4801F046F90C4B18607B
:10D690000C4B00221A60074B01221A7000E008258B
:10D6A000284602B070BD0E25FAE70725F8E70546C3
:10D6B000F6E700BFD039002059D50200E1D40200BE
:10D6C000CC390020D439002010B582B0204B1B7813
:10D6D000012B0DD05AB2002A35D0043BDBB2012B0E
:10D6E00033D80CF011FA044628B3204602B010BD1E
:10D6F00001F094FCFDF77AFDFCF7C2FB0446B8B1DB
:10D70000062815D0134B1B6813F4804FEDD0124B35
:10D710001B68012BE9DD114BD3F804350190104A49
:10D7200000924FF4C2720F49022002F01DFADCE7AA
:10D7300001F04EF8D5E7064B02221A700A4B186822
:10D7400001F00AF9D1E70824CFE70824CDE700BFAC
:10D75000D0390020242E0020202E0020001001406F
:10D760008C54040054540400CC39002008B5FDF753
:10D7700041FD08BD08B5FEF765F808BD08B5FEF720
:10D7800071F808BD08B500F0C1FD002008BD704764
:10D79000064A136801331360B3F1704F02D0034B94
:10D7A00018687047134601221A60F8E7D83900203C
:10D7B00010B5044618B100232360636010BD78469D
:10D7C000FCF710FCF7E738B50C46054668B184B1A4
:10D7D00000236360EFF3108372B62A686AB16A6847
:10D7E00054606C6003B962B638BD7846FCF7FAFB4A
:10D7F000EDE77846FCF7F6FBEAE72C60F1E710B5B9
:10D80000044658B1EFF3108372B6206808B142683D
:10D810002260226832B103B962B610BD7846FCF7C7
:10D82000E1FBEFE76260F6E710B5044608B1206857
:10D8300010BD7846FCF7D6FBF9E735DF70470000EE
:10D8400008B54FF0FF30FFF7F8FFBFF34F8F0549E2
:10D85000CA6802F4E062044B1343CB60BFF34F8FFE
:10D8600000BFFDE700ED00E00400FA05072814D82A
:10D87000DFE800F0080C1504110F0A066420704759
:10D8800014207047FA2070471E2070474FF4FA703A
:10D890007047322070474B207047FA20704796201F
:10D8A00070470000024B5868103840B2704700BF04
:10D8B00000ED00E0034600280FDB5B11084A52F838
:10D8C0002330424200F01F0002F01F0258BF5042B6
:10D8D00023FA00F000F00100704700F11F03ECE7AD
:10D8E00000E100E046DF7047F8B504460D464B1EE8
:10D8F000DBB2012B09D8002323616361A361E361DB
:10D900002046FFF7EFFF012016E07846FCF76AFBA0
:10D91000F1E7CA5CCE185200D2B2767842EAD6124B
:10D92000CA5401339BB20E2BF3D9CB7B5B00CB7374
:10D93000002F08DB0130C0B2A8420BD8214611F9F4
:10D94000207F0023EFE794F82F3083F0870384F8DB
:10D950002F30EFE7F8BD2DE9F04190B084460C463A
:10D9600096461F4602F10F084FEA281604AD0068DC
:10D97000DCF80410DCF80820DCF80C300FC50EF0E1
:10D980000F055FEA181302D07DB1002300E00023E9
:10D99000984663B1012104A8FFF7A6FFB8F1000F74
:10D9A0001AD0701E000110230EE00123F0E70221BF
:10D9B000F1E7013B9BB22218D25C10A9194411F87F
:10D9C000101C4A400DF80320002BF2D100250C95C5
:10D9D0000D950E950F9533E0711EADB22A4604EBFE
:10D9E0000111684615F0C9FC80230DF805306B1C49
:10D9F00003E000220DF8032001330F2BF9DD102383
:10DA00000AE0013B9BB21DF8032010A9194411F84C
:10DA1000101C4A400DF80320002BF2D1D6E7013A42
:10DA200092B210AB134413F8100C63189B5C58406F
:10DA300008AB9854002AF2D104A8FFF753FF013530
:10DA4000731EAB4202DD29011022F3E710230AE026
:10DA5000013B9BB210AAD11811F8402C11F8101CF0
:10DA60004A4008A9CA54002BF2D104A8FFF73AFF94
:10DA70000CAC0FCC38607960BA60FB6010B0BDE8C8
:10DA8000F081000010B50446134B1B6893B1416848
:10DA9000114B1B685B68CB1A002B0BDB0E4B1B6812
:10DAA00018465B691BB15A68521A002AF8DB636199
:10DAB000446103E0084B1A6862611C60064A93885F
:10DAC0009BB201339BB2938013B10123237010BD2D
:10DAD0007846FCF787FAF8E7E439002038B50546C0
:10DAE0001CE07846FCF77EFA6369204A1360002345
:10DAF000636193889BB2591E89B29180F3B1A36888
:10DB000003B302232370A36821692846984700F0D5
:10DB100017F905462378DBB2022B17D0134B1B688D
:10DB20001BB3124B1B685B685B1B642B1DD50F4B33
:10DB30001C682378DBB2012BD6D0D2E77846FCF7FD
:10DB400051FADCE77846FCF74DFADAE7E26812B9F9
:10DB500000232370E2E76368134463605B1B642B5C
:10DB6000F9D42046FFF78EFFD8E738BDE43900200E
:10DB700010B50446144B1B68834207D0124B1B6838
:10DB8000D3B15A69A2420ED01346F9E743690E4A4F
:10DB9000136093889BB2591E89B2918063B978460D
:10DBA000FCF720FA08E062695A6107498B889BB24A
:10DBB0005A1E92B28A8013B10023237010BD78469A
:10DBC000FCF710FAF8E700BFE439002008B5064B6F
:10DBD0001B6833B1044B1B680449586800F05CF9BA
:10DBE00008BD00F0B7F9FBE7E439002009DC0200CA
:10DBF00008B500F0A5F8FFF771FF00F0A1F8FFF7F6
:10DC0000E5FF012008BD000008B5024B186800F0D0
:10DC1000A3FE08BDDC39002008B50023064A1370B6
:10DC2000064A13605360064800F076FE054B186004
:10DC300000F078F808BD00BFE0390020E43900208A
:10DC4000F1DB0200DC39002010B50446154B1B78CF
:10DC50009BB900F055FFA0B1BCB1A368CBB123784C
:10DC6000DBB2012B19D0002363612046FFF70AFFC6
:10DC700000F066F8FFF7AAFF10BD7846FCF7B2F98E
:10DC8000E7E77846FCF7AEF9E6E77846FCF7AAF94D
:10DC9000E3E77846FCF7A6F9E1E77846FCF7A2F956
:10DCA000E1E700BFE039002010B5044600F028FF8E
:10DCB00050B16CB12046FFF75BFF0023636100F0B9
:10DCC0003FF8FFF783FF10BD7846FCF78BF9F0E7CC
:10DCD0007846FCF787F9EDE738B504460D46104B5A
:10DCE0001B788BB900F00CFF90B1ACB12046FFF768
:10DCF0003FFF0023636165602046FFF7C3FE00F02D
:10DD00001FF8FFF763FF38BD7846FCF76BF9E9E7CA
:10DD10007846FCF767F9E8E77846FCF763F9E5E74A
:10DD2000E039002008B515F0C5F900B108BD15F0BF
:10DD300039F90028FAD07846FCF754F9F6E70000E4
:10DD400070B4EFF3108172B6184B1A68184BD3F801
:10DD50000455D3F80431012B22D001B962B645EA4B
:10DD6000026500266B01EA0E5B1B62EB06025102A4
:10DD700041EAD3515802431941EB0600810141EABF
:10DD800093619A01D31A61EB00005B1946EB000026
:10DD900013F580437041DB0B43EA404070BC704791
:10DDA000034BD3F804550132D7E700BFEC3900200C
:10DDB0000010014010B50A4B4FF40032C3F848235D
:10DDC000C3F80823074B1B682BB1064B1C68FFF7F1
:10DDD000B7FFA04710BD7846FCF704F9F5E700BF90
:10DDE00000100140F8390020EFF3108172B6254B86
:10DDF0000022C3F80421244A13680133136001B9D7
:10DE000062B6224B1B68002B3AD0204B1A68013AAD
:10DE10001A601B68002B33D103F1804303F588336C
:10DE2000D3F804251A4B1B689A421BD2EFF31082D9
:10DE300072B6144BD3F80435981C1549096888420A
:10DE40000DD303330F49C1F8443502B962B60D4B07
:10DE50004FF40032C3F84423C3F8042370470C4B3B
:10DE60001B68EFE710B50B4B1B682BB1094B1C6807
:10DE7000FFF766FFA04710BD7846FCF7B3F8F5E75B
:10DE8000704700BF00100140EC390020F03900203D
:10DE9000F4390020F839002030B583B0044600235F
:10DEA00001930D46002936D0244B1D60FFF748FF33
:10DEB000031B002B33DB0023590CD803204C214AD1
:10DEC000002300194FF0000444EB010115F01CF988
:10DED000EFF31083019372B61B4BD3F8043503287C
:10DEE00038BF0320C3F1FF1202F57F42824218D3EC
:10DEF0000344154AC2F844354FF40033C2F84433A2
:10DF0000C2F80433114A1460114A1460019B03B92A
:10DF100062B603B030BD7846FCF764F8C4E7231A54
:10DF2000CAE7034403F17F4301331A0E0132074964
:10DF30000A6023F07F43064A1360E7E7F8390020C0
:10DF400020A1070040420F0000100140F0390020DE
:10DF5000F4390020074B4FF40032C3F84823C3F8CC
:10DF600008230023044A1360044A1360044A136020
:10DF7000704700BF00100140F0390020F439002044
:10DF8000F839002030DF704731DF704710B40346A6
:10DF900002684068A2EB70129C6880EAF430186056
:10DFA000D9680C445C60114499601044D8605DF8F5
:10DFB000044B704770B582B00D46064608B1002488
:10DFC0000BE07846FCF70EF8F9E79DF807103019DA
:10DFD000FFF7DAFF9DF807301C44A5420DD90DF17B
:10DFE0000700FFF7CFFF9DF80730002BF7D02A1B63
:10DFF0009342EAD98DF80720E7E702B070BD000030
:10E0000030B583B005460024019404210DEB0100D6
:10E01000FFF7D0FF074B2B60019B6B60AB60EB60A1
:10E0200003E02846FFF7B2FF0134132CF9D903B0FF
:10E0300030BD00BFED5EEAF1704708B5032004F083
:10E040002FFD08BD48DF704749DF70474ADF704742
:10E05000044B01225A7143F2B0629A6043F698224F
:10E06000DA607047583A0020094B03221A74094AB3
:10E070005A611A6840F6D8639A4204D9054B43F2B4
:10E08000B0629A607047034B40F6D8629A6070475E
:10E09000383A0020583A002008B50F4B1B78022B65
:10E0A00012D0032B08D0012B03D07846FBF79AFF40
:10E0B0000EE0022303740BE0084B00225A7108495A
:10E0C00099600849D960827103230374034B43614B
:10E0D000014B00221A7008BD693A0020583A00200E
:10E0E000A0860100FF1FA10738B50446002505746E
:10E0F000012343710E4A13680133136000F0C4FA20
:10E100000BF0C8FD23680B4A1168283101FB03F1AD
:10E11000094AA2FB0121A3EB9141084A783928461C
:10E1200000F02EFA00B938BD7846FBF75BFFFAE73E
:10E130006C3A0020543A002083DE1B4369E0020061
:10E1400010B5044600238360C36003680D4A9268DB
:10E150000260817991B10121017403B90A4B991AC6
:10E160006161B1F57A7F01D39A4202D94FF47A7393
:10E170006361FFF76DFF0123A37110BDFFF7B4FFCB
:10E18000F7E700BF583A00208096980010B50C467B
:10E1900031B1C3680133C36042690368134403604B
:10E1A000836801338360012202744269520842612C
:10E1B000012B0DD0022B19D0426903681344174973
:10E1C0008B4222D840F6D7639A4221D800231DE023
:10E1D000B2F5FA7F05D040F6D8639A42ECD8436195
:10E1E000EAE7002CF7D100234361E5E7C368022B7F
:10E1F00006D0012BE0D1002CDED100234361DBE708
:10E200000268064B9B1A4361D6E7002313B110BD89
:10E210000123FBE7FFF768FFF9E700BF809698004E
:10E2200043791BB90D4B00221A70704710B5044694
:10E230000BF04CFD23680A4A1068283003FB00F0FD
:10E24000084AA2FB0020A3EB9040783800F04CFA7B
:10E2500000236371014B00221A7010BD683A002040
:10E26000543A002083DE1B4308B5254B01221A7166
:10E27000244B1B7813B1244B1B781BB3204B00227B
:10E280001A7404281AD8DFE800F00314110C0700F0
:10E290001B48FFF755FF1CE001211948FFF776FFE7
:10E2A00017E000211648FFF771FF12E00BF09EFC0B
:10E2B0000FE000F0ABF90BF0D3FC0AE07846FBF777
:10E2C00091FE06E000F082F90D4B18601846FFF74A
:10E2D000E3FE0B4B1B7C023BDBB2012B08D9084B46
:10E2E0001B7C022B08D0064800230371103008BDA8
:10E2F0000348FFF795FFF2E7014B01221A76F2E798
:10E30000383A0020693A0020683A002008B50438FD
:10E31000042814D8DFE800F0182614030E00164B6A
:10E320001B7E012B0BD1FFF78FFE40B17846FBF728
:10E3300059FE04E0104B00221A760BF0EFFC08BDEA
:10E340007846FBF74FFEFAE7FFF782FE0B4840F6F0
:10E35000D8638360FFF77AFE0028F0D07846FBF799
:10E3600041FEECE70548FFF771FE0028E7D078464C
:10E37000FBF738FEE3E700BF383A0020583A0020A8
:10E3800010B40E4A0023137013710121517143F22E
:10E39000B064946043F69824D460094A1060094A36
:10E3A0001370094A1370094A1360094A13715371B3
:10E3B0001360137691715DF8044B7047583A002052
:10E3C000543A0020683A0020693A00206C3A002054
:10E3D000383A002008B5104B1B7E012B08D0022BC9
:10E3E00017D00BB1002008BD0C48FFF72BFE40B939
:10E3F0000B48FFF72BFE40B9074B02221A7600208C
:10E40000F1E77846FBF7EEFDF2E77846FBF7EAFD29
:10E41000F2E71120E7E700BF383A002069E2020086
:10E42000583A00200B4B1B7C023BDBB2012B0BD973
:10E43000094B1B78012B09D0022B09D0032B01D0EB
:10E44000002070470120704701207047012070476D
:10E4500001207047383A0020693A0020014B1868C3
:10E46000704700BF383A00200D4B5B790BB9002094
:10E47000704710B50A4B1C680A4B1B68283303FB16
:10E4800004F3094AA2FB0323A4EB9344783C00F075
:10E490009DF80346201A00D410BD181BFCE700BFEE
:10E4A000383A0020543A002083DE1B43014B187990
:10E4B000704700BF383A0020EFF3108372B6054A68
:10E4C000527922B1044A4FF48071C2F8001103B9A5
:10E4D00062B67047383A002000E100E008B5054B0D
:10E4E0001B7E022B00D008BD034B01221A70FFF7E0
:10E4F000E3FFF8E7383A0020693A002008B5074BF7
:10E500001B7E022B00D008BD012804D0044A1370E2
:10E51000FFF7D2FFF7E70323F8E700BF383A002000
:10E52000693A002008B5094B1B782BB148B9084B54
:10E530001B7813B1012300E00023044A107013B9C3
:10E5400008BD0023F9E7FFF7B7FFF9E7683A0020B5
:10E55000693A002010B4094B00F15002002443F83E
:10E56000224000F110040122A240C3F8042300F568
:10E57000A87043F820105DF8044B704700800040FD
:10E58000022817D810B5EFF310840C4B1C6072B63C
:10E590000B4B43F820200B4B002243F820200A4B62
:10E5A0001B7823B9054B186830B962B605E0FFF750
:10E5B000D1FFF7E707207047002010BD803A002008
:10E5C000703A00208C3A00207C3A0020EFF3108251
:10E5D0000A4B1A6072B60A4B1B7863B1094B0022D2
:10E5E000C3F84C210122DA64D3F84C05034B1B68B5
:10E5F00003B962B67047044B1868F7E7803A002009
:10E600007C3A002000800040843A00202DE9F0414F
:10E61000002411E00027174B43F82470012303FA6C
:10E6200005F5154EC6F80853FFF7D0FFC04704F1B3
:10E63000500346F823700134022C18D804F150031B
:10E640000D4A52F82330002BF5D0D2F8043304F1F0
:10E650001005EB4013F0010FEDD0064B53F824806A
:10E66000B8F1000FD6D17846FBF7BCFCD2E7BDE885
:10E67000F08100BF703A002000800040014B1B6811
:10E6800018447047883A002010B500230CE0114A66
:10E6900003F5A871002042F8210003F1500142F86F
:10E6A000210052F821200133022BF0D90A4B1B68BC
:10E6B0001BB90A4B4FF480721A60094B01221A7081
:10E6C000FFF73EFB0446FFF781FF241A054B1C6051
:10E6D00010BD00BF00800040803A002000E100E053
:10E6E0007C3A0020883A0020002307E000220C49F1
:10E6F00041F823200B4941F823200133022BF5D99F
:10E70000094B1860094B00221A70094B4FF0FF3279
:10E71000C3F80823074B4FF48072C3F88021704779
:10E72000703A00208C3A0020843A00207C3A002085
:10E730000080004000E100E008B503783BB1012B08
:10E7400004D1436813B1C1688068984708BD436825
:10E75000002BFBD080689847F8E70000044B1B783B
:10E760000F2B04D0034B4FF48022C3F800217047D5
:10E77000FC3B002000E100E010B5104C2070104878
:10E78000104B0360102343608360FDF7DDFE0E48ED
:10E79000FFF70EF823780F2B0FD0072B0AD8EC22A7
:10E7A0001A4112F0010F05D05B01DBB2074A82F873
:10E7B000123302E07846FBF715FC10BDFC3B00204D
:10E7C000983A0020AC3A0020003C002000E100E034
:10E7D00008B5124B1B780F2B00D108BD104B93F8D6
:10E7E00012335A09EC23134113F0010F0ED00D4BD5
:10E7F0009B6833B10B4A136843F4802313600023F2
:10E8000006E0074A4FF48021116001E042F2020362
:10E81000002BE2D07846FBF7E5FBDEE7FC3B00206F
:10E8200000E100E06C5B002038B5EFF3108472B6B5
:10E83000194A1368591C116003BB184B1B780F2B26
:10E840001CD0EFF3108272B6154B9B68E3B91449E4
:10E8500001238B60134BD3F88000134D28400860D0
:10E86000C3F88050D3F8840048604FF0FF31C3F8FC
:10E8700084100E4B0021197002B962B6064B1B685A
:10E8800033B104B962B638BD084B01211970F3E702
:10E890007846FBF7A7FBF4E7AC3B0020FC3B0020ED
:10E8A0006C5B002000E100E0FC06FFBDFD3B0020AA
:10E8B00010B5EFF3108472B6124B1B68F3B1114A16
:10E8C0001368013B1360B3B90F4B1B780F2B12D0A9
:10E8D0000E4B1A780E4B9B686BB162B9EFF3108147
:10E8E00072B60B4B18680B4A1060586850600022D3
:10E8F0009A6001B962B604B962B610BD7846FBF7FA
:10E9000071FBDCE7AC3B0020FC3B0020FD3B002022
:10E910006C5B002000E100E010B5044680B10C4BB8
:10E920001B68102B10D8EFF3108272B6084B1868D2
:10E93000411C1960074B43F8204002B962B610BD74
:10E940007846FBF74FFBEAE77846FBF74BFBEAE735
:10E95000B03B0020B43B002038B504460D4B1B688B
:10E96000834213D9EFF3108572B661090A4A04F0A5
:10E970001F04012303FA04F452F82130234342F820
:10E980002130FFF7EBFE05B962B638BD7846FBF7DC
:10E9900029FBE7E7B03B0020F83B002070B50D46AF
:10E9A0001646044658B175B1EFF3108372B6A560F0
:10E9B000E66000222274246003B962B670BD784616
:10E9C000FBF710FBEFE77846FBF70CFBECE70000EA
:10E9D00038B5044650B1A36863B1EFF3108572B641
:10E9E000237C5BB1112005B962B638BD7846FBF7D0
:10E9F000F9FAF0E77846FBF7F5FAEEE7012323741E
:10EA000021460348FEF7DFFEFFF7A8FE0020EAE7F5
:10EA1000003C002010B5044608B1207C10BD7846AB
:10EA2000FBF7E0FAF9E7000070B584B02C4B1B78D7
:10EA300023B901252A4B1D7000240AE07846FBF714
:10EA4000D1FAF6E7274B53F8243098470646F0B141
:10EA50000134254B1B68A3421ED96109234A52F891
:10EA6000213004F01F00C34013F0010FF0D0EFF38A
:10EA7000108672B6012303FA00F052F8213023EA1F
:10EA8000000342F82130002EDCD162B6DAE72046DE
:10EA9000FFF762FF3546DBE71548FEF7B0FE0AE0F8
:10EAA0007846FBF79FFAA368E06898470023237431
:10EAB0000F48FEF7A4FE20B10468237C002BF2D19E
:10EAC000EEE769460B48FDF75BFD18B96846FFF7AE
:10EAD00033FEF6E7024B00221A70284604B070BDE0
:10EAE000083C0020B43B0020B03B0020F83B002055
:10EAF000003C0020983A002008B5FFF795FF08BDBC
:10EB000000B583B0FEF7CEFE8DF807009DF8073004
:10EB10005BB213F1100F18D09DF807305BB2002BD9
:10EB200021DB03F1604303F5614393F800335B0994
:10EB30000093154B1B78009A934220D0009A934281
:10EB400017D3002003B05DF804FB0F4B1B780F2B8D
:10EB500001D10120F6E71220FEF7ACFE08B100203B
:10EB6000F0E70120EEE703F00F03084AD35C5B09EE
:10EB7000DEE71220FEF79EFE18B10020E2E701203A
:10EB8000E0E70120DEE700BFFC3B002014ED00E0E1
:10EB900046DF704770B58CB003460E4614466D468E
:10EBA000006859689A68DB680FC530687168B26898
:10EBB000F3680FC56846FFF7EBFF08AD0FCD206087
:10EBC0006160A260E3600CB070BD08B5FEF7C3FEE3
:10EBD00008BD08B502F09FF808BD08B502F0D4F8EA
:10EBE00008BD38B5022931D84CB2002C54D10029C7
:10EBF0007ED11970817A5A7861F306025A70C17A0F
:10EC0000D2B261F3C7125A70C168C1F3074201F46E
:10EC10007F44224300249A70120ADA701971018924
:10EC20000A0A42EA0122A3F80520DC711C7201697C
:10EC30000A0202F47F0242EA0162080A00F47F40FD
:10EC4000024342EA1162C3F8092038BD03294FD1BB
:10EC5000197000215970C468C4F3074204F47F4559
:10EC60002A439A70120ADA701C710489220A42EA55
:10EC70000422A3F80520D971197201690A0202F46D
:10EC80007F0242EA0162080A00F47F40024342EA3E
:10EC90001162C3F80920D8E71970597801F0800192
:10ECA00062F3C7115970C168C1F3074201F47F4490
:10ECB00022439A70120ADA70197101890A0A42EA2B
:10ECC0000122A3F8052041880A0A42EA0122A3F89A
:10ECD000072001690A0202F47F0242EA0162080A7F
:10ECE00000F47F40024342EA1162C3F80920ACE716
:10ECF0007846FBF777F9A8E770B584B00D4614465F
:10ED0000064668B162B10023009301930293039316
:10ED100023462A4631466846FFF757FF04B070BDC8
:10ED20007846FBF75FF9EEE72DE9F04184B00E4637
:10ED300014461D460B9F804610B10AB103B117B9A6
:10ED40007846FBF74FF96B46324641462046FFF7BF
:10ED50003CFF3B469DF8282029466846FFF735FFD3
:10ED600004B0BDE8F08100002DE9F0418EB00E4600
:10ED700014461F46054608B101B113B97846FBF7A2
:10ED800031F9002C4DD0102C4FD82A4B049305AAF2
:10ED9000042104A8FFF7B0FF6B461022294605A8FE
:10EDA000FFF713FF2246314605A814F0E6FA0EAB32
:10EDB0002344012203F8242CA21805AB92B2194671
:10EDC0006846FFF702FF9DF8233003F07F033D46BE
:10EDD00005F8013B2246314609A814F0CEFA04F1A9
:10EDE00010080EAB9844022308F8243C1134A4B256
:10EDF0002B46224605A96846FFF7E7FE05AE2868C0
:10EE00006968AA68EB680FC6032308F8243C07F179
:10EE10001103224605A96846FFF7D7FE0EB0BDE8EC
:10EE2000F0817846FBF7DEF8ADE77846FBF7DAF8D5
:10EE3000ABE700BF736D6B3230B589B00C46054649
:10EE4000F8B1F1B1114B039304AA042103A8FFF711
:10EE500053FF04AB102229461846FFF7B6FE0C4BB1
:10EE600093E8030001908DF8081004AB052201A976
:10EE70001846FFF7AAFE06AB03CB2060616009B01D
:10EE800030BD7846FBF7AEF8DCE700BF736D6B333F
:10EE9000B454040030B587B00C460546E8B1E1B182
:10EEA000104B019302AA04210DEB0100FFF724FF90
:10EEB00002AB102229461846FFF787FE0A4B009343
:10EEC00002AB042269461846FFF77FFE9DF8173013
:10EED00003F03F03237007B030BD7846FBF782F89C
:10EEE000DEE700BF736D6B346964360110B504460C
:10EEF00078B123789BB1E268B2F1807F11D2E27AD7
:10EF00000AB1022B0FD094F90A30002B05DB012047
:10EF100006E07846FBF766F8EBE7002000E000200B
:10EF200010BD0020FCE70020FAE730B587B00446AA
:10EF3000037C8DF8003002688368D27A32B30822ED
:10EF40001344093301932368029363680393E368CE
:10EF5000049305A9684602F015FC50EA01031AD093
:10EF6000237C012B07D0206800F10C011030FDF745
:10EF70007BFF054660B92168059800F006FA059BFD
:10EF8000093363610025284607B030BD0422D7E766
:10EF900002F0A0FCF7E70425F5E7000070B582B0A9
:10EFA00004466946008909F0FDFF18B1002528468E
:10EFB00002B070BD0646012004F044FC054600285E
:10EFC000F5D0A37A012B14D92378012B09D00A4B51
:10EFD0001B68002BEBD0A27A6188208998470546F0
:10EFE000E5E76946608809F0DDFF0028EFD0354687
:10EFF000DDE73546DBE700BF0C3C002008B538B143
:10F000004268054B1A60FDF757FD03F043F908BD50
:10F01000014B00221A60F6E70C3C002008B5FDF712
:10F020006FFD03F077F908BD10B5044668B1236899
:10F030007BB123685B6983B1237C012B11D8E36822
:10F040009BB12046FFF771FF10BD7846FAF7CAFF63
:10F05000EDE77846FAF7C6FFEBE77846FAF7C2FF26
:10F06000EAE77846FAF7BEFFE9E77846FAF7BAFF2B
:10F07000E7E70000F0B5C7B0064630B3736943B3A5
:10F08000336853B333685B695BB3706900F0E3F9CD
:10F090000546254B1B6813F0020F3BD0234B1B6822
:10F0A000042B37DD00231C2B1FD8EA5C204908689D
:10F0B00014095900075D05AC04F8137002F00F0243
:10F0C0000131825C62540133EDE77846FAF78AFF3A
:10F0D000D4E77846FAF786FFD2E77846FAF782FF58
:10F0E000D0E77846FAF77EFFCFE705AA00238DF830
:10F0F0004E3003F1804303F58833D3F80435029290
:10F100000C4A01920C4A00924FF497720B49052069
:10F1100000F02AFD00232A46B168306800F0EAFAC0
:10F1200002F09EFB47B0F0BD242E0020202E0020D0
:10F13000282E0020EC54040064390400E05404003C
:10F14000F0B589B004460E461546837A013B8372BA
:10F15000029004924FF0FF330393DF2305930123C2
:10F160008DF8183002A8FFF7E0FE074698B1114B62
:10F170001B6813F0020F16D00F4B1B68012B12DD1A
:10F180000E4BD3F804350E4A0092AD220D490220F1
:10F1900000F0EAFC07E02A463146079814F0EDF843
:10F1A00002A8FFF767FFA37A0133A372384609B0BC
:10F1B000F0BD00BF242E0020202E002000100140B2
:10F1C000F4540400E0540400F0B5D5B0002800F079
:10F1D000B6800E461746054600F041F9421B294607
:10F1E0004CA814F0CAF8574B1B6813F0020F31D02B
:10F1F000554B1B68042B2DDDB646802E28BF4FF0E3
:10F20000800E00230FE0E85C504A116802095C00A0
:10F2100011F802C005AA02F813C000F00F00013473
:10F22000095C115501337345EDD305AA002302F89B
:10F230001E3003F1804303F58833D3F8043502927E
:10F24000434A0192434A009240F253124249052038
:10F2500000F08AFC002300934CAB2A46314646A8B6
:10F2600000F0FCF9044610B1204655B0F0BD46A8A8
:10F27000FFF73CFE0028F7D0324B1B6813F0020F5B
:10F2800030D0314B1B68042B2CDDB446802E28BFB8
:10F290004FF0800C0FE04CAB1B5D2C4A1068190935
:10F2A0006200455C05A901F8145003F00F03013218
:10F2B000C35C8B5401346445EDD305AA002302F8E6
:10F2C0001C3003F1804303F58833D3F804350292F0
:10F2D000224A01921F4A00924FF4AE721E49052045
:10F2E00000F042FC4B9B03B3314646A800F0ABF85C
:10F2F000C5B23B4646AA29460DF23910FCF7DAF9A9
:10F300000446394646A8FFF749FE90B13B462A46D7
:10F310000DF2391146A8FFF713FF0028A4D149992F
:10F32000BDF82001FAF7E0FE9EE77846FAF75AFEAC
:10F33000DAE74999BDF82001FAF7D6FE94E70E24E2
:10F3400092E700BF242E0020202E0020282E00202F
:10F350002455040064390400E054040034550400CA
:10F360004B78DB09C3724B7803F07F0383728A7892
:10F37000CB781B0243EA02430A791343C3604A79FC
:10F380008B7943EA02230381704738B50C46054662
:10F39000002840D0002C42D02089FEF76DF80128CB
:10F3A00041D194F90A30002B41DBE368B3F1807F4F
:10F3B00041D26369002B42D0236903F001022B780C
:10F3C00003F07F0343EAC2132B706269127803F0E3
:10F3D000800302F07F0213432B70E27A6B7803F014
:10F3E0007F0343EAC213DBB26B70A27A03F080039F
:10F3F00002F07F0213436B70E3681A0CAA701A0ABA
:10F40000EA702B7123891A0A6A71AB7163881A0A30
:10F41000EA712B7238BD7846FAF7E4FDBAE7784610
:10F42000FAF7E0FDB8E77846FAF7DCFDB9E7784689
:10F43000FAF7D8FDB9E77846FAF7D4FDB9E7784688
:10F44000FAF7D0FDB8E7C37A1BB10820081A0938CB
:10F4500070470420FAE709387047073070470130D9
:10F46000704770B588B004460D46164600230093D9
:10F470008DF804300269130203F47F0343EA026348
:10F48000110A01F47F410B4343EA1263CDF80530C2
:10F490002846FFF7E2FF0368CDF8093082888379B8
:10F4A000ADF80D208DF80F30606904AA694611305F
:10F4B000FFF770FB3046FFF7D2FF04462846FFF700
:10F4C000CEFF06234BB1013B9BB2C25C08A9194495
:10F4D00011F8101C4A40E254F4E708B070BD000077
:10F4E0002DE9F041D2B004460D4617461E469DF860
:10F4F000648100238DF84731ADF8283149934EAB34
:10F5000046931046FFF7A9FF47903046FFF7A5FF47
:10F510004B90589B6361324639462046FFF7A1FF66
:10F5200031462046FFF71CFF2089FDF7A5FF012883
:10F5300011D1A5F10902E37A23B108239A4203D23B
:10F54000002309E00423F9E7E1682089FAF7A6FD22
:10F55000E8B9012300E0002383B3E37ACBB10821AB
:10F56000C9B28DF834116D1A073DADB2ADF8205116
:10F57000479B1D444C95B8F1000F0ED0B8F1010F18
:10F5800009D07846FAF72EFD4FF0000805E0002379
:10F59000E2E70421E4E74FF003084EAB00224146C6
:10F5A0002046FFF71EFB6369013345930DF24711B7
:10F5B00045A8FFF712FB9DF8473123B99DF8470195
:10F5C00052B0BDE8F081F379307A40EA03206080E0
:10F5D000FDF752FF20701B4B1B6813F0020FEDD09C
:10F5E000194B1B68032BE9DDBDF82061802E28BF75
:10F5F000802600230FE04B9AD25C14490C68100956
:10F600005900255C04A800F8135002F00F020131E4
:10F61000A25C42540133B342EDD304AA002302F8A2
:10F62000163003F1804303F58833D3F80435029292
:10F63000074A0192074A0092E4220749042000F099
:10F6400093FABBE7242E0020202E0020282E002035
:10F650007855040064390400685504002DE9F0472A
:10F6600084B00E4615461F469DF83090804618B16E
:10F6700012B10BB19A4202D17846FAF7B3FC082EC8
:10F6800030D91D2E30D82878C009FDF731FCC8F8D4
:10F6900010000023C8F8143095F800A00AF07F0A83
:10F6A0000293039301E0029BD3B103AA02A950463F
:10F6B00009F082FB0024012CF5D804AB03EB840392
:10F6C00053F8080C0028EED0CDF8049000903B468B
:10F6D0002A4631464046FFF703FF48B90134EAE7BE
:10F6E000052002E0092000E0092004B0BDE8F08711
:10F6F0000020FAE7F0B58FB00D4616461C460746C7
:10F7000050B16EB1012C0FD89CB1012C10D07846AD
:10F71000FAF768FC00240CE07846FAF763FCF0E79F
:10F720007846FAF75FFCEDE77846FAF75BFCEBE723
:10F7300003240AAB002221463846FFF752FAFB7A2F
:10F7400003B308238DF824307B69013301930AAB9E
:10F7500002933046FFF781FE03900790A91C89B2FF
:10F76000ADF810100023ADF8183005930844089048
:10F7700001A8FFF72EFA324631463846FFF771FEF0
:10F780000FB0F0BD0423DDE738B50D460446C8B11F
:10F790002378AB421AD9EDB962682378134413F881
:10F7A000013CA1780B44DBB212789B1ADBB2CBB1DF
:10F7B0006368585DA378013B1840A368627802FB38
:10F7C000003038BD7846FAF70DFCE1E77846FAF7E5
:10F7D00009FCE0E76268531913F8013C525D9B1A7B
:10F7E000DBB2E4E70020ECE738B50C460546A0B1F3
:10F7F0002B78A34215D9C4B96A682B78134413F83F
:10F80000013CA9780B44DBB212789B1ADBB21BB126
:10F810006A68135D0133135538BD7846FAF7E2FB89
:10F82000E6E77846FAF7DEFBE5E76A68131913F8AE
:10F83000013C125D9B1ADBB2E9E710B5044640B10A
:10F84000002322789A4208D962680021D1540133FA
:10F85000F7E77846FAF7C6FBF2E710BD10B50446A5
:10F8600043786BB12378012B0ED9A36883B1636809
:10F8700093B1A378A3B15A1E134217D0002310E00E
:10F880007846FAF7AFFBEDE77846FAF7ABFBECE723
:10F890007846FAF7A7FBEAE77846FAF7A3FBE8E72A
:10F8A00000232BB12046FFF7C8FF10BD0123F8E766
:10F8B0007846FAF797FBF5E738B50C46054678B178
:10F8C0002B78A34210D99CB96A682B78134413F89B
:10F8D000010CAB781844C0B21378C01AC0B238BD5E
:10F8E0007846FAF77FFBEBE77846FAF77BFBEAE727
:10F8F0006B681A1912F8010C1B5DC01AC0B2EEE752
:10F9000028B108B529B1FFF7C5FA002008BD0E20BF
:10F9100070470E20FAE770B130B583B00B4661B185
:10F9200000248DF8074001220DF10701FFF71CFAB2
:10F93000204603B030BD0E2070470E20F9E70000CE
:10F9400000B330B58BB00C460546E9B11031FFF776
:10F9500073FA0E4B09930E4B93E803000790ADF832
:10F96000201003AA042109A8FFF7C6F90194062371
:10F97000009307AB03AA10212846FFF7D5F9002012
:10F980000BB030BD0E2070470E20F9E76E6B626B36
:10F990008C55040010B330B587B00C460546F9B15C
:10F9A000104B019302AA04210DEB0100FFF7A4F90B
:10F9B00002AB102229461846FFF707F99DF81630CA
:10F9C0001B0203F47C536FEA43436FEA53439DF8F1
:10F9D000172013432380002007B030BD0E2070474E
:10F9E0000E20F9E77674616470B50E46044648B19E
:10F9F00041B12368B34209D0256865B92660002368
:10FA0000336017E07846FAF7EDFAF2E77846FAF74E
:10FA1000E9FAF1E725462C682CB1B442FAD17846D0
:10FA2000FAF7E0FAF6E735B12EB1B54202D02B680D
:10FA300033602E6070BD7846FAF7D4FAF5E738B532
:10FA400005460C4689B180B12B68BBB1A34210D0EA
:10FA50001A461B680BB1A342FAD18AB1A34211D155
:10FA6000236813600020206038BD7846FAF7BAFAA0
:10FA7000EAE723682B6000202060F5E70520F3E724
:10FA80000520F1E70520EFE72DE9F0410E46174686
:10FA9000054608B101B112B97846FAF7A3FA2B6806
:10FAA000B34204D02C6834B14FF0000809E0784626
:10FAB000FAF798FAF6E72E60002030600FE0A046D3
:10FAC0002C4654B131462046B84730B92568AE427D
:10FAD000F5D17846FAF786FAF1E714B10F20BDE8C0
:10FAE000F081B8F1000F09D046B1B04504D0D8F884
:10FAF00000303360C8F800600020F0E77846FAF77D
:10FB000071FAF2E730B583B010461A4606AC54F8E5
:10FB1000045B00900B46054900200BF0DFFA2246FB
:10FB2000294600200BF0E6F903B030BD94550400DF
:10FB3000034B1860034B1960034B1A60704700BFFA
:10FB4000242E0020202E00202C2E002030B583B043
:10FB5000044C246824B1079D0195069D0095A0479B
:10FB600003B030BD2C2E002030B585B008AC54F861
:10FB7000045B039401940095FFF7E8FF05B030BDE6
:10FB8000C3681A795979521A03EB023342699B1AF6
:10FB90008068181A704770B50579012D01D90020C9
:10FBA00070BD044606683046FFF7EAFF3DB9A389F9
:10FBB0009B00834205DB73682BB90020F0E700232C
:10FBC000F7E70020ECE70120EAE738B505460C46E8
:10FBD00010F0030F0DD114F0030F0ED10023B3EB7F
:10FBE000940F0ED255F82320B2F1FF3F0BD1013311
:10FBF000F5E77846FAF7F6F9EDE77846FAF7F2F91D
:10FC0000ECE7012038BD0020FCE770B50546002474
:10FC10000EE0002300E00023184643B35379A342CB
:10FC20001CD1EB6833441A792B699A421AD10134FA
:10FC30002B69A3421AD9EB68260303EB04329B5DC0
:10FC4000083BDBB2F62BE6D85379FF2B04D01379AF
:10FC5000FF2BDED00123DFE70023DDE77846FAF74C
:10FC6000C1F9DEE77846FAF7BDF9E0E7012070BD9B
:10FC7000F0B585B004460368DB68187819795A79BD
:10FC8000891AE28903EB0131184401F02BFD074684
:10FC90002568AB68002B45D021688E6826F47F6309
:10FCA00023F00F0303F58055A81BA2899300B0EB46
:10FCB000820F45D9F51804F10C02A3899B0001209D
:10FCC0008DF8000001960392029300226946FDF729
:10FCD000E9FA00285AD101208DF800000195324B35
:10FCE000039304230293314A6946FDF7DBFA0028A7
:10FCF00050D19FB122683988536803EB8103536068
:10FD000001208DF800000197294B039304230293EF
:10FD1000264A6946FDF7C6FA00283FD1A6600020B2
:10FD200005B0F0BDEB68187819795A79891A47F649
:10FD3000FF7203EB0131184401F0D4FCA860ABE77B
:10FD4000CA68117992F805C0A1EB0C0102EB0132EF
:10FD5000954227D0834202D12B781D44ABE7012086
:10FD60008DF800000196134B0393042302930022A5
:10FD70006946FDF797FA28B92E782E44A58906EB37
:10FD8000850598E77846FAF72DF9F5E77846FAF70A
:10FD900029F9A0E77846FAF725F9AAE77846FAF7AD
:10FDA00021F9BBE70120BBE710560400363D0020D7
:10FDB000085604000C56040010B584B004460368CD
:10FDC000DB68187819795A79891AE28903EB0131CD
:10FDD000184401F087FCE0B10346A0602168008868
:10FDE0004A6802EB80024A6001208DF8000001930E
:10FDF000094B039304230293084A6946FDF752FA1C
:10FE000010B9002004B010BD7846FAF7EBF80020D6
:10FE1000F8E70220F6E700BF08560400363D002050
:10FE200070B584B005460368DE68437B06EB033695
:10FE300008213046FFF7C9FE80B9002403E0784668
:10FE4000FAF7D0F80134072C08D8335D05F1080221
:10FE5000125D9342F6D0FF2BF4D0F0E70835012075
:10FE60008DF800000196039508230293054A694620
:10FE7000FDF718FA10B9002004B070BD7846FAF703
:10FE8000B1F8F8E7363D002000B585B00368DA68C0
:10FE90001B691B0302218DF8001001920293074A8F
:10FEA00069460120FDF7FEF918B9002005B05DF89C
:10FEB00004FB7846FAF796F8F7E700BF363D0020D6
:10FEC00082890379012B0FD010B59200022B11D03B
:10FED0000BB1012010BD00F10C01806813F01AFA7B
:10FEE000B0FA80F04009F5E783685888B0FA80F0EE
:10FEF000400970470368DB68447B0822811803EBE4
:10FF0000043013F007FAB0FA80F04009E2E700008D
:10FF100038B501460C48FBF7A7FE0C4B5D6845B9A8
:10FF200038BD2368002222609A68D8689047A542AD
:10FF3000F6D00648FDF763FC04460028F1D1784668
:10FF4000FAF750F8EDE700BF103C0020243D0020F8
:10FF50002DE9F041044617460E4611B9FFF7B0FFF0
:10FF600058B10EB104F10C0725682379042B5BD836
:10FF7000DFE803F0053A415A50000326F2E73EB1AC
:10FF8000AB69002B50D032463946284698474BE0A3
:10FF9000D4F80880B8F80030C3B1B8F8003008EBE6
:10FFA000830323F47F6222F00F02934212D0B8F849
:10FFB0000220B2F5FE4F0DD0AB605A8847F6FF73B2
:10FFC0009A42DDD07846FAF70DF8D9E77846FAF785
:10FFD00009F8E2E728F47F6828F00F0808F5805850
:10FFE00098F800304344E7E7EB69EBB13246E1892A
:10FFF0002846984718E02B78012B07D1627B237B9A
:020000023000CC
:10000000013B9A4210D102232B700DE07846F9F79C
:10001000E9FFF3E7BEB92B78012B01D000232B7049
:100020002B6A0BB128469847094B9C4203D303F532
:1000300082739C4202D97846F9F7D4FF201FFFF75C
:1000400067FFBDE8F0817846F9F7CCFFE3E700BF32
:100050001C3C002000B583B00023019382B201A9AB
:100060000548FBF726FD20B90198043003B05DF880
:1000700004FB0020FAE700BF103C002070B50546E5
:10008000002436E01020FFF7E5FF0646002861D087
:100090000223037108230372042343721023C372E3
:1000A000837244732B6903734FF6FF73C38105603A
:1000B000294B984203D303F58273984202D97846BC
:1000C000F9F790FF36F8042C311F2448FBF72AFD7E
:1000D0000EE0002300E0002353B3EB6833445B7968
:1000E000A34229D1EB681E4432792B699A4227D169
:1000F00001342B69A34227D9E868260300EB0430BA
:1001000040F6FC710430FFF760FD0028BAD1EB68BF
:100110009A199B5D083BDBB2F62BDCD85379FF2B99
:1001200004D01379FF2BD4D00123D5E70023D3E7E4
:100130007846F9F757FFD0E77846F9F753FFD1E74C
:100140007846F9F74FFFD3E7054B1868FEF704FC34
:10015000002070BD0420FCE71C3C0020103C002067
:100160002C3D002038B50546C3681C781C4400208F
:100170000DE07846F9F736FF19E024F47F6323F0A9
:100180000F0303F580531A78134420461C46EB688E
:100190001A795979521A03EB02339C4215D26288BC
:1001A0004FF6FF739A4210D02388002BE1D02388AA
:1001B00004EB830323F47F6222F00F029342DCD02E
:1001C0006288B2F5FE4FE0D1D7E738BD38B50446B6
:1001D000FCF758F958B92046FFF7C4FFA06050B1AA
:1001E000428847F6FF739A4211D1002038BD784605
:1001F000F9F7F8FEEFE7E2681378134459884FF6F1
:10020000FF72914201D00020F0E7A360EEE70820E2
:10021000FFF720FF0546C0B10323037104600C4BB8
:10022000984203D303F58273984202D97846F9F7CE
:10023000D9FE35F8042C291F0648FBF773FC064B42
:100240001868FEF789FB0020D0E70420CEE700BF46
:100250001C3C0020103C00202C3D0020F8B5067905
:100260004379F61A00EB063604782518002711E0CA
:100270002B88F3B12C8805EB840424F47F6323F0EE
:100280000F039C4219D06B88B3F5FE4F15D0A642E0
:100290001CD925466B884FF6FF7293421AD047F659
:1002A000FF72934216D0002BE2D12B8807EB830715
:1002B000DEE77846F9F796FEDCE725F47F6424F064
:1002C0000F0404F5805423781C44E0E77846F9F7DE
:1002D00089FEDEE73846F8BD70B584B00546006893
:1002E000FFF740FF044600B3638813BB2E682388E2
:1002F000002B30D0238804EB830323F47F6222F0A9
:100300000F0293422BD06288B2F5FE4F27D0B36024
:100310002B689968DB681A795879121A03EB023353
:10032000994225D3002004B070BD7846F9F75AFEF3
:10033000DAE701208DF800000194244B0393042395
:100340000293234A6946FCF7ADFF0028CED07846D9
:10035000F9F748FECAE77846F9F744FECAE724F4FD
:100360007F6323F00F0303F580531A781344CEE71D
:100370002388F3B1238804EB830323F47F6222F004
:100380000F02934219D06288B2F5FE4F15D00120BA
:100390008DF8000001930F4B0393042302930C4A42
:1003A0006946FCF77FFF0028BCD07846F9F71AFEB3
:1003B000B8E77846F9F716FEDCE724F47F6424F00A
:1003C0000F0404F5805423782344E0E70856040022
:1003D000363D00201056040008B50379042B13D8CD
:1003E000DFE803F00306090C0F00FFF741FC08BD2E
:1003F000FFF7E2FCFBE7FFF713FDF8E7FFF76CFF01
:10040000F5E7FFF741FDF2E77846F9F7EBFD00204D
:10041000EDE700002E4B1B78022B57D110B582B0B0
:1004200040E00023019301A92A48FBF7B1FB90B9F2
:10043000019C201D284B1860284B01221A70FFF7E1
:10044000AAFB58B30323224A1370626813706068D2
:10045000FCF746F822E0224B1B6803B198470120C5
:1004600002B010BD1C4B1868FFF7B6FF1D4B18708B
:1004700018B91A4B02221A7010E0184B03221A7096
:100480000CE0154B1B68EBB1134B18688268154BD9
:100490001978FFF75DFD114B00221A700C4B1B7889
:1004A000022BDCD10D4B1B78032BF7D801A252F89D
:1004B00023F000BF23040300650403005F0403006E
:1004C000830403007846F9F78DFDDDE701207047CE
:1004D000343D0020103C0020383D0020203D00200D
:1004E000303D00203C3D002008B5074B1B8893425F
:1004F00000D008BD054B1B78022BFAD1034B032219
:100500001A70FFF787FFF4E7363D0020203D0020FA
:1005100008B54FF4827210491048FBF74AFA1049A7
:100520000120FCF7ADFE0F48FEF7F6F90E4B186000
:1005300000230E4A13700E4A13800E48FDF738F957
:10054000FBF73EFF18B10C4B03221A7008BD0A4B93
:1005500002221A70FAE700BF1C3C0020103C002069
:10056000E9040300150403002C3D0020203D002079
:10057000363D0020243D0020343D002038B504469F
:100580000378022B00D0F3B90820FFF763FD05467E
:10059000D8B104232370037104600D4B984203D338
:1005A00003F58273984202D97846F9F71BFD35F8B6
:1005B000042C291F0748FBF7B5FA074B1868FEF70C
:1005C000CBF9002038BD0820FCE70420FAE700BF83
:1005D0001C3C0020103C00202C3D00202DE9F04F59
:1005E00085B00F4691460093834650B10120FCF739
:1005F00009FFFBF7A3FF01904FF0000AD046012549
:100600009CE07846F9F7EEFCF0E7019901F580519E
:1006100002910AF10101914213D032781644728896
:10062000013A92B247F6FE618A420ED84EB1019A63
:10063000131D107972880299184401F053F800B123
:100640000290019B0433029E89E003F50053344677
:1006500003951D4616E07846F9F7C4FC15E024F42E
:100660007F6424F00F0404F5805423781C44A542D1
:100670001DD9A6421ED26388013B9BB247F6FE629B
:10068000934211D92388002BE5D0238804EB830300
:1006900023F47F6222F00F029342E0D06288B2F529
:1006A000FE4FDCD01C46E2E7039D2646BEE7039DD5
:1006B0000026BBE7039D0026B8E7002343B108F1FD
:1006C0000108B9F1000F03D000992046C84705463C
:1006D000238823B3238804EB830323F47F6222F06F
:1006E0000F0293421FD06288B2F5FE4F1BD01C460A
:1006F000B44221DA012D1FD16288531E9BB247F606
:10070000FE618B42D9D837B179883B884A40134281
:1007100003D00023D2E70123D0E70123CEE77846B8
:10072000F9F760FCD6E724F47F6424F00F0404F5A5
:10073000805423782344DAE70AF1010ADBF8102019
:1007400052450FD9012D0DD1DBF80C4004EB0A33D3
:1007500003F580560199096899423FF456AF1C7819
:100760001C44C5E70020FCF74DFE404605B0BDE83F
:10077000F08F38B50C46054630B100231A462146A5
:100780002846FFF72BFF38BD7846F9F72BFCF4E736
:1007900070B50D461446064658B16B1E9BB247F61F
:1007A000FE6293420BD947F6FF739D4205D00023AA
:1007B00006E07846F9F716FCEFE7012300E0012395
:1007C000D3B1802C1CD83378F3B104F11000FFF7BB
:1007D00041FC80B100230371C5810334A4080134B6
:1007E000A4B284810660012C04D900EB84044FF08C
:1007F000FF33A3600C3070BD7846F9F7F3FBE0E7F8
:100800007846F9F7EFFBDEE70020F4E710B5044681
:100810000F4B984203D303F58273984202D978466E
:10082000F9F7E0FB0C3C0A4B9C4203D303F58273BF
:100830009C4202D97846F9F7D5FB34F8042C211FE5
:100840000448FBF76FF9044B1868FEF785F810BDF4
:100850001C3C0020103C00202C3D002070B50D46B3
:10086000064658B16B1E9BB247F6FE6293420BD907
:1008700047F6FF739D4205D0002306E07846F9F75E
:10088000B1FBEFE7012300E001230BB31020FFF7DA
:10089000E1FB044600B301230371C5814FF6FF73EA
:1008A000838106600D4B984203D303F5827398420F
:1008B00002D97846F9F796FB34F8042C211F084832
:1008C000FBF730F9074B1868FEF746F8002070BDBB
:1008D0007846F9F787FBD9E70420F8E71C3C0020AD
:1008E000103C00202C3D00202DE9F0410546FBF78F
:1008F000C9FD58B9EC6894F8008004EB08073E463F
:10090000AB68BB4206D80020BDE8F0817846F9F715
:1009100069FBEFE734F80830B3B134F8084007EB6F
:10092000840424F47F6323F00F039C4203D07B886C
:10093000B3F5FE4F1AD127F47F6727F00F0707F5AD
:1009400080573C783C4411E07846F9F74BFBE4E7EC
:100950007846F9F747FB0FE024F47F6323F00F0399
:1009600003F580531A78134426461C46AB68A3420D
:1009700010D02388002BEBD0238804EB830323F4CF
:100980007F6222F00F029342E6D06288B2F5FE4FFA
:10099000EAD1E1E77288531E9BB247F6FE618B42B3
:1009A00001D90020B0E7EB6818783146184400F010
:1009B00099FE30B1864206D041882846FFF74EFFA7
:1009C000A2E70020A0E700209EE7000030B583B03A
:1009D00004460D462F4B1B6813F4801F03D02E4B8B
:1009E0001B68062B25DC002323702B68C3F30B0345
:1009F0006BBB6B68FE2B2ED82A686B68A868E96809
:100A0000E26023616061A1612A696B69E26123622E
:100A10000023A36063602046FFF7F7F800282ED07C
:100A20002046FBF72FFDD0B103232370002003B035
:100A300030BD1A4BD3F804350A680192184A009267
:100A400040F2363217490720FFF78EF8CBE7784699
:100A5000F9F7C8FACDE77846F9F7C4FACCE7216987
:100A6000E068FFF7FBFB60602046FFF7AFFB002864
:100A7000DDD1022323702046FFF736FFD7E701239D
:100A800023702046FFF7FAFA0028D0D1E368083334
:100A9000A360CCE7242E0020202E0020001001406F
:100AA000F4550400E455040010B5044620B1A368D1
:100AB00033B1236843B110BD7846F9F793FAF6E7EE
:100AC0007846F9F78FFAF4E7246021460148FCF7ED
:100AD0007AFEF0E7243D002008B50648FBF7E9F868
:100AE00008B9002008BDFBF7F3FC08B90120F9E7BD
:100AF0000020F7E7103C002010B590B10446C36811
:100B0000187819795A79891A47F6FF7203EB01317F
:100B1000184400F0E7FDA06078B1022323700023A1
:100B200063600A4B02221A7009490120FCF7A8FBF6
:100B3000084B1868FDF710FF10BD2046FFF746FB75
:100B40000028EAD07846F9F74DFAE6E7343D002070
:100B5000E90403002C3D002008B5FBF7EFFC08BDBD
:100B600050B110B50446064B1B6813B17846F9F72F
:100B700039FA034B1C6010BD014B00221A6070470C
:100B8000303D00200078012814BF0020012070476C
:100B90000078042814BF00200120704746DF70470A
:100BA0002DE9F04707460E468589012411E0013BF7
:100BB0009BB2C1181EF801201CF803A082EA0A02A9
:100BC00008F80120002BF2D1A5EB0905ADB20134E4
:100BD000A4B2BDB1230A43EA0423F3833046FFF7EE
:100BE000DDFFA946102D28BF4FF01009D7F8188057
:100BF000601E0001D7F808E006F1200C5FFA89F9C1
:100C00004B46DFE7BDE8F0872DE9F047814688468F
:100C100017461C4600F1100500F1200616E052466A
:100C20004146281912F0A9FB2744BFB2103FBFB2BA
:100C3000D0441DE0013B9BB2F45CEA5C5440EC54B0
:100C4000002BF7D14846FFF7A9FF002497B1C4F164
:100C5000100A5745E3DA3A464146281912F08DFB4F
:100C60003819C0F110020021284412F0AFFB002710
:100C70001023E5E7BDE8F08770B505460C4616463B
:100C8000838A002B3BD0402295F82030023B03EBB7
:100C9000D3735B10DB0003F03803134343F001030D
:100CA00023746B68186859689A68C4F81100C4F80E
:100CB0001510C4F819201B7B6377AA89130A43EA2D
:100CC0000223E3832046FFF769FFAB8A6BB1B3F5DC
:100CD0007F4F16D2AA8A130A43EA022323820223F1
:100CE000AA8A29692046FFF78FFFAA896AB995F871
:100CF000202004F12001304612F03FFB70BD00229D
:100D0000C2E77846F9F76EF9E4E70023A9682046C0
:100D1000FFF77AFFEBE730B58DB0044603686D4608
:100D2000186859689A68DB680FC5E2696946204609
:100D3000FFF7A2FFE569636801228DF810201868AB
:100D400059689A68CDF81100CDF81510CDF8192022
:100D50001B7B8DF81D300023ADF81E306846FFF771
:100D60001DFF94F820304BB1013B9BB2EA5C0CA90B
:100D7000194411F8101C4A40EA54F4E76946204629
:100D8000FFF70EFF0DB030BD70B590B004460E46B3
:100D900090F82030102B35D8236804AD18685968B6
:100DA0009A68DB680FC5A38983BBA568A369A360A4
:100DB0006A4604A92046FFF75FFF636801228DF8A9
:100DC0002020186859689A68CDF82100CDF82510C0
:100DD000CDF829201B7B8DF82D300023ADF82E3067
:100DE00004A8FFF7DBFE94F820303BB3013B9BB235
:100DF00010AAD11811F8402C11F8101C4A400DF817
:100E00000320F2E77846F9F7EDF8C5E763680122B9
:100E10008DF82020186859689A68CDF82100CDF81F
:100E20002510CDF829201B7B8DF82D300023ADF83F
:100E30002E3004A92046FFF7B3FEB6E7A56094F86C
:100E40002020E169684612F065FAB0FA80F04009A6
:100E5000307010B070BD000030B583B001900D4609
:100E6000040C293CA4B2272C05D8054B33F81430C8
:100E70002B8003B030BD7846F9F7B4F8F5E700BF32
:100E8000F03E002030B583B001900D46040C293CA3
:100E9000A4B2272C06D82A88044B23F8142000205B
:100EA00003B030BD7846F9F79DF8F4E7F03E002036
:100EB00030B583B001900D46040C013CA4B2272C40
:100EC00009D8074B03EBC40153F834204B682A6060
:100ED0006B6003B030BD7846F9F784F8F1E700BFE6
:100EE0004C3D002030B583B001900D46040C013C10
:100EF000A4B2272C11D80B4B03EBC40228686968F5
:100F000043F834005160084B1B781BB9074A13683B
:100F100001331360002003B030BD7846F9F762F862
:100F2000E9E700BF4C3D0020483D0020443D002043
:100F3000F0B583B0FBF784FF0546002413E0784644
:100F4000F9F750F81FE0364B1B6822E07846F9F7B6
:100F500049F839E07846F9F745F83FE07846F9F77F
:100F600041F84BE001342F4B1B68A34254D92E4E5D
:100F700006EBC4062A4B1F88F3889F4203D0013337
:100F80009BB29F42DBD1F2889742DCD2244B1B6894
:100F9000013B1B0C1B0413449D42E3D06A1E9A4282
:100FA000E0D0204A1368013B1360204A1268019286
:100FB000A6B2721CADF806201B4901EBC3010198D3
:100FC00001F016FD0028C1D1164B1B680133ADF8A6
:100FD0000630019801F03DFD0028BBD1134B5B6842
:100FE00001932936ADF806600E4B1968104B03EBE0
:100FF0004101019801F0FCFC0028AFD1094B1B68AE
:101000002933ADF80630019801F023FD0028AAD05D
:101010007846F8F7E7FFA6E7014B1D6003B0F0BD87
:10102000403D0020443D00204C3D0020145604006B
:10103000F03E002008B50378022B00D008BDFFF772
:1010400077FFFBE72DE9F04383B0884616461F463D
:101050000024474D2D68A5424FD9464D05EBC405E8
:10106000AB88834201D00134F3E7424D05EBC40560
:10107000414BB3F80090EB88994503D001339BB204
:10108000994514D1EA88914515D23B4B1B68013B29
:101090001B0C1B0413449E4210D09E4215D9012301
:1010A000ABB907B13C60002003B0BDE8F0837846DF
:1010B000F8F798FFE6E7304B1B68E9E72D4A52F84E
:1010C00034209045E9D90123EAE70023E8E7294BDA
:1010D00003EBC402D68043F83480284B1B6801938D
:1010E000631CADF806302946019801F081FC002808
:1010F000D7D07846F8F776FFD3E7272D01D904201B
:10110000D2E71C4B03EBC5018880CE8043F83580C5
:101110001A4B1B6801930135ADF80650019801F098
:1011200067FCE8B9124B1B6815494FF6FF7221F8AE
:101130001320124A5268019203F12902ADF80620E9
:1011400001EB4301019801F053FC68B917B1084B5A
:101150001B683B60064A1368013313600020A3E755
:101160007846F8F73FFFDDE77846F8F73BFFEDE715
:10117000443D00204C3D0020403D0020145604001A
:10118000F03E002010B50A48FCF7F4FA0024094BA1
:101190001C70094B1C604FF4A0722146074812F0E6
:1011A00015F950222146064812F010F910BD00BF73
:1011B000302E0020483D0020443D00204C3D0020C2
:1011C000F03E002008B5044B01221A70FBF738FEF0
:1011D000024B186008BD00BF483D0020403D002084
:1011E00008B50023FFF72EFF08BD00002DE9F047EA
:1011F00084B006460C461546ADF806308B4260D8E2
:1012000003AB2A4621463046FFF71CFF064600285E
:1012100053D1039F364B33F817204FF6FF739A4292
:101220003ED0BDF80680334B03EBC709324BB3F811
:1012300000A0B9F806309A4503D001339BB29A4515
:1012400043D1B9F80620924543D22B4B1B68013B92
:101250001B0C1B041344274A52F837C0244A32F8A7
:101260001720190A1806CCF30C03934234D2D21A71
:101270006244A2F50052801841F100012B0A2A06AF
:10128000C4F30C0545452AD2A8EB05084444A4F54F
:101290000054121943F10003994208BF90420CD246
:1012A000164B5B680293039B2933ADF80A300DF1AE
:1012B0000601029801F09CFBA8B9304604B0BDE8D5
:1012C000F0877846F8F78EFE9AE77846F8F78AFEB8
:1012D000B7E7094B1B68BBE7D21A6244CBE7A8EB20
:1012E00005084444D5E77846F8F77CFEE5E700BFFB
:1012F000F03E00204C3D0020403D002014560400EC
:101300002DE9F0410E46154600241E4B1B68A342F2
:1013100035D91D4B03EBC4039B88834201D00134B4
:10132000F3E7194F07EBC407184BB3F80080FB88AD
:10133000984503D001339BB2984510D1FA88904567
:1013400011D2124B1B68013B1B0C1B0413449D4222
:101350000CD09D4211D9012080F0010010E07846A8
:10136000F8F740FEEAE7094B1B68EDE7064A52F83A
:1013700034209642EDD90120EEE70020ECE7002072
:10138000BDE8F081443D00204C3D0020403D002060
:101390008B426AD82DE9F8430F4690461E4600243A
:1013A000334D2D68A5425DD9324D05EBC405AB88A0
:1013B000834201D00134F3E72F4B33F814204FF66A
:1013C000FF739A4201D100204DE02A4D05EBC40580
:1013D0002A4BB3F80090EB88994503D001339BB2B8
:1013E000994530D1EA88914531D2244B1B68013BA5
:1013F0001B0C1B0413441F4A52F834501E4A32F887
:101400001420190A1806C5F30C03934222D2D31AEA
:101410002B44A3F50053C01841F100014FEA1823F3
:101420004FEA0862C7F30C04B44216D2361B3744A5
:10143000A7F50057D21943F10003994208BF904223
:101440000ED301200FE07846F8F7CCFDCAE70B4B2E
:101450001B68CDE7D31A2B44DDE7361B3744E9E799
:10146000002000E00020BDE8F8830120704700BFA5
:10147000443D00204C3D0020F03E0020403D002037
:101480008B4267D82DE9F8430F4690461E4600244C
:10149000314D2D68A5425AD9304D05EBC405AB88B6
:1014A000834201D00134F3E72C4D05EBC4052C4BEE
:1014B000B3F80090EB88994503D001339BB299456E
:1014C00034D1EA88914535D2254B1B68013B1B0C72
:1014D0001B041344214A52F83420224931F81440A5
:1014E000190A1806C2F30C03A34226D2E51A1544C2
:1014F000A5F50055421941F100034FEA18214FEAC2
:101500000860C7F30C05AE421AD9761B3744A7F51D
:101510000057C01941F100014FF6FF75AC4212D0DF
:10152000994208BF904210D0002011E07846F8F7A9
:1015300059FDC6E70A4B1B68C9E7E31A9D18D9E7AE
:10154000761B3744E5E7002002E0012000E00020A0
:10155000BDE8F88300207047443D00204C3D00204A
:10156000403D0020F03E002010B50024084B1C60D8
:101570004FF4A0722146074811F028FF502221465F
:10158000054811F023FF052001F08AFA10BD00BFC5
:10159000443D00204C3D0020F03E0020F0B5C7B097
:1015A0000C4616460546F0B12CB3E1B20139C9B27A
:1015B0002878E0B1012820D02C4B1B6813F4807FE1
:1015C00003D02B4B1B68012B1CDC284B1B6813F42E
:1015D000807F10D0264B1B68032B0CDD802C28BF8E
:1015E000802400232BE07846F8F7FCFCDCE7324649
:1015F000681C0CF03FF847B0F0BD3246681C00F0A4
:10160000C7FEF8E71B4BD3F8043501901A4A009245
:101610004C221A490220FEF7A7FAD6E76A1CD25CD0
:10162000174807681609580017F806C005AE06F8EF
:1016300013C002F00F020130BA5C32540133A342EE
:10164000ECD305AA002302F8143003F1804303F51C
:101650008833D3F8043502920A4A01920A4A00926A
:101660004D2206490420FEF77FFAC4E7242E00200D
:10167000202E00200010014054560400485604005B
:10168000282E00207C560400643904002DE9F04126
:101690000546E0B10F4616461C46DAB1E3B1FF2914
:1016A0001CD01C2B1CD803F102085FFA88F808F143
:1016B000010107F000FF054648B180F811802B2397
:1016C0008374C77422463146143011F056FE284602
:1016D000BDE8F0811546FAE70025F8E70025F6E7B2
:1016E0000025F4E7F8B506460D461746884201D8AE
:1016F000344613E07846F8F775FCF9E77846F8F7D2
:1017000071FC21E024F47F6424F00F0404F580547C
:1017100023781C44A5422AD9A6422BD26288BA4219
:1017200026D024F47F6323F00F0303F58053AB42EC
:1017300007D3B2F5FE4F16D0238804EB8303AB42E8
:1017400013D22388002BD9D0238804EB830323F4FE
:101750007F6222F00F029342D4D06288B2F5FE4F2E
:10176000D0D01C46D6E7002402E0002400E000248C
:101770002046F8BD0024FBE7014B1860704700BF0E
:10178000983F0020F8B50E46054688B1A6B12B78E3
:10179000012B15D8304BD3E90823134314D16B68C0
:1017A0001D2B15D82B78012B16D02C4B1C6820E054
:1017B0007846F8F717FCE9E77846F8F713FCE6E710
:1017C0007846F8F70FFCE5E77846F8F70BFCE6E714
:1017D0007846F8F707FCE5E7EB68B3F1FF3FE4D0A4
:1017E00003F50073012BE0D97846F8F7FBFBDCE743
:1017F000246814B3A4F108002A6914F8033C1A42BF
:10180000F6D054F8083C1B68294698470028EFD1C9
:1018100014F8041C0122A1F12003C1F1200002FAF6
:1018200003F322FA00F003438A400B490F6A486A27
:101830003A4303430A624B62DAE7074BD3E90823D2
:10184000134304D06A68044B03F8012B3360024B46
:10185000D3E90801F8BD00BF703F00209C3F002085
:10186000F8B51A4BD3E90823134302D0184B1C6870
:1018700004E07846F8F7B6FBF8E7246804B3A4F16F
:10188000080C124A136A506A14F8045CC5F120016E
:10189000A5F12002EB4000FA01F10B4320FA02F21D
:1018A000134303F00106002756EA0703E5D054F876
:1018B000083C5B68054911F8012B60469847DCE756
:1018C000024B00200021C3E90801F8BD703F002051
:1018D0009C3F0020F8B5194BD3E90823134302D0ED
:1018E000174B1C6804E07846F8F77CFBF8E724689F
:1018F000ECB1A4F1080C114A136A506A14F8045CA4
:10190000C5F12001A5F12002EB4000FA01F10B43E3
:1019100020FA02F2134303F00106002756EA0703F8
:10192000E5D054F8083C9B6860469847DFE7034BD6
:1019300000200021C3E90801F8BD00BF703F00206E
:101940009C3F00202DE9F0410F4616461C4680467C
:1019500050B1074B1D682DB12346324698F804104C
:101960003846A847BDE8F0817846F8F73BFBF0E73A
:10197000983F002070B50C4615460646D8B1F4B124
:101980000DB3FF2D23D023682BB363683BB3A3684B
:10199000002B28D0184B1B783F2B28D83460164AD0
:1019A0001378591C11703371757106F108011348D1
:1019B000FEF71AF870BD7846F8F714FBDFE77846B3
:1019C000F8F710FBDCE77846F8F70CFBD9E7784628
:1019D000F8F708FBD7E77846F8F704FBD5E7784631
:1019E000F8F700FBD3E77846F8F7FCFAD2E7784639
:1019F000F8F7F8FAD2E700BF683F00209C3F0020CC
:101A0000054B5B6833B14FF6FF72934202D0013B46
:101A1000014A5360704700BFAC3F002000B583B05F
:101A2000019040F20713B3EB104F09D1064B00228F
:101A30001A605A609A60DA601A6103B05DF804FBBC
:101A40007846F8F7CFFAF1E7AC3F00202DE9F041F6
:101A500004460F4616461D465B68C3B10A23237031
:101A6000002323732B88E381DFF82C80B8F8000073
:101A70006082FBF701FD20746B68A3616760A6605C
:101A800098F80C302377FF232362BDE8F081784675
:101A9000F8F7A8FAE2E700BFAC3F002000B58DB030
:101AA00003460D4A127B02F07F028DF800200B4A9C
:101AB000127800218DF801108DF80220032269466A
:101AC00003A8FFF7C3FF6FF0020103A8F9F7B0FB0B
:101AD0000DB05DF804FB00BFAC3F0020D43F0020F8
:101AE0000E4B1B88CBB100B583B00D4B1B683BB1CF
:101AF0000B4B1B686846984730B103B05DF804FB98
:101B00007846F8F76FFAF3E76846FFF7C7FF003843
:101B100018BF0120034B1870EFE77047AC3F00205F
:101B200010400020F53F002008B5094B1B781842F3
:101B30000CBF012200228A4200D008BD4340044A63
:101B40001370044BDB890342F7D0FFF7C9FFF4E7BA
:101B5000D43F0020AC3F002000B583B00191C1F319
:101B60000741012902D003B05DF804FB0028FAD137
:101B700011780120FFF7D8FFF5E7000008B50378DA
:101B8000012B00D008BD034B1B78002BFAD0FFF7C8
:101B9000A7FFF7E7F53F002008B5144B1B8823B1DA
:101BA000124B5B6813B1012300E000238BB1104B93
:101BB0001B6893B10E4A13681846B3F5E16F28BF4E
:101BC0004FF4E1600B4901FB00F111611B1A136036
:101BD00008BD074B00221A61FAE7FFF711FFFFF774
:101BE0007FFF024B9A68024B1A60E3E7AC3F00208C
:101BF000D83F002040420F0030B583B001900C4622
:101C000040F20713B3EB104F09D1074D0FCD206001
:101C10006160A260E3602868206103B030BD78464F
:101C2000F8F7E0F9F1E700BFAC3F002010B50D4B2D
:101C30001B789BB10C4B9B681C46B3F5E16F28BF2A
:101C40004FF4E1641B1B094A1360FCF779F808495B
:101C500001FB04010748FCF73FF810BD0024034BCB
:101C60001C60F2E7F43F0020AC3F0020D83F00208A
:101C700040420F00DC3F002008B5044B00225A60B0
:101C80009A600348FCF710F808BD00BFAC3F002085
:101C9000DC3F002070B582B001900C4640F2071383
:101CA000B3EB104F36D12088FBF7E6FB02283FD07C
:101CB0006368B3F5004F03D94FF6FF72934239D1F1
:101CC000A368B3F5803F37D894F90C30002B35DB8F
:101CD0001B4D26460FCE0FC533682B6023882BB9CA
:101CE000A5F1100300225A609A601A73154B1B78F5
:101CF000A3B1134B5B684FF6FF72934214BF0023EE
:101D0000012313B10E4B9B6873B9FFF7B5FF002099
:101D100002B070BD7846F8F765F9C4E7084B5B6818
:101D2000003B18BF0123ECE7FFF780FF0020EFE73F
:101D30000720EDE70720EBE70720E9E70720E7E7C3
:101D4000AC3F0020F43F00200D4B9B681BB1013BD2
:101D50000B4A9360704710B58CB00A48FBF7A4FF9C
:101D6000074C0021A1602C2201A811F02FFB0623B3
:101D70008DF80430029401A8F9F73CFD0CB010BDB9
:101D8000C43F0020F83F002003780A2B47D1C389C5
:101D9000234A1288934242D1418A214A5288914271
:101DA0003DD18268032A3AD11D4A9268002A36D072
:101DB00000B58DB01A4A5268B2F5004F02D2013216
:101DC00017494A6005228DF8042041680A7802F01C
:101DD0007F028DF808200A7802F07F02007F121A35
:101DE000D2B20132D2B28DF80920897801F00F0108
:101DF000ADF80A10ADF80C3093B2094A92899342BB
:101E000001D2074A9381064AD289934201D9044AF2
:101E1000D38101A8F9F7EEFC0DB05DF804FB704723
:101E2000C43F002008B501210C48F9F799FC80B99E
:101E30000B4B0C4ADA600C4B0C4A9A600C4ADA6085
:101E40000C480D4B0360F9F7FDFC0C4B01221A7096
:101E500008BD7846F8F7C6F8EAE700BF9C560400CC
:101E6000D83F0020991B0300F83F0020491D0300C4
:101E700040420F00A03F00207D1B0300F43F0020E4
:101E800070B590B0044600283ED00FA90DF13E0079
:101E900007F0A4F8A368B3F5803F43D82088FBF788
:101EA000EBFA012804D02088FBF7E6FA002839D1A4
:101EB0006088FBF7E1FA58BB254B0BAD0FCB85E8EB
:101EC0000F00A3681BB122880AB1618861BB204B57
:101ED00000221A805A809A601E48FBF7E5FE2C22E9
:101EE0000021684611F072FA06238DF80030BDF823
:101EF0002E305BB30BAB0193154B02936846F9F799
:101F000079FC002010B070BD7846F8F76BF8BCE79C
:101F10006088FBF7B1FA0328CED06288BDF83E3066
:101F20009A42C9D00720EDE7094C22806180A36066
:101F3000084DEE68FBF704FF31182846FBF7CCFE8E
:101F40007F23A3810023E3816360C8E70023D2E7F6
:101F5000C43F0020F83F002000487047C43F0020E5
:101F600000487047AC3F002008B50146034B0022F3
:101F70001A70034B186800F03BFD08BDF43F0020C9
:101F80009056040008B5044B186000B108BD7846AF
:101F9000F8F728F8FAE700BF10400020114B196845
:101FA00048680288013202EB820293005B089BB210
:101FB000B3F5167F28BF4FF416730A2B38BF0A23D8
:101FC00083804A6893780133DBB29370022B00D090
:101FD0007047044A1368596800238B70126852686E
:101FE0001380F5E71441002000B583B00190084B41
:101FF00001221A70074807F025FAFBF7A1FE064BED
:10200000D96801441846FBF767FE03B05DF804FB8E
:10201000F440002014400020FC40002010B582B0A5
:1020200001900C46000CB0F5837F04D1044B1B7863
:10203000237002B010BD7846F7F7D4FFF6E700BF73
:10204000F440002010B582B001900C46000CB0F5B1
:10205000837F0BD12478114B1B7803B954B903B19A
:10206000A4B10E4B1C70002002B010BD7846F7F7EB
:10207000B9FFEFE70A4807F0E5F9FBF761FE094B06
:10208000D96801441846FBF727FEEAE7044807F041
:102090000BFA0448FBF708FEE3E700BFF44000201A
:1020A00014400020FC40002030B585B005460846AD
:1020B00014466B460D222946FCF787FD6B4603CB81
:1020C0002060616005B030BD2DE9F04792B0044654
:1020D0000DF147025449002006F0DCFE0CE0191B0C
:1020E0009288524B03FB02F38B4213D90DF1470246
:1020F0004D49002006F0CEFE4B4B1B68002B5BD0F9
:102100005868FFF74BFF484B1B685A689368E11A01
:10211000E6D5E4E7FAF794FE0546FAF7F5FE9DF8F2
:102120004730022B4BD0404A11680831022B14BFB4
:10213000002201229DF8303062F30003012814BF11
:102140000022012262F341036FF387038DF83030E0
:102150000B4653F8102F5B68CDF83120CDF83530A1
:102160002B0203F47F0343EA05632A0A02F47F4249
:10217000134343EA1563CDF839300DF13D020CA845
:10218000FFF792FF15230CAA01212948FFF77EFAD9
:10219000014688B101230371254807F0C9F9254B91
:1021A0001B6813F0020F03D0234B1B68042B0ADCBF
:1021B0001D4B1B685B689C6012B0BDE8F0871A4A33
:1021C00011682031B2E71D4BD3F804359DF831106A
:1021D0009DF832009DF833609DF834709DF835C04D
:1021E0009DF836E09DF837809DF838909DF83020B6
:1021F000C2F3400A02F001020B950A92CDF824A026
:10220000CDF82090CDF81C80CDF818E0CDF814C0A2
:102210000497039602900191094A0092F722094916
:102220000520FDF7A1FCC3E71441002040420F0048
:1022300014400020242E0020202E002000100140F9
:10224000D8560400C856040008B5FBF779FDFFF71F
:102250003BFF08BD08B5FFF737FF08BD30B583B0B9
:1022600005460C4608220131103011F053F810B128
:10227000002003B030BD6A4629462046FFF714FF10
:10228000082204F10D01684611F044F8B0FA80F01C
:102290004009EEE710B582B00023154A1360154CD3
:1022A000154AE260154AA260236104210DEB01008A
:1022B000FBF780FEFBF744FDE2680199B1FBF2F306
:1022C00002FB1313184460600D4C34230D4A0E4971
:1022D000204607F02FFA4FF47A71204607F0A4F950
:1022E0000A4A04210A48FCF707FD02B010BD00BFEE
:1022F00014410020FC4000208096980055220300E5
:1023000014400020B040002049220300E440002097
:102310001C57040008B5074B1B7803B108BD0648DD
:1023200007F090F80548FBF78FFC024B01221A706A
:10233000F4E700BFF440002014400020FC400020DF
:1023400000B585B08DF807000DF10701054B186841
:1023500000F04EFB10B905B05DF804FB7846F7F7C6
:1023600041FEF8E76857040000B583B00DF107019E
:10237000064B186800F04EFB20B99DF8070003B02B
:102380005DF804FB7846F7F72DFEF6E76857040082
:102390002DE9F04F9BB017460446F8B1002318937F
:1023A000D4F809301D0205F47F0545EA03651A0AD1
:1023B00002F47F42154345EA1365464B1B6813F050
:1023C000020F03D0444B1B68042B0BDC661C0DF181
:1023D000670218A9304606F05DFD61E07846F7F720
:1023E00001FEDBE73D4BD3F804356178A078E67851
:1023F00094F804C094F805E094F8068094F80790E7
:1024000094F808A02278C2F3400B02F001020B9569
:102410000A92CDF824B0CDF820A0CDF81C90CDF8CC
:102420001880CDF814E0CDF810C003960290019109
:102430002B4A00924FF4D1722A490520FDF794FBF4
:10244000C4E77846F7F7CEFD2FE09DF867300BB371
:10245000214618982030FFF701FFD8B1189A203292
:102460002CE001330B8004238DF83430214611F821
:102470000D3BC3F340008DF84C00C3F300038DF80F
:102480004D301295189B0E930F92109711910DA835
:10249000F9F7B0F90DF1670218A9304606F0FAFC19
:1024A000189B9BB15B68002BCBD021461898083055
:1024B000FFF7D4FE0028C8D0189A0832189B596834
:1024C0000B884FF6FF708342CBD1CCE71BB0BDE841
:1024D000F08F00BF242E0020202E0020001001408D
:1024E00024570400C8560400C0EBC000014B03EBA6
:1024F0008000704714350400014B03EBC0007047A7
:102500006438040082B0019189B203681A8891424C
:1025100002D0002002B070475B88BDF806209342CD
:1025200005D8C1880B44934203DC0020F2E7002069
:10253000F0E70120EEE7000010B582B00190074CF3
:10254000074B9C4206D001992046FFF7DBFF10B9EC
:102550001C34F5E70024204602B010BD14350400F9
:102560005C38040002460548054B984204D00388B5
:10257000934202D00830F7E7002070476438040027
:102580009C3804002DE9F04182B00546884601924E
:102590001F460B4C00E008340A4A94420CD02268D3
:1025A00011682846FFF7AEFF0028F4D066683A4667
:1025B00001994046B047EEE702B0BDE8F08100BFA8
:1025C0005C3804006438040008B5064B1B6823B16E
:1025D000044A1368013B136008BD7846F7F702FD13
:1025E000F6E700BF1C41002030B583B004460191DE
:1025F00003685D88C5EB1145C388AB4203D9A06968
:10260000284403B030BD7846F7F7ECFCF7E700004C
:1026100030B58DB0044642884FF6FE739A4237D0EB
:10262000D0F802000B900B98FFF786FF05460028B4
:1026300038D00B992846FFF7D7FF0546037813F0EB
:10264000040F33D02B7823F004032B70224B1B682C
:10265000002B2FD0204A1368013B13602378032BF3
:1026600014D11E4B1B7823B160884FF6FE7398423D
:1026700024D12C220021684610F0A8FE13238DF8E7
:1026800000300B9B01936846F9F7B4F80DB030BDEC
:1026900003781BB9A36818680B90C4E77846F7F76E
:1026A000A1FCF7E77846F7F79DFCC2E77846F7F715
:1026B00099FCC7E77846F7F795FCCBE7FFF752FFA1
:1026C0008378012BD5D12B7813F0020FD1D043F0B2
:1026D00001032B70DAE700BF1841002020410020E1
:1026E00070B5164D1DE07846F7F77CFC23E01C34EE
:1026F000B44215D0A54213D02A68108823681988DF
:102700008842F4D152885988E3880B449A42EEDA21
:10271000EB881A449142EADA7846F7F763FCE6E779
:102720001C35074EB54208D02B685B88EA881344F5
:10273000B3F5803FD7D2014CDAE770BD1435040001
:102740005C38040010B592B0044608460191236934
:1027500002A99847A28802A9019800F0DFFA12B0F6
:1027600010BD0000F0B583B0314B1F68002F3FD182
:10277000304C48E07846F7F735FC4EE001992046AA
:1027800000F0F4FD30E0019800F0F3FA2CE02A4A62
:10279000136801331360A269535D23F0010353559D
:1027A000A269535D43F0040353550135E388AB42FE
:1027B00028D9A3695B5D03F00502012AF5D12268DF
:1027C0001068019005EB1040ADF8060013F0020F01
:1027D000D9D0B378012B03D1184B1B78002BCDD166
:1027E00001992046FFF7AEFF0028D0D0052801D080
:1027F00003B0F0BDA269535D23F001035355D4E744
:102800003D46D3E71C340E4B9C42F1D02368188818
:10281000FFF7A8FE06460028ACD0B378012BEFD016
:10282000022BEFD1054B1B78002BEBD03D46BDE7CB
:102830001C410020143504001841002020410020D4
:102840005C38040000B58DB00378022B07D0FFF789
:10285000DFFE0D4B1B682BB10DB05DF804FBFFF7DD
:10286000B3FEF6E7FFF77EFF084B1B68002BF3D1A2
:102870002C22002101A810F0A9FD12238DF80430AC
:1028800001A8F8F7B7FFE7E71C4100201841002036
:1028900070B582B00446084601911546E3681146BA
:1028A0009847064610B1304602B070BD01992046E7
:1028B000FFF79AFE037843F0030303702368188838
:1028C000FFF750FE40B1FFF74DFF2B46019A002164
:1028D0002046FFF757FEE6E77846F7F783FBF2E777
:1028E000F0B58FB001900D46144680B24FF6FE73DE
:1028F000984216D155F8040B0190141F01231D4A6C
:1029000013701E460198FFF717FE0746C8B183886B
:10291000A34218D8C36829460198984738B10126C0
:1029200012E0114601A805F07FF90026EAE736B16A
:10293000032401993846FFF757FE047016E002247D
:10294000F7E7022600E000262C22002103A810F061
:102950003DFD14238DF80C308DF810600198CDF8F2
:1029600012000695079403A8F8F744FF01200FB062
:10297000F0BD00BF2141002030B583B00024124BD0
:102980001C60124B1C60124B1C70124B1C70FFF72A
:10299000A7FE2046FFF7A8FD05462046FFF7ACFD41
:1029A00002460D490D4BC91A89080D4BA3FB013195
:1029B0000C4B00930C4B0D481B1ADB08284600F00B
:1029C0002DF903B030BD00BF184100201C4100208C
:1029D00020410020214100205C380400143504000F
:1029E00025499224452803009C38040064380400DB
:1029F00010B582B0019049B10C46FFF79DFD38B18A
:102A000022460199FFF744FF02B010BD0E20FBE7FC
:102A10000520F9E730B583B00190B1B10D46FFF75D
:102A20008BFD044698B1037A33B123692946019896
:102A30009847002003B030BD0199FFF7D5FD03781A
:102A400013F0020FF1D10820F4E70E20F2E7052081
:102A5000F0E710B582B00190FFF76EFDD8B10446E3
:102A60000199FFF7C1FD037813F0020F15D003F0B1
:102A7000FD0343F00103037063690BB101989847AC
:102A8000FFF770FE0023019A01212046FFF77AFD2F
:102A9000002002B010BD0520FBE70820F9E7000088
:102AA000F0B583B00646FFF75DFD00282FD007463E
:102AB0001C4C21E00023019A01212046FFF762FD12
:102AC000A269535D23F0030353550135E388AB42FC
:102AD00011D9A3695B5D13F0020FF6D02368186863
:102AE000019005EB1040ADF806006369002BE1D0C2
:102AF00001989847DEE71C340B4B9C4205D02368B5
:102B00001B88B342F7D10025E0E7BB780BB903B0CF
:102B1000F0BD064A136801331360786800F0ECFAE0
:102B2000F5E700BF143504005C3804001C410020A8
:102B300010B5134800F03AF9124B1B780BB9124C40
:102B400008E0104B00221A704FF6FE70FFF7A8FF46
:102B5000F5E708340D4B9C4210D0A378022BF8D136
:102B600022884FF6FE739A42F3D0606800F02BFB88
:102B70000028EED12088FFF793FFEAE710BD00BFE1
:102B8000E128030021410020643804009C3804003F
:102B90007047000001460023094A12689A420CD986
:102BA000084A126802EBC30032F833208A4201D08F
:102BB0000133F1E743681A8070470020704700BF77
:102BC000244100202C41002050B10188013189B2FC
:102BD000002318460F4A12689A421AD930B407E007
:102BE0000021F5E7204601330A4A12689A420ED9BD
:102BF000094A126802EBC30432F833208A42F2D346
:102C00000028EFD00588AA42EDD22046EBE730BC81
:102C100070477047244100202C4100202DE9F843E3
:102C2000884615461C46089E074688B1B8F1000F35
:102C300012D0ADB1C4B1354B00221A60344B1D60C7
:102C4000344B1C60A6B1304600F0F0F900242AE0B5
:102C50007846F7F7C7F9E9E77846F7F7C3F9E8E701
:102C60007846F7F7BFF9E5E77846F7F7BBF9E2E70B
:102C7000294EE8E77846F7F7B5F973685D88B9F843
:102C8000040000F087FAB9F8063003FB0055B5F5EB
:102C9000803F1AD273685D807268B9F806309188F7
:102CA0000B4493800134444513D2C4EBC40307EBB7
:102CB000830957F823301888FFF76CFF0646002871
:102CC000D8D04368002BD8D1D4E77846F7F78AF9F3
:102CD000E0E7002409E07846F7F784F9204600F0A1
:102CE0005EFA0A4A1368034413602046FFF76CFF3C
:102CF000044640B1A378002BF0D0606800F0A8F93A
:102D00000028EBD0E7E7BDE8F88300BF28410020AA
:102D10002C41002024410020912B030070B582B08B
:102D2000019014460E46A1B1BCB1BDF80400FFF7F6
:102D300031FF0546A8B16B685B88B3B16B68BDF81D
:102D40000620DA8022463146686800F0D9F902B0E0
:102D500070BD7846F7F746F9E6E77846F7F742F9A7
:102D6000E3E77846F7F73EF9E5E77846F7F73AF90B
:102D7000E4E710B582B0019080B2FFF70BFF044684
:102D800058B163685B8863B16368BDF80620DA8078
:102D9000606800F0CAF902B010BD7846F7F722F972
:102DA000EFE77846F7F71EF9EEE7000038B505467D
:102DB00008B1002408E07846F7F714F9F9E7294646
:102DC000586800F0CBF90134064B1B68A34207D9C1
:102DD000054B1B6803EBC4039A78002AF3D0EEE797
:102DE00038BD00BF244100202C41002000B583B035
:102DF0000B4649684288CA8059680988ADF80410B2
:102E0000ADF80620014631F8042B02F18042013A68
:102E10001B68920001989847024B185C03B05DF85C
:102E200004FB00BFF057040000B585B0134602B1A3
:102E300003238DF8003030F8083CADF802304B88A1
:102E4000ADF804300B1D02930B8803F18043013B66
:102E50009B000393034B1B686846984705B05DF8D9
:102E600004FB00BF3441002000B585B092B90123B6
:102E70008DF8003030F8083CADF80230ADF80410A1
:102E8000002302930393044B1B686846984705B0E0
:102E90005DF804FB0323EBE73441002000B58DB05F
:102EA0002C22002101A810F091FA0E238DF8043095
:102EB00001A8F8F79FFC0DB05DF804FB30B587B0B2
:102EC0000446436900938369019343880293124B3C
:102ED0000393124B0493124B059369460830FDF798
:102EE00075FD0546042800D050B9042D0CD00D4BBB
:102EF0006363A46304F12C00FDF7D6FD07B030BD79
:102F00007846F7F76FF8F0E7074B6363A46304F1C3
:102F10002C00FDF7C9FDF1E7292E0300692E0300FF
:102F20002D2F0300892F0300812F030010B582B0DD
:102F3000A0F108040D4B1B6813F4801F03D00C4B49
:102F40001B68042B04DC2046FFF7B8FF02B010BD5D
:102F5000084BD3F8043530F8082C0192064A009249
:102F6000A52206490520FCF7FFFDECE7242E0020F2
:102F7000202E002000100140B05704009457040098
:102F800008B5FFF79BFF08BD00B585B0037A022B9B
:102F90000FD102238DF800300388ADF802300023F2
:102FA00002930393064B1B686846984705B05DF88B
:102FB00004FB044B436380632C30FDF775FDF5E79C
:102FC00034410020892F030008B5FDF7C5FD08BD79
:102FD00070B5044600F108063046FDF7D9FD00B192
:102FE00070BD3046FDF7CAFA0546042805D020B169
:102FF00008280ED07846F6F7F5FF042D01D0082DED
:10300000EED1074B6363A46304F12C00FDF74CFD84
:10301000E6E73046FDF7B6FD0028EED1EAE700BF4F
:103020002530030008B5FFF7D3FF08BD08B5054BF1
:1030300000221A70044B1860FDF76AFA0348FDF786
:103040008FFD08BD30410020344100209D2E03003B
:1030500070B58AB00446438803F6F773DB081C4A50
:10306000A2FB03239E091B4D2A7802EB93132B70BE
:10307000FFF7AAFF2B78A0EB033004F108050490BA
:10308000059663880693144B0793144B0893144BCF
:103090000993144B1B6813F4801F03D0124B1B6859
:1030A000062B05DC04A92846FDF790FC0AB070BD8C
:1030B0000E4BD3F804352288029201900C4A0092FC
:1030C00040F25F120B490720FCF74EFDEAE700BF14
:1030D0000508102030410020292E0300692E03002E
:1030E0002D2F0300242E0020202E00200010014050
:1030F000C45704009457040008B5FFF769FF08BDE2
:1031000070B50C461546C1880830FDF741FB50B13B
:1031100006462A462146043010F02FF93046FDF7C6
:1031200075FB002070BD0420FCE730B583B0044679
:103130004FF6FF73ADF80430C388ADF8063000F1E8
:10314000080501A92846FDF714FB28B1E1882846A7
:10315000FDF784FB03B030BD0520FBE730B583B03D
:103160000C46054658B174B1009401956B46084A67
:10317000002105F10800FDF731FA03B030BD7846B3
:10318000F6F730FFEFE77846F6F72CFFECE700BFE5
:10319000ED2D0300073080B220F0030070478378E4
:1031A000022B0ED1436858880330800800EB800260
:1031B00000EBC2009B88642202FB030000F5FA705A
:1031C00070470020704743691A795979521A03EB06
:1031D000023302699B1AC06998428CBF002001200B
:1031E0007047000010B50A4B834202D07846F6F7CC
:1031F000F9FE084B1B6833B1064C206800F039FB20
:103200000023236010BD7846F6F7ECFEF4E700BF1C
:103210003841002050410020F8B50D461446114BAE
:10322000834202D07846F6F7DDFE0F4B1B681B6920
:10323000A34212D30C4E37682246294607F11400E8
:1032400010F09BF839460948FAF7BDFA00233360BD
:10325000074B1868FBF780FBF8BD7846F6F7C2FE0F
:10326000E8E700BF384100205041002044410020E1
:103270004C41002010B50C46104B834202D07846DA
:10328000F6F7B0FE236913F0200F13D00C4B1B6828
:103290000BB1012010BD6068143000F0E6FA084B55
:1032A000186048B123780372E368C3606368036100
:1032B0000020EFE70120EDE70220EBE73841002096
:1032C0005041002030B587B0002300930193029352
:1032D00003930493059303238DF800301048FAF705
:1032E0008EFA0446CCB1E3680193257AFAF728FDFB
:1032F0000246E36829460B48FEF724FB6A4621692B
:1033000004F11400FBF760FF0548FAF778FA054668
:10331000204600F0AEFA2C46E4E7012007B030BDAD
:10332000444100203841002008B50748FBF7F4FA73
:10333000064B1860202206490648FEF71BFB06488C
:10334000FAF736FA08BD00BFC53203004C41002031
:10335000F4570400384100204441002082B000208E
:1033600002B0704782B002B07047000010B594B050
:10337000044601914FF6FE73ADF80830094A1388F0
:10338000ADF80A300133138008460391236904A97C
:103390009847A288043203A90298FFF7BFFC14B033
:1033A00010BD00BF3C2E002030B583B001900D460B
:1033B000C0F30744012C17D80D4804EB84035A01CD
:1033C00000EB43131B792B7083586B7004EB840460
:1033D00000EB4414636F03F5FA73064AA2FB032360
:1033E0009B096B8003B030BD7846F6F7FBFDE3E741
:1033F000D4410020D34D621030B583B001900D460A
:10340000C0F30744023CE4B2012C09D804EB840465
:10341000054B03EB441494F82C302B7003B030BDF3
:103420007846F6F7DFFDF1E7D441002010B582B011
:103430000190C0F30744012C19D804EB8403154A0A
:1034400002EB43131B79B3B1012C1CD004EB8403B2
:103450005B01104A0121D15004EB84040D4800EBBC
:1034600044101421043006F0DFF802B010BD784695
:10347000F6F7B8FDE1E704EB840002EB40100430FE
:1034800005F0E0FFE0E704EB84035B01014A012162
:10349000D150E1E7D441002030B583B001900D4612
:1034A000C0F30744012C0CD86B78013BDBB2072B2F
:1034B00038D86B88143B9BB2B3F5967F05D90720AB
:1034C00031E07846F6F78EFDEEE704EB8403174A09
:1034D00002EB43131A792B7803B18AB103B9C2B94D
:1034E0006A78124804EB84035B01C25004EB840445
:1034F00000EB44106988043006F096F8002012E0D2
:1035000004EB8400094B03EB4010043005F09AFFF4
:10351000E6E704EB8400054B03EB4010043005F0B4
:10352000C3FFDDE7072003B030BD00BFD44100205A
:1035300010B582B00190C0F30744023CE4B2012C04
:103540000AD804EB8404064800EB44100021043040
:1035500006F0ACF802B010BD7846F6F743FDF0E790
:10356000D441002030B583B001900D46C0F307442C
:10357000023CE4B2012C0BD804EB8404064800EBB7
:1035800044102978043006F091F8002003B030BDD3
:103590007846F6F727FDEFE7D441002010B584B058
:1035A0000190C0F30744043CE4B2012C0DD802A8FA
:1035B00006F096F804EB8404064800EB441002A9D8
:1035C000043006F00CF804B010BD7846F6F70AFD9A
:1035D000EDE700BFD441002030B583B001900D4627
:1035E000C0F30744043CE4B2012C08D82B7813F054
:1035F000FE0308D0022B06D0072003B030BD78466A
:10360000F6F7F0FCF2E704EB8404044800EB441006
:103610002946043005F0E3FF0020EEE7D441002006
:1036200030B583B001900D46C0F30744043CE4B2CA
:10363000012C0ED804EB840464016834074B1C444D
:1036400054F8043F2B60A288A379AA80AB7103B021
:1036500030BD7846F6F7C6FCECE700BFD441002049
:1036600010B50D4B834202D07846F6F7BBFC0B4BEE
:103670005B686BB1094C207800EB8000084B03EBD2
:1036800040106168043005F09BFF0023636010BDAB
:103690007846F6F7A7FCEDE7C84100201443002068
:1036A000D4410020F8B50F461546134B834202D093
:1036B0007846F6F797FC114B5B68C3B10F4E746800
:1036C0002A23A3746B1C63742A46394604F1130041
:1036D0000FF053FE307800EB8000094B03EB4010F5
:1036E0002146043005F024FF00237360F8BD7846BE
:1036F000F6F778FCE2E700BFC84100201443002041
:10370000D441002010B50C46144B834202D07846B9
:10371000F6F768FC124B5B6813B17846F6F762FC6B
:103720002078616800EB80000E4B03EB4010023103
:10373000043005F0C0FE0A4B586068B1E3680360CE
:10374000237803EB83035B01064AD3580371227885
:10375000034B1A70002010BD0220FCE7C841002076
:1037600014430020D441002010B50B46043805490D
:10377000401A4011044C04FB00F0C1B20348FEF7AC
:10378000E1F810BDD4410020CDCCCCCCC841002004
:1037900001280ED800B583B0074B1B68019300F5D4
:1037A0008070ADF806000198FFF722F903B05DF8CC
:1037B00004FB0720704700BF0458040001280ED8FE
:1037C00000B583B0074B1B68019300F58070ADF81E
:1037D00006000198FFF71EF903B05DF804FB07200F
:1037E000704700BF0458040070B5104C01262546F0
:1037F00045F8046B4FF480730D4A0E49284605F0D6
:1038000099FF284605F01EFEC4F8A060A43480236A
:10381000094A0021204605F08DFF204605F012FEE2
:10382000324606490648FEF7A5F870BDD44100208F
:103830002843002069370300284400201C58040056
:10384000C841002010B50446012806D804EB8404C2
:10385000044800EB4414207910BD7846F6F7C2FB0B
:10386000F4E700BFD4410020704708B50FF0B4FC66
:1038700008BD08B50FF0F8FC08BD00000378142B54
:1038800000D07047C3880F2BFBD8024B01221A705F
:10389000F7E700BF0045002008B50020F9F7D0FF8A
:1038A00008BD10B50446FDF717F910B123780E2BAB
:1038B00000D010BDFFF7F0FFFBE708B5F9F704FFF4
:1038C00008BD08B5FAF7B9FB01F0E7FC04F0E2F92E
:1038D000F9F7D8F8FDF748FE08BD08B505F0B6FBC6
:1038E00008BD000070B582B0002840D00E460446E6
:1038F000F9F77AFE054610B1284602B070BD04F013
:103900000BFA01F0D5FC20690EF01EFC05460028DC
:10391000F2D1237F0193A3690093636959220021A7
:1039200014480EF089FF05460028E5D1236A03B14B
:103930009847114C2046F9F71DFFFFF7F9F820468C
:10394000F9F71CFF04F090F9044601F0BBFA0B2CC8
:1039500004D00B2802D0094B1B7813B1FFF7B1FF3D
:103960000B25FFF7BAFF002EC6D03070C4E70E2536
:10397000C2E700BFA8440020402E002000450020E0
:1039800008B5FDF7A9F810B1FFF786FF08BD02489A
:10399000F9F7F0FEFAE700BF4C2E002038B50546D7
:1039A000837803F00303032B21D8DFE803F0020C34
:1039B000131981788B081A4A11681944A960194BA8
:1039C0001B6800241AE0837803F0FC0101EB9301EB
:1039D0004B00F0E783789B08642101FB03F3EAE7DF
:1039E00083789B0841F2707101FB03F3E3E77846AB
:1039F000F6F7F8FA0023DEE71C46DB681BB19A688D
:103A00008A1A002AF8DA1CB133B1E560EB6038BDE0
:103A1000EB60044B1D60FAE7E5600023EB60F6E71E
:103A20001C4500202445002010B5714B19688B7887
:103A300003F003036F4A1278934240F3B5808C6819
:103A40006D4B1B68E31A6D4C04FB03F4032A26D864
:103A5000DFE802F0022A2123684BB4FBF3F4644B45
:103A60001B689B7803F00303022B36D0032B57D03F
:103A7000012B1BD000231846002B40F0AC80FAF736
:103A80005FF904465B4B1B78032B00F28680DFE86E
:103A900003F07D8980825A4BDFE75A4BDDE7784699
:103AA000F6F7A0FA0023D8E7574BD6E703F1CC335B
:103AB000A3FB0423DB0803EB8303B4EB430F02D027
:103AC00000231846D8E7FAF73BF900F5742000F513
:103AD00010700123474A1370CEE7464B1A783AB963
:103AE0004A4BA3FB04135B09642101FB13436BB135
:103AF000012A02D000231846BEE7454BA3FB04234E
:103B0000DB0803EB8303B4EB430F3CD1FAF718F95E
:103B100003463B481844374B02221A700123ABE797
:103B2000344B1A7842B93B4BA3FB0413DB0941F237
:103B3000707101FB134383B1012A04D0022A16D00D
:103B40000023184698E7344BA3FB04139B094FF45A
:103B5000167101FB1343002BF0D1FAF7F1F803467D
:103B600028481844234B03221A70012384E72B4B67
:103B7000A3FB04235B09C3EB0313B4EB830FECD06B
:103B80000023184678E70023184675E71B482044B1
:103B900021E01B48FBE71B48F9E77846F6F722FAD5
:103BA0000020F4E71848F2E7FAF7CAF80446104B89
:103BB0001B689B7803F00303032B11D8DFE803F0A5
:103BC00002150C0E0D482044094B1B689B78C3F36B
:103BD0000103084A137010BD0948F4E70948F2E7E9
:103BE0007846F6F7FFF90020EDE70748EBE700BF5E
:103BF00024450020214500201C450020A08601000E
:103C0000809698000046C32340420F001F85EB5169
:103C1000CDCCCCCCF1197605B5814E1B898888882E
:103C200038B5294B1B7873B9284B1B68002B43D040
:103C3000FFF7FAFE0146244B1B78002B34D02448B2
:103C4000FAF74AF83BE0224B5D68FAF779F8044648
:103C5000204B1B78032B16D8DFE803F0021A111350
:103C60001D4B601B18441B4B1B789BB94CF2503307
:103C700098420FD9194A136801331360D4E7184BDF
:103C8000EFE7184BEDE77846F6F7ACF90023E8E7E5
:103C9000154BE6E74009154BA3FB00300F4A1368AC
:103CA00003EBD0101060BFE7074B01221A700848E1
:103CB0004160F9F7C9FF02E0034B1B7803B938BD37
:103CC0000348F9F7F1FFFAE72045002024450020DA
:103CD0000445002021450020A08601001C4500204D
:103CE000809698000046C32340420F00C55A7C0AC4
:103CF00030B583B009E07846F6F774F96368019946
:103D0000284698472046FFF749FE0F4B1C68B4B180
:103D1000A3680E4A1268934204D00C4A12689B1A98
:103D2000002B0CDA2588E268074B1A600023019308
:103D300001A9284602F004F90028DFD0DBE7FFF7ED
:103D40006FFF03B030BD00BF244500201C4500209C
:103D500008B5134B1B78032B1ED8DFE803F0020CC9
:103D60001116104A1368013313600F4B00221A70AA
:103D7000FFF7BEFF08BD0B4A13680A331360F4E770
:103D8000084A136864331360EFE7064A136803F5C3
:103D9000BB5310331360E8E77846F6F723F9E4E7FE
:103DA000214500201C4500202045002010B5044678
:103DB000FFF7F4FD034B1B68A34200D010BDFFF7D3
:103DC0002FFFFBE724450020074A002313605360C0
:103DD000D3601361536105499160054A1360054A38
:103DE0001360054A1370704704450020513D0300DD
:103DF0001C450020244500202045002008B5054B27
:103E00001B7813B9FFF7E0FF08BD0348F9F74CFF33
:103E1000F8E700BF204500200445002070B50E469D
:103E20001546044650B1FAF7FFFC144B1B680020FE
:103E300043B1A34206D01846DB68F9E77846F6F7A7
:103E4000D1F8F0E7A17866F3010165F38701A1706D
:103E500013B138B1DA68C26045B903B150B1FAF7AD
:103E600027FD70BDD968054A1160F5E72046FFF7C8
:103E70009DFFF4E7FFF7D4FEF1E700BF24450020E3
:103E800000234FF6FF70032B22D830B404E018460D
:103E900001339BB2032B19D803EBC30291000D4AE7
:103EA0000A4492F83920002AF2D04FF6FF7290426D
:103EB000EDD0084A1144096B00EBC005AC00224468
:103EC000126B8A1A002AE3DA1846E1E730BC704721
:103ED000704700BF2845002070B5044600EBC002C3
:103EE0001A4B03EB820393F8393033B3174BB3F813
:103EF000A83033B3154A04EBC40302EB830300215B
:103F000083F83910B2F8A830013B9BB2A2F8A83070
:103F100023B913464FF6FF72A3F8AA200B4DE60013
:103F200004EBC40305EB8303986AFFF7A2FC344457
:103F300005EB84050023AB6270BD7846F6F752F8B6
:103F4000D4E77846F6F74EF8D4E700BF28450020BE
:103F5000F8B506464E4BB3F8A8301BB106F57A7794
:103F6000002421E07846F6F73DF8F7E72046FFF712
:103F7000B3FF17E0002861D105EBC502444B03EB0A
:103F8000820292F83830013BDBB282F83830002BE5
:103F900058D03F4A05EBC50302EB8303596B1A6BFC
:103FA000114419630134A4B2032C4FD8254604EB05
:103FB000C403374A02EB830393F83930002BF1D066
:103FC00004EBC40302EB83031B6BDB1B002BE9DA5E
:103FD000104604EBC4018900183104EBC40200EB65
:103FE0008202938D926A0144204601F037F910282D
:103FF000C0D801A353F820F0793F0300753F0300B8
:10400000753F0300753F0300793F03006D3F0300D8
:10401000753F03006D3F0300793F03006D3F0300D0
:10402000753F0300753F0300753F0300753F0300B4
:10403000753F0300793F03006D3F03007846F5F7B5
:10404000D1FF99E72046FFF747FFABE7FFF718FFDF
:104050000F4BA3F8AA00B3F8A830A3B103280CD8DB
:104060000B4BB3F8AA2002EBC20203EB82031B6BDB
:104070009A1B06D4064BDA60F8BD7846F5F7B2FF16
:10408000EEE7F21AF6E7024B0022DA60F4E700BF2F
:10409000284500202DE9F8430446884616469946EF
:1040A000F9F74EFE8646154F04EBC40507EB850570
:1040B00005F1180C96E80F008CE80F00C5F8289061
:1040C000BDF82030AB8598F80030C3F3020385F8C3
:1040D000383098F80000C3084CF2503003FB000061
:1040E000686370442863012385F83930B7F8A83035
:1040F0000133A7F8A830BDE8F88300BF28450020A9
:1041000010B50446FFF7BCFE0E4BB3F8AA3083424D
:1041100011D00C4BA3F8AA004FF6FF7398420DD0B4
:104120000848B0F8AA3003EBC30300EB8303196B14
:10413000F9F7D2FD10BDA342FCD1EAE77846F5F7C6
:1041400051FFEDE72845002010B5064CAA220021BA
:1041500020460FF03BF9044BA3604FF6FF73A4F821
:10416000AA3010BD28450020513F03002DE9F04141
:1041700082B004460D4616461F46BDF8208003282F
:104180001FD815B32EB32B7813F0070F25D047B3E4
:10419000B8F1000F29D004EBC403184A02EB8303E3
:1041A00093F839302BBBCDF800803B463246294688
:1041B0002046FFF76FFF2046FFF7A2FF02B0BDE8E1
:1041C000F0817846F5F70EFFDBE77846F5F70AFF52
:1041D000D8E77846F5F706FFD5E77846F5F702FF0A
:1041E000D5E77846F5F7FEFED2E77846F5F7FAFE12
:1041F000D1E72046FFF770FED5E700BF2845002035
:104200004FF6FF7399420CD00C4B00EB400203EBCE
:104210004202D27800EB400003EB4000531CC37015
:104220007047064B00EB400203EB4202927800EB32
:10423000400003EB4000531C837070471846002079
:1042400030B482B001911B4B00EB400103EB410104
:10425000897800EB400403EB4403DB78D94201D0BA
:10426000002303E0002021E001339BB2032B1CD884
:10427000C3EB0311104C04EB8101098A8142F3D195
:10428000C3EB031104EB81014C88BDF806108C428E
:10429000EAD1C3EB0315084931F82540BDF80410F5
:1042A0008C42E1D11380012000E0002002B030BC3C
:1042B000704700BF184600203046002082B000231F
:1042C0000093027802F0C003802B1ED012D80BB1ED
:1042D000402B05D1ADF800204FF6FF73ADF802304A
:1042E000009B00209AB262F30F001B0C63F31F4087
:1042F00002B07047C02BF3D1ADF80020437882782C
:1043000043EA0223ADF80230EAE7437843EA0222A7
:10431000ADF800204FF6FF73ADF80230E0E782B051
:1043200001904FF6FF72B2EB104F08D0030CBDF8AE
:1043300004200A704B701B0A8B7002B07047BDF8E6
:10434000043013F47F4F03D01A0A0A704B70F4E75D
:104350000B70F2E782B001904FF6FF73B3EB104F92
:1043600018D1BDF8040010F47F4F07D000F440408E
:10437000B0F5004F14BF0020012014E020F07F03AF
:104380009BB22BB97F2801D001200CE000200AE06D
:10439000002008E0BDF8040020F03F0080B2C028F3
:1043A00014BF0020012002B0704770B506460D46CC
:1043B0000024AC4207D256F83400FFF7CBFF034687
:1043C00010B10134F5E70123184670BD30B482B056
:1043D0000191002300E00133018E994210D9C16A96
:1043E00001EBC30531F83340BDF804108C42F2D123
:1043F0006C88BDF806108C42EDD11360012000E0FE
:10440000002002B030BC7047428A032A0FD80A4B02
:1044100003EB021304334A0953F8223001F01F0161
:1044200023FA01F111F0010F03D0012070470020A1
:1044300070470020704700BF28470020000CA0F5FF
:10444000405080B2032820D8114B1B7813F0040F82
:1044500017D00020704751F82320D44303EB800588
:104460000C4A02EB850254600133022BF3D9094A4E
:104470000001135C03F0F9031354002002B030BCB8
:10448000704730B482B00023EFE70520704700BFCB
:10449000244700202847002082B0000CB0F5805F40
:1044A0001AD1114B1B7813F0040F18D1A0F58050CE
:1044B00080B20A8800EB40010C4B33F811309A426D
:1044C0000FD10A4B03EB4102527903EB410002F09A
:1044D000F9034371002000E0052002B0704700207E
:1044E000FBE70B20F9E700BF244700201846002017
:1044F00082B0000CB0F5804F05D10A78034B1A70DA
:10450000002002B070470520FBE700BF582E0020B6
:1045100010B582B001900C46000C012806D1012391
:1045200063800423A380238002B010BD7846F5F792
:1045300059FDF4E710B582B001900C46000C01283B
:104540000FD16388012B10D1A388042B10D12388AD
:10455000042B0FD1084A137843F001031370002095
:1045600004E07846F5F73EFDEBE70B2002B010BD06
:104570000B20FBE70B20F9E72447002030B583B080
:1045800001900D46040CA4F54054A4B2032C01D8AC
:1045900000230DE07846F5F725FDF9E703EB8401EC
:1045A000054A02EB81025268D24345F823200133C9
:1045B000022BF3D903B030BD2847002030B583B0BB
:1045C00001900D46040CB4F5805F0AD1A4F5805427
:1045D000A4B204EB4404054B33F814302B8003B031
:1045E00030BD7846F5F7FEFCF0E700BF1846002026
:1045F00010B582B001900C46000CB0F5804F04D18C
:10460000044B1B78237002B010BD7846F5F7EAFC26
:10461000F6E700BF582E0020F8B504460D461646B2
:104620001F4653B12B89B3F5BE7F0AD309233B60E4
:104630003868B0FA80F04009F8BD7846F5F7D2FC4A
:10464000F0E7032C0BD8C4EB04131C4A02EB8303E2
:1046500093F8383013F0010F0DD1002300E0002350
:1046600033B1C4EB0413154A02EB83031B8A23B155
:1046700005233B60DCE70123F2E736B12868FFF74A
:1046800069FEB8B907233B60D2E7C4EB04130B4AB9
:1046900002EB83039A884FF6FF739A42F2D0C4EB81
:1046A0000414064B03EB8404E2884FF6FF739A422E
:1046B000E4D1E7E700233B60BAE700BF30460020C3
:1046C000F8B50E4617461D460C4603281AD8DFE8F3
:1046D00000F00502101401EB81004400BDF8180041
:1046E000B4FBF0F03F2816D800233B7076B92B704E
:1046F000F8BD642000FB01F4F0E741F2707000FBAC
:1047000001F4EBE77846F5F76DFCE7E7012838BFE1
:1047100001202870ECE740F27623984208D8012364
:104720003B7003F1CC33A3FB0030C0082870DFE7F7
:1047300041F69C03984207D802233B70064BA3FB2B
:10474000003040092870D3E703233B70034BA3FBE1
:104750000030C0092870CBE71F85EB51F1197605B1
:1047600030B583B001900D46040CA4F50054A4B2FA
:10477000032C13D80B4AC4EB041402EB840352F845
:1047800024105A689C68D86829606A60AC60E86048
:1047900019695A6929616A6103B030BD7846F5F735
:1047A00021FCE7E730460020000CA0F5005080B265
:1047B000032847D8294B1B7813F0040F44D1F0B4D9
:1047C00082B00C8AC0EB0013254A02EB83031B8ADC
:1047D0009C423BD10A88C0EB0013214C34F82330B3
:1047E0009A4237D14C88C0EB00131D4A02EB830379
:1047F0005B889C4230D14C8AC0EB001302EB8303F0
:104800005B8A9C4201D00B2021E0C0EB001602EB3A
:1048100086030D684C68D1F808C0CF6842F826506E
:104820005C60C3F808C0DF600D694C691D615C61A4
:1048300093F8383002EB860003F0F90380F8383043
:10484000002004E005207047002070470B2002B0D4
:10485000F0BC70470B20FAE70B20F8E72447002054
:104860003046002038B50446C0884FF6FF739842A2
:104870000FD1628A042A4BD0274B03EB02131D1D74
:104880005A6800235AB90133022B13D855F8232054
:10489000F8E703F09DFA03460028EAD039E05142D8
:1048A0000A401E4901FB02F2D20E1D498C5C04EB4A
:1048B00043140DE056240BE062421440174A02FBF9
:1048C00004F4E40E164A145D04EB431400E056248D
:1048D000562C1BD0A0B203F013FB0346C8B9013419
:1048E000552CF4D8630955F8232004F01F04012146
:1048F00001FA04F464421440002CDDD10133022B90
:1049000002D855F82340F7E75624E1E7002300E0FA
:104910000023184638BD00BF2847002031B57C076A
:10492000185904000D4B1B7813F0040F06D10C4AE4
:104930000001135C43F004031354704700B583B0C7
:10494000084B1B68019300F54050ADF80600019834
:10495000FEF77FF803B05DF804FB00BF244700209A
:1049600028470020E8580400184B1B7813F0040F68
:104970000AD000B585B0164B1B68009300F5405374
:10498000ADF80230002313E0124A0001135C43F03B
:1049900002031354704703EB80010E4A02EB8102BD
:1049A0005268D24304A901EB830141F80C2C013376
:1049B000022BF0D901A90098FEF71AF810B905B03A
:1049C0005DF804FB7846F5F70DFBF8E72447002077
:1049D000E858040028470020134B1B7813F0040FFD
:1049E00009D1124B00EB400203EB4202537943F032
:1049F00002035371704700B583B00D4B5B680193A0
:104A000000F58053ADF8063000EB4000074901EB9C
:104A100040010198FDF7ECFF10B903B05DF804FB0D
:104A20007846F5F7DFFAF8E724470020184600201B
:104A3000E8580400144B1B7813F0040F0BD1134BF0
:104A4000C0EB001203EB820292F8383043F002030D
:104A500082F83830704700B583B00D4B9B680193E6
:104A600000F50053ADF80630C0EB0010074901EB2C
:104A700080010198FDF7BCFF10B903B05DF804FB9D
:104A80007846F5F7AFFAF8E72447002030460020D3
:104A9000E858040038B500240AE02046FFF742FF3A
:104AA0002A492B01CA5C02F0F902CA540134A4B2AB
:104AB000032C0DD825462301244AD35C13F0040FA0
:104AC000EBD113F0020FEBD02046FFF74DFFE7E7E5
:104AD00000240CB1002429E0254604EB44035A00CD
:104AE0001B4B13445B7913F0020F0BD1184A05EBF3
:104AF00045014B0013445A7922F002025A710134E5
:104B0000A4B2E6E72046FFF767FFEFE72046FFF78E
:104B100091FF104AC5EB05118B00134493F8382020
:104B200022F0020283F838200134A4B2032C0BD8FF
:104B30002546C4EB04139A00064B134493F838300F
:104B400013F0020FE5D0E1E738BD00BF2847002091
:104B5000184600203046002000B585B0084B596942
:104B600018690190ADF8081001A9D868FDF740FF59
:104B700010B905B05DF804FB7846F5F733FAF8E7AD
:104B8000E858040030B583B004460D460378012B85
:104B900007D042884FF6FB739A420CD8002003B02E
:104BA00030BD01A803F000F96388BDF804209B1A0A
:104BB0002B800120F3E700230B800120EFE70000AA
:104BC00010B5F022002114480EF000FC134B002415
:104BD0001C609C804022214611480EF0F7FB2146C4
:104BE00013E00D4AC1EB0110830013444FF6FF7030
:104BF000D880988004245C821882C1EB0110830065
:104C00001A4401231385194489B20329E9D9054BB4
:104C100028221A7010BD00BF304600201846002020
:104C200028470020582E00202DE9F04FD3B005462C
:104C3000884614461F46BDF8709151A803F0B4F899
:104C4000C5EB0512644B03EB82031E8ABDF84631A7
:104C50009E4280F0BA80BDF844311E44B6B23CB3E7
:104C6000B4F81EA0B4F824B04FAB2169E06883E823
:104C700003000CB1247F3CB1C5EB0515564800EB91
:104C800085056C7DFF2C28D057B3B9F1000F2BD0D0
:104C90002422002146A80EF099FB4CAA5146584602
:104CA00004F034F8054618B3284653B0BDE8F08F39
:104CB000C5EB0513484A02EB8303B3F804A04FA9E0
:104CC000D88803F063F9002840F08180BDF83E31B8
:104CD000002B7ED04FF6FF7BCBE7404B1C78D3E711
:104CE0007846F5F77FF9D0E77846F5F77BF9CFE717
:104CF00046AB50994F9883E80300ADF820618DF8DA
:104D0000224198F80A208DF8232198F80B208DF87D
:104D100024214A97ADF82C91D8F80C204E9200210E
:104D20001846F8F723FD05460028BDD12C4B1B681B
:104D300013F4005F03D02B4B1B68042B20DC284BA3
:104D40001B6813F4005FAFD0264B1B68042BABDD50
:104D5000B9F1800F28BF4FF080092B464B451ED27A
:104D6000FA5C21490C6810095900265C05A800F876
:104D7000136002F00F020131A25C42540133EDE7EF
:104D80001A4BD3F80435B8F800200192184A009263
:104D900040F2A91217490520FAF7E6FECFE705AA67
:104DA000002302F8193003F1804303F58833D3F868
:104DB00004350292104A0192104A00924FF4D572C3
:104DC0000C490520FAF7D0FE6EE710256CE70525A3
:104DD0006AE7102568E700BF30460020582E002003
:104DE000242E0020202E0020282E0020001001401C
:104DF000585804004E5804006C58040064390400EC
:104E000008B5054A137803F0FE036FF341031370EE
:104E10000220FDF745FE08BD244700202DE9F0479C
:104E200084B0064690461F460C4691B303AB4246FB
:104E300021463046FFF7F0FB78B3236802934FF624
:104E4000FF72B2EB134F2CD04FF0030A2589554463
:104E5000ADB22846FEF709FD814688B301462068B9
:104E6000FFF75DFA2289616809EB0A000EF085FA06
:104E700000954B46424621463046FFF7D5FE03904B
:104E8000C8B9C7B10C9BB3B1C7F800900C9B1D808B
:104E900004E07846F5F7A6F8C8E7039804B0BDE843
:104EA000F087BDF80830FF2B02D94FF0020ACDE79A
:104EB0004FF0010ACAE74846FEF7DBFC0398EDE72E
:104EC0000420EBE738B5224A137843F0040313704B
:104ED00013F0020F37D113F0010F27D0002401E0A7
:104EE0000134A4B2032C21D8C4EB0413194A02EBF9
:104EF00083031A8A4FF6FF739A42F1D0C4EB041071
:104F0000144B03EB8000FFF7ADFCF0B9114BC4EB81
:104F1000041203EB8202927DC4EB041503EB8505BA
:104F200002F0FC036FF38703AB75D9E7FFF7B2FD1F
:104F3000074B1B7813F0010F01D0002038BDFFF79D
:104F40000BFE0520FAE70B20F8E70B20F6E700BF81
:104F500024470020304600202DE9F04F8DB0064652
:104F600000F11404204604F04BF810B90DB0BDE870
:104F7000F08F4FF6FF73ADF82A300AA92046FFF7ED
:104F800001FE099008B100243DE00DF12A01204600
:104F900003F0AAF80028F6D07846F5F723F8F2E7F0
:104FA000BDF82A103846FFF72FFA81463EE03F4B06
:104FB000D3F804353E4AC4EB041102EB810032F809
:104FC000212041880697CDF814B0CDF81090CDF887
:104FD0000CA002910192374A00924FF48662364942
:104FE0000720FAF7C1FD47E0C4EB0413304A02EB97
:104FF0008303DA6A0B9902EBC10255685A6B31469A
:10500000A0B2A8470134032CB0DCC4EB0417284B32
:1050100003EB8707099B002BC2D0388ABDF8289084
:10502000814514BF4FF000094FF00109204AC4EB3D
:10503000041302EB830393F8388008F0010AC4EBF1
:1050400004139B0008331344F28B510953F8215089
:1050500002F01F02D54005F0010B0BAA316838465B
:10506000FFF7B4F90746154B1B6813F4005F03D034
:10507000134B1B68062B9ADCBAF1000FC2D0B9F1B2
:10508000000FBFD0BBF1000FBCD0002FBAD0337DD2
:10509000012BA9D1C4EB0413054A02EB83035A6B1D
:1050A0003146A0B201F062FA9EE700BF0010014055
:1050B00030460020745804004E580400242E00206E
:1050C000202E00202DE9F041D0B00446002868D001
:1050D0002068FFF7F3F84F9085B27F2D00F09580A0
:1050E0004B4B1B6813F4005F03D04A4B1B68042B27
:1050F0005BDCE06903F079F88046A06903F05EF8B4
:105100004F9B459326684FF6FF72B2EB134F58D072
:1051100003231E444696A3884F9A04924FF6FF71CC
:10512000B1EB124F53D003229B1A9FB2ADF81C7102
:10513000237A8DF820316389ADF82231E3684993F1
:10514000237C8DF82831638AADF82A3163694B934B
:1051500094F820308DF83031ADF83281636A4D9388
:10516000ADF838012A4B1B6813F4005F4AD0294B75
:105170001B68042B46DD802F28BF80270023BB42FD
:105180002BD2F25C24490C6810095900255C04A854
:1051900000F8135002F00F020131A25C42540133B7
:1051A000EDE77846F4F71EFF92E71C4BD3F8043581
:1051B00001951B4A0092FD221A490520FAF7D4FCFA
:1051C00097E7FF2D01D90223A3E70123A1E7FF2DD4
:1051D00001D90222A8E70122A6E704AA002302F8C7
:1051E000173003F1804303F58833D3F80435029276
:1051F0000D4A01920D4A00924FF48A720949052026
:10520000FAF7B2FC45A8FFF7A7FE50B0BDE8F08161
:10521000242E0020202E0020282E002000100140E7
:10522000CC5804004E580400E058040064390400CF
:1052300008B5037813B1142B04D008BD0430FFF770
:1052400041FFFAE7C388022BF7D1034A137843F0F2
:1052500002031370F1E700BF24470020B1B1F0B59D
:1052600085B0064614461D460F468AB193B103AB7E
:105270000022FFF7D1F908B903980CE00095234606
:10528000002239463046FFF7CFFC04E00E2070477D
:105290000E2000E00E2005B0F0BD08B501F0B4F915
:1052A000FEF7ACFDFFF78CFCFFF7AAFD08BD000080
:1052B00008B5FFF785FC0948094B0360F8F75AFA6F
:1052C00001F08EF9FEF780FDFEF73EFF054A1378E8
:1052D00003F0FC036FF38203137008BD2446002023
:1052E0003152030024470020002800F0B08070B540
:1052F0000C460546002900F0AC80C3681BB18368EA
:10530000002B00F0A8804FF6FF732380EB681BB9D9
:10531000AB68002B40F0A180AB88002B40F09F8051
:1053200003F094FE002841D122462968A888FEF7A0
:1053300087FF50B12388C3EB03134C4A02EB83036E
:1053400093F8383013F0010F30D1E968A868FFF7FF
:105350002CF8002800F0858020884FF6FF739842D3
:1053600066D022882969414BC2EB021203EB82020C
:1053700051632288A968C2EB021203EB8202D16258
:10538000E9682288C2EB021203EB820211862288AE
:105390006969C2EB021203EB8202D1612288C2EB7F
:1053A000021103EB81031A83002059E00F2057E01C
:1053B00098B220804FF6FF73984254D02B4EC0EB2A
:1053C000001006EB80001A46C3802388C3EB03134A
:1053D00006EB83039A802388A988C3EB031306EBAB
:1053E0008303198223886988C3EB031306EB8303C5
:1053F000598023882988C3EB031326F823102388B8
:10540000C3EB031306EB83035A752988A888FEF7BC
:10541000F7FE2388C3EB031206EB820292F83830C2
:1054200043F0010382F838302088FFF703FB98E748
:105430000023032BBDD8C3EB03120C4901EB8202FE
:1054400092F8382012F0010FB2D00133F1E70E20AC
:1054500070470E2004E00E2002E0092000E0052045
:1054600070BD0720FCE70420FAE700BF30460020AB
:1054700070B584B051B304460D460022ADF80E203D
:105480000DF10E03009302ABFFF7C8FC0646B0B95E
:10549000C4EB04130E4A02EB8303DB7D13F0070F0A
:1054A00010D0C4EB0411890010311144BDF80E3046
:1054B0000093029B2A4607312046FEF757FE3046EE
:1054C00004B070BD0298FEF7D4F9F8E70E26F6E7AF
:1054D0003046002059B110B582B014460A4644B196
:1054E000002300932146FFF799FC02B010BD0E2067
:1054F00070470E20F9E7000008B503280BD8C0EB71
:105500000013144A02EB830393F8383013F0010FB1
:105510000FD1002300E00023BBB1552917D8C0EB01
:1055200000130C4A02EB8303DB888B4203D100207B
:1055300008BD0123F0E7C0EB0012064B03EB82032A
:10554000D980FFF777FA0020F2E70520F0E707207F
:10555000EEE700BF30460020F1B110B40C4603283E
:105560000BD8C0EB00130E4A02EB830393F83830DC
:1055700013F0010F0ED1002300E0002373B1C0EB44
:105580000010074B03EB8000C388238000205DF8E8
:10559000044B70470123F1E70E2070470520F6E722
:1055A0003046002003282AD808B5C0EB0013174A5C
:1055B00002EB830393F8383013F0010F21D0C0EBD6
:1055C000001302EB8303DB7D03F0070301F0070206
:1055D00093420AD1C0EB00130C4A02EB8303DA7D3D
:1055E000C1F3C403B3EBD20F0DD0C0EB0012074BD5
:1055F00003EB8203D975FFF71DFA002008BD0520D3
:1056000070470520FAE70020F8E700BF3046002089
:10561000B1B110B4032815D8C0EB00130B4A02EB4C
:10562000830393F8383013F0010F0DD0C0EB001056
:1056300002EB8000C37D0B7000205DF8044B7047C7
:105640000E2070470520F8E70520F6E730460020D9
:1056500081B310B40C467AB303280BD8C0EB001307
:10566000184901EB830393F8383013F0010F1FD171
:10567000002300E000230BB3C0EB0013114901EB42
:105680008303DB69E3B10B46C0EB001103EB81013F
:10569000897DC1F301012170C0EB001003EB800094
:1056A000837DC3F38503137000205DF8044B7047BE
:1056B0000123E0E70E2070470E20F6E70520F4E70F
:1056C0000620F2E73046002070B584B0054600237E
:1056D0008DF80F308DF80D300DF10D020DF10F0129
:1056E000FFF7B6FFE0B9104E2C01C5EB051306EB32
:1056F00083031B8D009303AB0DF10E029DF80D107B
:105700009DF80F00FEF7DCFF601B800018309DF84D
:105710000C209DF80E103044FEF780FB04B070BDE5
:105720007846F4F75FFCDEE73046002003281BD8FC
:1057300008B5C0EB0013104A02EB830393F838302E
:1057400013F0010F12D0C0EB001302EB8303DB69EF
:1057500073B179B1C0EB0012074B03EB82031985DB
:10576000FFF7B2FF002008BD052070470520FAE7CB
:105770000620F8E70720F6E73046002003283DD84A
:1057800010B50446C0EB0013224800EB830393F8E6
:10579000383013F0010F33D0C4EB041300EB830354
:1057A000DB697BB33F2A2FD803292FD8C4EB04131E
:1057B00000EB83039B7DB2EB930F08D1C4EB041382
:1057C00000EB83039B7D03F003038B4220D0114841
:1057D000C4EB041300EB83039B7D62F38703C4EBEC
:1057E000041200EB820061F3010383752046FFF78A
:1057F0006BFF2046FFF71EF9002010BD0520704703
:105800000520FAE70620F8E70720F6E70720F4E787
:105810000020F2E73046002010B5044603F016FCE5
:1058200000283BD1032C0BD8C4EB04131E4A02EB17
:10583000830393F8383013F0010F16D1002300E0F2
:1058400000236BB3C4EB0413174A02EB83035B8A98
:10585000042B27D1002003281ED80301134AD35C50
:1058600013F0010F03D00130F5E70123E9E703F05E
:10587000FB03020143F001030C498B5480B2C4EBDB
:105880000412094B03EB82035882FFF76DF82046A0
:10589000FFF7D0F8002006E0042004E00F2002E02B
:1058A000052000E0002010BD3046002028470020E1
:1058B00070B503280BD8C0EB00131F4A02EB83031B
:1058C00093F8383013F0010F1ED1002300E00023BD
:1058D0005BB3C0EB0013184A02EB83035A8A042A15
:1058E00025D0552925D8154B03EB021304334D0958
:1058F00053F8252001F01F0122FA01F414F00104ED
:1059000004D00024204670BD0123E1E7012606FAF9
:1059100001F10A4343F82520C0EB0010064B03EBCE
:105920008000408AFFF720F8ECE70524EAE7062428
:10593000E8E70724E6E700BF3046002028470020BC
:1059400038B5034603280BD8C0EB00121E4800EB05
:10595000820292F8382012F0010F1CD1002200E0E0
:1059600000225AB3C3EB0312174800EB8202508A9D
:10597000042825D0552925D8144A02EB00120432F8
:105980004D0952F8254001F01F0124FA01F010F0F2
:10599000010002D138BD0122E3E7012000FA01F144
:1059A00024EA010442F82540C3EB0313064A02EB44
:1059B0008303588AFEF7D8FF0020EBE70520E9E7CC
:1059C0000620E7E70720E5E73046002028470020CB
:1059D00000293ED02DE9F84317468846002A3AD0E0
:1059E00003280BD8C0EB00131F4A02EB830393F884
:1059F000383013F0010F11D1002300E0002363B30E
:105A00000646C0EB0010184B03EB8000438A042BC2
:105A100025D0B7F8009000243C8002E00123EEE797
:105A20000134552C13D8C6EB0610A5B229460E4BEF
:105A300003EB8000FEF7E8FC0028F1D03B88994595
:105A40000FD928F813503B8801333B80E8E700204A
:105A500008E00E2070470E2004E0052002E006203A
:105A600000E00920BDE8F8833046002070B5032827
:105A70000BD8C0EB0013184A02EB830393F83830BD
:105A800013F0010F18D1002300E00023FBB12929F6
:105A90001FD8C0EB00139B0008330F4A13444D0975
:105AA00053F8252001F01F0122FA01F414F001043B
:105AB00004D00024204670BD0123E7E7012606FA42
:105AC00001F10A4343F82520FEF7B4FFF2E705246D
:105AD000F0E70724EEE700BF3046002038B5034664
:105AE00003280BD8C0EB0012184800EB820292F892
:105AF000382012F0010F16D1002200E0002202B37C
:105B0000292920D8C3EB0312920008320F4802441F
:105B10004D0952F8254001F01F0124FA01F010F060
:105B2000010002D138BD0122E9E7012000FA01F1AC
:105B300024EA010442F825401846FEF77BFF0020C6
:105B4000F0E70520EEE70720ECE700BF3046002035
:105B5000A1B370B40D469AB303280BD8C0EB001361
:105B60001A4901EB830393F8383013F0010F0AD17F
:105B7000002300E000232BB316880023138023B1F9
:105B8000002070BC70470123F5E7C0EB00118900CD
:105B900008310E4C21445C0951F8241003F01F0415
:105BA000E14011F0010F07D011888E420CD925F881
:105BB00011301188013111800133E0E70E20704768
:105BC0000E20DEE70520DCE70920DAE7304600207A
:105BD00008B503280BD8C0EB0013144A02EB83036B
:105BE00093F8383013F0010F0FD1002300E00023A9
:105BF000BBB1292917D8C0EB00130C4A02EB830371
:105C00009B888B4203D1002008BD0123F0E7C0EB45
:105C10000012064B03EB82039980FEF70BFF002076
:105C2000F2E70520F0E70720EEE700BF304600204E
:105C3000F1B110B40C4603280BD8C0EB00130E4A88
:105C400002EB830393F8383013F0010F0ED10023D9
:105C500000E0002373B1C0EB0010074B03EB8000A2
:105C60008388238000205DF8044B70470123F1E70F
:105C70000E2070470520F6E73046002000B585B0BD
:105C80008DF8070010F0800F0AD101280AD00DF11D
:105C90000701054B9869FCF7ABFE05B05DF804FB06
:105CA0000720FAE70720F8E7E8580400014B1878C6
:105CB000704700BF582E0020F1B110B40C460328E5
:105CC0000BD8C0EB00130E4A02EB830393F8383075
:105CD00013F0010F0ED1002300E0002373B1C0EBDD
:105CE0000010074B03EB8000037D237000205DF85C
:105CF000044B70470123F1E70E2070470520F6E7BB
:105D00003046002008B503280BD8C0EB0013154A15
:105D100002EB830393F8383013F0010F11D1002305
:105D200000E00023CBB181F080037E2B17D9C0EBBC
:105D300000130C4A02EB83035B7D8B4203D10020EE
:105D400008BD0123EEE7C0EB0012064B03EB820314
:105D50005975FEF76FFE0020F2E70520F0E70720F7
:105D6000EEE700BF30460020F1B110B40C46032826
:105D70000BD8C0EB00130E4A02EB830393F83830C4
:105D800013F0010F0ED1002300E0002373B1C0EB2C
:105D90000010074B03EB8000437D237000205DF86B
:105DA000044B70470123F1E70E2070470520F6E70A
:105DB0003046002041B148B900EB4000044A32F8B7
:105DC00010200A80002070470E2070470520704781
:105DD0001846002049B150B900EB4000054B03EBD9
:105DE000400083780B70002070470E20704705201C
:105DF000704700BF1846002049B150B900EB400081
:105E0000054B03EB4000C3780B70002070470E2059
:105E100070470520704700BF184600200A46F9B1B8
:105E200003280BD8C0EB00130F4901EB830393F851
:105E3000383013F0010F11D1002300E000238BB1A3
:105E40000949C0EB001301EB83035B885380C0EB6F
:105E5000001031F820301380002070470123EEE756
:105E60000E207047052070473046002030B482B0C5
:105E700001915AB3154658BB4FF6FF731380034682
:105E800001E001339BB2032B1CD8C3EB0312114971
:105E900001EB8202128A8242F3D1C3EB031201EBBF
:105EA00082025188BDF806209142EAD1C3EB031467
:105EB000084A32F82410BDF804209142E1D12B8029
:105EC000002000E0052002B030BC70470E20FAE749
:105ED0000520F8E73046002039B3F0B40F4632B35E
:105EE00038BB16880023138000E00133032B19D838
:105EF0001588B5421FD2C3EB0311104C04EB81018E
:105F000091F8381011F0010FEFD0C3EB031104EB3F
:105F10008101098A8142E8D127F8153011880131C1
:105F20001180E2E70020F0BC70470E2070470E2081
:105F3000F9E70520F7E70920F5E700BF3046002024
:105F4000F1B110B40C4603280BD8C0EB00130E4A75
:105F500002EB830393F8383013F0010F0ED10023C6
:105F600000E0002373B1C0EB0010074B03EB80008F
:105F7000436B236000205DF8044B70470123F1E779
:105F80000E2070470520F6E7304600202DE9F0414D
:105F9000044603280BD8C0EB0013224A02EB83030C
:105FA00093F8383013F0010F37D1002300E00023BD
:105FB000ABB31C4F4FEA0418C4EB04108000183038
:105FC000002211463844FDF729FF204600F058FB17
:105FD000A8EB040507EB8505E88801F045FF4FF6BF
:105FE000FF73EB80AB80EB7D03F0F8036FF3C70327
:105FF000EB7500266E75AB7D03F0030366F30103BA
:10600000AB75AB7E03F0030366F30103AB7620466A
:10601000FEF710FD3046BDE8F0810123C8E70520FA
:10602000F9E700BF3046002029281AD830B583B0E0
:106030000546002401E00134A4B2032C0ED80DF172
:1060400006012046FFF7F4FD0028F4D1BDF8063024
:10605000AB42F0D12046FFF799FFECE7002003B0F8
:1060600030BD07207047000010B44FF6FF730B805F
:10607000002300E00133032B0ED80C4C2C2202FB32
:10608000034292F84020002AF4D02C2202FB034263
:10609000128B8242EED10B8008884FF6FF73C01A34
:1060A00018BF01205DF8044B704700BF7047002007
:1060B0000B4BB3F8C83073B1094AB2F8CA302C217F
:1060C00001FB03239B6B01FB0020826B9B1A002BBF
:1060D00003DB01207047012070470020704700BF9C
:1060E0007047002010B4124B2C2202FB0030836B4F
:1060F000104C1C4400234FF6FF7001E001339BB2AB
:10610000032B11D80A492C2202FB031292F84020DB
:10611000002AF3D02C2202FB0312926B111B0029E0
:10612000ECDA18461446E9E75DF8044B704700BF07
:106130007047002000879303F8B507460E461546C2
:106140004FF6FF730B8004231360F8F76DFB164BBB
:10615000B3F8C830042B25D9F8F7AAFB2868B0FAA1
:1061600080F04009F8BD10492C2202FB0312118B6C
:106170003A88914213D00133032BEDD80A4A2C24DC
:1061800004FB032494F84020002AECD131884FF618
:10619000FF729142EFD100222A603380EBE708239F
:1061A0002B60D9E70023E7E77047002010B50446CD
:1061B000204A2C2303FB002393F84030B3B11D4B3E
:1061C000B3F8C830B3B11B4A2C2303FB04230021CE
:1061D00083F84010B2F8C830013B9BB2A2F8C83037
:1061E00023B3B2F8CA30A34208D010BD7846F3F703
:1061F000F9FEE4E77846F3F7F5FEE4E72046FFF71B
:1062000071FF0C4BA3F8CA004FF6FF73984209D0F8
:106210000848B0F8CA302C2202FB0303996BF7F749
:106220005BFDE2E77846F3F7DDFEF1E70148F7F7BB
:106230003BFDDAE770470020F0B585B005466B4BB3
:10624000B3F8C8305BB16A4B01221A7005F57A7653
:10625000664B4FF6FF72A3F8CA20002491E07846FF
:10626000F3F7C0FEEFE72C2303FB0423002183F8A0
:106270004010B2F8C8100139A2F8C81003A9188B51
:10628000FFF75EFE48B9594A2C2303FB04235F6BDA
:1062900001220399188BB84772E07846F3F7A2FE03
:1062A000F1E7524BA3F8CA402C2202FB04F202F1A0
:1062B0001801194413440431188BFFF7D9F8074625
:1062C00040B14C4B1B6813F4005F03D04A4B1B6872
:1062D000042B0ADCAFB1082F13D0042F2AD00F2FC4
:1062E00028D07846F3F77EFE15E0444BD3F804350A
:1062F0000190434A0092832242490520F9F734FC79
:10630000E8E73A4A2C2303FB0423DA6B996B114428
:1063100099635200DA63354A2C2303FB04231A6B7A
:106320009B6BD31A002B2BDA30492C2303FB04136D
:106330009A6325E02D4B2C2202FB0434A36B03F55A
:106340001C434033A363294BB3F8C830002B49D01A
:10635000264BB3F8CA30032B3ED8244AB2F8CA30D1
:106360002C2101FB03239B6B5A1B39D41F4BDA6092
:106370001F4B00221A7005B0F0BD1C4BA3F8CA4099
:106380000134032CDFD8194A2C2303FB042393F890
:106390004030002BF4D02C2303FB04231B6B9B1BEE
:1063A000002BFFF660AF114A2C2303FB04239B6BE9
:1063B0009A1B002AFFF675AF0C4AB2F8CA204FF6B6
:1063C000FF718A42D9D009492C2000FB0212926B3E
:1063D0009B1A002BD4DAD0E77846F3F703FEBCE72C
:1063E000EA1AC3E7014B0022DA60C1E770470020D8
:1063F0006C470020242E0020202E00200010014099
:10640000705904005E59040010B582B004460DF1C5
:1064100007010088FFF7A8FC48BB9DF80730FF2B59
:1064200029D0636800934FF6FF72B2EB134F27D069
:106430000322A38913449BB29DF8070044F620620F
:1064400002FB00F202F5433202F5A0720B2B08D9D1
:106450000B330F4981FB03135B1044F6206101FBF2
:106460000322A069904228BF104602B010BD7846B2
:10647000F3F7B8FDD1E7FFF719FC8DF80700D0E777
:10648000BDF80030FF2B01D90222D2E70122D0E76C
:10649000ABAAAA2A2DE9F04105460C46314A2C2325
:1064A00003FB002393F84030002B48D1F7F748FC5A
:1064B00007462C4E2C2303FB05F808F1180E06EBBB
:1064C0000E03D4F800C06068A168E26846F80EC008
:1064D00058609960DA60D4F810C06069A169E26917
:1064E000C3F810C058619961DA612046FFF78CFF4C
:1064F00006EB0803D8631A6B3A441A63384498636E
:10650000F8F792F9184B1B782BB1B6F8CA204FF662
:10651000FF739A4217D02846FFF7CAFDB0B9114B56
:106520002C2000FB0535012285F84020B3F8C82057
:106530000132A3F8C820F8F7BBF9BDE8F08178462E
:10654000F3F750FDB2E7A6F8CA50E8E7054C2C2354
:1065500003FB0543996B2046F7F7BEFBA4F8CA502E
:10656000DDE700BF704700206C47002070B582B0A7
:1065700004460E461546032815D8F8F755F90DF1CF
:1065800006012046FFF770FD48B1BDF80600134A2A
:106590002C2303FB00239A8D33889A4207D0F8F707
:1065A00087F902B070BD7846F3F71CFDE5E70B4AAA
:1065B0002C2303FB0023DA8D73889A42EFD1FFF777
:1065C000F5FDBDF80630054A2C2101FB03235B6B6A
:1065D0000022294620469847E1E700BF7047002087
:1065E00010B5064CCC22002120460CF0EFFE044BE7
:1065F000A360044B00221A7010BD00BF704700203A
:10660000396203006C47002070B582B0F8F70CF9CE
:106610001A4BB3F8C8300BB900240EE0174800231A
:10662000A0F8C830F7F740FBF6E77846F3F7DAFC56
:10663000022201992846B0470134032C1AD80F4A88
:106640002C2303FB042393F84030002BF4D0104696
:106650002C2202FB04F3C1180D8B4E6B1833002162
:1066600018440CF0B3FE01A92846FFF769FC002886
:10667000DED0DAE7F8F71CF902B070BD70470020F1
:1066800010B582B0032803D90524204602B010BDFE
:106690000446F8F7C9F80DF102012046FFF7E4FCC3
:1066A00018B90524F8F704F9EFE7BDF80200FFF781
:1066B0007DFD01A92046FFF743FC60B9BDF802301B
:1066C000074A2C2101FB03235B6B02220199204620
:1066D00098470024E6E77846F3F784FCEEE700BF2E
:1066E0007047002048B310B582B00446C36933B385
:1066F0000388032B25D88369A3F5F413A3F59063CE
:10670000124A93421FD801AA0DF10201FFF714FDAE
:1067100008B9019818E0214631F8040BFEF7A8FEED
:10672000019018B1042801D008280DD12146BDF8E8
:106730000200FFF7AFFE002006E00E2070470E209B
:1067400002E0052000E0072002B010BD80027503C2
:1067500003460F4A126812F0010F0AD00D4A128840
:1067600090420AD30B4840880244934207DB002240
:1067700000E00022104622B970470022FAE7012209
:10678000F8E74B8001230B7000234B60F4E700BF58
:1067900048480020444E00200B8833B901334FF69F
:1067A000FF720A80FBB910B40AE00023F7E703EB9D
:1067B00083020E4C34F8222082420DD0013373B98B
:1067C0005A090B4C54F8222003F01F04E24012F047
:1067D000010FECD10B80F1E70B80012000E00020DD
:1067E0005DF8044B70470020704700BF084F002041
:1067F0004C4800204FF6FF730B800023542B21D808
:1068000010B407E00C884FF6FF72944216D00133A3
:10681000542B15D85A090C4C54F8222003F01F04AD
:10682000E24012F0010FEDD0084A32F823208242F4
:10683000EDD10B8001205DF8044B70470B80E6E73B
:106840000020F8E7002070473C4800205048002016
:106850004FF6FF730B800023282B25D810B407E0D8
:106860000C884FF6FF72944219D00133282B19D8A7
:106870005A090E4C54F8222003F01F04E24012F093
:10688000010FEDD0162202FB03F2094CA25A8242FC
:10689000EBD101330B8001205DF8044B70475A1C8B
:1068A0000A80E2E70020F7E700207047D449002083
:1068B000DC4900204FF6FF730B8000235BB1002002
:1068C00070470B8001201CE00C884FF6FF72944249
:1068D00013D10B8011E010B45A090B4C54F822204C
:1068E00003F01F04E24012F0010FEDD02A2202FB58
:1068F00003F2064CA25A8242E3D00133002BEBD0C4
:1069000000205DF8044B7047A4490020A8490020EE
:10691000F0B416680023136013B10120F0BC704777
:106920005C09114D55F8244003F01F05EC4014F0AC
:10693000010F06D00D4D2A2404FB035464888442C1
:1069400001D00133E8E71568B5420AD02A2404FBD8
:1069500003F4064F3C5B21F81540146801341460C1
:10696000EFE70020DAE700BFA4490020A849002093
:1069700070B40D6800230B6013B1012070BC704728
:106980005A090D4C54F8222003F01F04E24012F083
:10699000010F0CD00C68AC420BD0AC2202FB03F20E
:1069A000064EB25A20F814200A6801320A600133F8
:1069B000E2E70020E2E700BF584E00205C4E0020D6
:1069C00030B445091A4C54F8254000F01F05EC403E
:1069D00014F0010F2AD0174CAC2505FB004090F8AD
:1069E000640010B114788C4209D010B11878884234
:1069F0000ED013788B4212D0002030BC70471C7828
:106A00008C42F2D102990A60039A13600120F4E7E4
:106A1000029A13600023039A13600120EDE7029BA2
:106A20001A600023039A13600120E6E70020E4E7E0
:106A3000584E00205C4E0020B0B110B40446002334
:106A4000282B0FD8162202FB03F208498A5AA242C9
:106A500001D00133F4E7162202FB0313181D5DF881
:106A6000044B70470020FAE700207047DC49002003
:106A7000292860D830B480BB334C80BB03465D0905
:106A800054F8254003F01F0324FA03F313F0010F19
:106A900053D00C884FF6FF739C4222D00B88002BFA
:106AA0004DD15909294C54F8211003F01F04E1403D
:106AB00011F0010F45D0002833D12549AC2404FB47
:106AC000031393F86430022B1AD022492A2303FBC4
:106AD00000100430106000202BE01F4CCDE7431E57
:106AE000CDE730B91B4C2A2303FB00435B880B80A6
:106AF000D4E7431E194C162505FB03435B88F6E7D4
:106B000014492A2303FB00139B7D002BDDD02A238D
:106B100003FB00F010300B460344073313600020E2
:106B200007E001380D4B162101FB003004301060E6
:106B3000002030BC7047052070470520F9E7082089
:106B4000F7E70820F5E700BFA4490020584E0020D1
:106B50005C4E0020A8490020D4490020DC490020D8
:106B60000A4B23F8210003EB81030022DA709A70AC
:106B70004809074A01F01F01012303FA01F152F805
:106B800020300B4342F82030704700BF50480020AF
:106B90003C48002010B582B001900B46000CA0F5D7
:106BA000805081B2542911D84A09094850F822402E
:106BB00001F01F02D44014F0010403D00024204649
:106BC00002B010BD1888FFF7CBFFF8E70524F6E701
:106BD0003C48002010B582B001900C46000C012802
:106BE00009D1012323802922A28063802381552398
:106BF000E38002B010BD7846F3F7F4F9F1E7000046
:106C000010B582B001900C46000C012815D12388E4
:106C1000012B16D1A388292B16D16388012B15D1FE
:106C20002389012B14D1E388552B13D10A4A1378F9
:106C300043F001031370002004E07846F3F7D2F923
:106C4000E5E70B2002B010BD0B20FBE70B20F9E7B6
:106C50000B20F7E70B20F5E7544E002010B582B06B
:106C600001900C46000C022809D1094B1B6813F057
:106C7000010F08D0074B1B68236002B010BD784697
:106C8000F3F7B0F9F1E77846F3F7ACF9F2E700BFB4
:106C900048480020444E002030B583B001900D4696
:106CA000040CA4F58054A4B2542C0FD863090B4AE9
:106CB00052F8233004F01F02D34013F0010F09D023
:106CC000074B33F824302B8003B030BD7846F3F700
:106CD00089F9EBE77846F3F785F9F1E73C480020BE
:106CE0005048002010B5044630B10A4B9C420ED3E8
:106CF00006D94FF6FF700CE07846F3F773F9F4E726
:106D0000E01A054CA4FB0030C0F34F1001E04FF631
:106D1000FF7010BDD04E002083BEA02F38B50446B2
:106D200020B1002030B14FF6FF7038BD7846F3F740
:106D300059F9F6E71449AC2303FB001393F86410E8
:106D4000A1B1AC2303FB00F303F120020E4B13446B
:106D50000233A342E9D0AC2303FB00F303F140026A
:106D6000094B13440333A3420AD1DEE7AC2303FBF0
:106D700000F303F12002044B13440233A342D4D0A6
:106D8000013080B2CEE700BF5C4E002010B5044653
:106D900058B1002068B1184B9C4229D303F55C73AD
:106DA0009C421BD94FF6FF7024E07846F3F71AF99E
:106DB000EFE7124A2A2303FB00230433A3420BD03C
:106DC0002A2303FB00F303F110020C4B1344073397
:106DD000A34201D00130DDE780B20BE0A3F55C7087
:106DE000201A074CA4FB00300009013080B201E0FA
:106DF0004FF6FF7010BD00BFE0490020A8490020F9
:106E0000A38B2EBA2DE9F84306460F4690469946C5
:106E10001068002874D0FFF7B9FF013018E06BB19B
:106E20003C4A2A2303FB00239B7D3BB12A2303FB1F
:106E300000231B7E7B4013F03F0F49D0354A2A23A5
:106E400003FB00235B797B4013F03F0F4ED00130F2
:106E5000002857D14509304B53F8255000F01F0347
:106E6000DD4015F0010FF2D02A4A2A2303FB00234C
:106E70005B88B342EBD1294AAC2303FB062393F88A
:106E80006430002BCBD023492A2202FB0012927DD2
:106E9000002AC4D02A2202FB001252797A4012F052
:106EA0003F0FBCD12A2202FB0012127E7A4012F060
:106EB0003F0FB4D10B462A2202FB00F40A19043218
:106EC000C8F80020103423440733C9F800301EE00E
:106ED0002A2303FB00F303F110020E4B1344073384
:106EE000C8F800300023C9F8003010E02A2303FB63
:106EF00000230433C8F800300023C9F8003006E04E
:106F00000020A5E70023C8F80030C9F80030BDE82C
:106F1000F88300BFA8490020A44900205C4E00204F
:106F200030B583B001900D46000C022808D10E4BFD
:106F30001C6814F0010407D00024204603B030BDC3
:106F40007846F3F74FF8F2E72888F6F795FA012824
:106F500008D12A68054B1A60034A136843F00103FD
:106F60001360EAE70B24E8E748480020444E00207D
:106F700070B506460D4614464FF6FF730B80F6F7C4
:106F80007BFA2070022822D0032841D0012841D06A
:106F9000002020E029884FF6FF72914208D003EBD1
:106FA00083021E4931F82220B2420DD001330FE096
:106FB0005A091B4951F8222003F01F01CA4012F060
:106FC000010FECD12B80F1E72B80012003E000239F
:106FD000002BDFD0002070BD124A32F82320B242CD
:106FE00013D00133542B17D82C884FF6FF729442DC
:106FF000F2D15A090C4951F8222003F01F01CA406E
:1070000012F0010FE8D12B80EBE72B800120E2E7A3
:107010000023E7E70023E5E70020DCE7084F002036
:107020004C480020504800203C48002030B583B038
:1070300001900D46040CB4F5005F1ED1A4F500507C
:1070400084B2C0F34A12114B53F8223000F01F00F3
:1070500023FA00F010F0010F13D004EB84040C4B62
:1070600003EB840353F8040F59689A68DB682860BF
:107070006960AA60EB6003B030BD7846F2F7B2FFFA
:10708000DCE77846F2F7AEFFE7E700BF4C480020A8
:10709000084F0020F0B583B001900D46040CA4F514
:1070A000A044A4B2282C1ED86309134A52F82330F6
:1070B00004F01F02D34013F0010F18D00F4916231C
:1070C00003FB04F40A19134653F8067F5E689868B8
:1070D000DB686F60AE60E8602B610B5B2B805388D0
:1070E0006B8003B0F0BD7846F2F77CFFDCE77846B2
:1070F000F2F778FFE2E700BFD4490020DC49002026
:10710000F0B5013B124E162505FB03F57419D2F8B4
:1071100000E0D2F804C09768D268C4F806E0C4F86A
:107120000AC0C4F80E70C4F8122000226271012255
:107130002271618070535809064903F01F0302FA57
:1071400003F351F82020134341F82030F0BD00BF75
:10715000DC490020D449002030B583B00190000CF8
:10716000A0F5A04292B2282A19D80D4651090D4B1C
:1071700053F8214002F01F0224FA02F212F0010437
:1071800003D00024204603B030BDA0F59F407F38D7
:1071900083B22A1D69882888FFF7B2FFF2E7052429
:1071A000F0E700BFD449002070B5A1F1550404EB0D
:1071B00084020F4901EB8201066845688268C36852
:1071C0004E608D60CA600B61F8F7E4FB60B961093D
:1071D000084A04F01F04012303FA04F452F8213092
:1071E000234342F8213070BD7846F2F7FBFEEEE70C
:1071F000084F00204C48002010B582B00190030CCD
:10720000B3F5005F17D10A46A3F50051C1F34A1444
:107210000B4850F8244001F01F01CC4014F0010449
:1072200001D0002408E0A3F5FD530B3B99B21046B2
:10723000FFF7BAFF00E00524204602B010BD00BFF2
:107240004C48002070B582B001900D46040CB4F596
:10725000405F2ED1A4F54054A4B224220021284638
:107260000CF0B4F86209214B53F8223004F01F02ED
:10727000D34013F0010F20D01D49AC2303FB04F3CE
:10728000CA18CB5A2B8092F86430AB70134653F86F
:10729000026F58689968DB68C5F80360C5F8070095
:1072A000C5F80B10C5F80F3092F864304BB902B036
:1072B00070BD7846F2F796FECCE77846F2F792FE7C
:1072C000DAE7AC2303FB04F404F11003084C1C447C
:1072D00054F8020F6168A268E368C5F81300C5F8A6
:1072E0001710C5F81B20C5F81F30E0E7584E0020E6
:1072F0005C4E0020F0B583B001900C46050CB5F54E
:10730000804F2DD1A5F58045ADB226220021204623
:107310000CF05CF86A091F4B53F8223005F01F028D
:10732000D34013F0010F1FD01B482A2202FB05F2A5
:1073300081180B4653F806CF5F689E68DB68C4F877
:1073400005C0C4F80970C4F80D60C4F81130835A40
:1073500023804B8863808B7D23714BB903B0F0BDD4
:107360007846F2F73FFECDE77846F2F73BFEDBE7E3
:1073700002F1100305461D4455F8090F6968AA6813
:10738000EB68C4F81500C4F81910C4F81D20C4F83F
:107390002130E3E7A4490020A8490020F8B50D46B4
:1073A00014462D4BAC2202FB04F202F16801194491
:1073B00013449967064610B9284B01221A70AC2174
:1073C00001FB04F12031244B194402312846F8F71F
:1073D000A2FAC8BBAC2101FB04F178311E4B194461
:1073E00004312846F8F7ACFA90BB1B4FAC2000FBE9
:1073F00004F03A18D5F800E0D5F804C0A968EB68A5
:10740000C2F802E0C2F806C0C2F80A10C2F80E3094
:1074100000F110033B440021C3F80210C3F806102A
:10742000C3F80A10C3F80E103E5282F864106109C6
:107430000B4A04F01F04012303FA04F452F821302C
:10744000234342F82130F8BD7846F2F7CBFDC1E77F
:107450007846F2F7C7FDC8E75C4E0020414E002099
:10746000584E0020F0B583B00190000CB0F5405F9D
:107470003ED10D46A0F5405086B2C0F34A121E4BD5
:1074800053F8224000F01F0024FA00F010F001042D
:1074900001D000242DE031F8030B3246FFF77EFFC8
:1074A000AA781649AC2303FB061383F8642002B3C1
:1074B000AC2303FB06F606F110030B44284650F8F4
:1074C00013CF47688568C268C3F802C0C3F8067066
:1074D000C3F80A50C3F80E20403631440331F8F7A0
:1074E0001AFA08B9044604E07846F2F77BFD00E09A
:1074F0000524204603B0F0BD584E00205C4E00200D
:1075000030B583B001900D46040C04F54054A4B28C
:1075100031F8030B2246FFF741FFAB78064AAC2156
:1075200001FB042484F86430044A137843F0040314
:107530001370002003B030BD5C4E0020544E00207C
:107540002DE9F04106460D4610461C461F4B2A22E7
:1075500002FB04F29918D0F80080D0F804E0D0F8CB
:1075600008C0C768C1F80680C1F80AE0C1F80EC0BB
:10757000C1F81270103213440022C3F80920C3F876
:107580000D20C3F81120C3F815200531F8F7B8F91C
:10759000B8B90E492A2303FB04F3CA18002010715E
:1075A0009075CE5255806109094B04F01F040122E9
:1075B00002FA04F453F82120224343F82120BDE8C5
:1075C000F0817846F2F70EFDE3E700BFA8490020FE
:1075D000A4490020F0B583B00190000CB0F5804FB5
:1075E00042D10D46A0F5804086B2C0F34A12204B2E
:1075F00053F8224000F01F0024FA00F010F00104BC
:1076000001D0002431E033464A1D49882888FFF71D
:1076100097FF2A7917492A2303FB06139A7522B389
:107620002A2101FB06F101F11003124919442846F1
:1076300050F8157F45688268C368C1F80970C1F8C1
:107640000D50C1F81120C1F815300831F8F758F97C
:1076500030B9084B2A2202FB06363379F37504E071
:107660007846F2F7BFFCF4E70524204603B0F0BDEE
:10767000A4490020A8490020F0B583B001900D4630
:10768000000CB0F5604F1BD0B0F5704F41D100F544
:10769000805084B20126204A137843F0040313700B
:1076A00023462A1D69882888FFF74AFF27461B4A78
:1076B0002A2303FB04239E753EB9002003B0F0BDCE
:1076C00000F5005084B20026E5E72A2101FB04F40E
:1076D000103411462144284650F8145F44688268EB
:1076E000C368C1F80950C1F80D40C1F81120C1F8B4
:1076F00015300831F8F704F938B9084B2A2202FB93
:1077000007373B79FB750020D8E77846F2F76AFC2B
:10771000F3E70520D2E700BF544E0020A84900201F
:1077200010B584B0084A52F8044B6B4607CA03C32D
:107730001A8069462046FBF75BF908B904B010BD12
:107740007846F2F74FFCF9E7045A040030B583B0ED
:1077500005460C460023ADF800304B0952F82330A3
:1077600001F01F02D34013F0010F0CD00123ADF83C
:1077700004302C44ADF8064069460198FBF738F90F
:1077800028B903B030BD7846F2F72CFCEEE7784616
:10779000F2F728FCF5E70000002940D070B582B070
:1077A000054614460E460DF1070201A9FFF7E0FB5E
:1077B0002CB99DF80730032B01D010201DE0012CBF
:1077C0001DD078B9BDF804104FF6FF73994228D048
:1077D0002846FFF7C5F9144ABDF804104FF480504D
:1077E000FFF7B4FFBDF80430338084B90F4A02EBD1
:1077F0008303DA780132DA70002002B070BD9DF8A0
:107800000730032BDDD0012BDBD01020F5E7074A32
:1078100002EB83039A7801329A700020EDE70E2084
:1078200070470420E9E700BF3C4800205048002092
:10783000264B1B7813F0040F46D030B583B0234B92
:107840001A786FF382021A70214B1B69019300248E
:1078500034B11F4B5B6901930024DCB103B030BD30
:1078600063091C4A52F8233004F01F02D34013F07E
:10787000010F0DD0A5B205F54053ADF806300198C3
:10788000FBF7E7F8134A29464FF44050FFF75EFF35
:107890000134DDE76309104A52F8233004F01F0277
:1078A000D34013F0010F0DD0A5B205F58043ADF81C
:1078B00006300198FBF7CDF8074A29464FF480407F
:1078C000FFF744FF0134C8E7704700BF544E002063
:1078D000045A0400584E0020A44900202DE9F0412C
:1078E00082B007460C4615464E0952F8263001F084
:1078F0001F0823FA08F313F0010F15D00123ADF888
:1079000004303C44ADF806400198FBF7A2F878B982
:10791000012303FA08F255F8263023EA020345F85A
:10792000263002B0BDE8F0817846F2F75BFBE5E770
:107930007846F2F757FBEBE708B5542820D84309FF
:10794000254A52F8233000F01F02D34013F0010FF4
:1079500016D0224B03EB80039B7823B91F4B03EB1C
:107960008003DB780BB1002008BD1C4B002223F8FC
:107970002020194A01464FF48050FFF7AFFFF2E78D
:10798000A0F1550189B219BB4B09154A52F82330B1
:1079900001F01F02D34013F0010F1BD001EB810354
:1079A000104A02EB83039B782BB901EB810302EBB6
:1079B0008303DB780BB10020D6E701EB81039B004A
:1079C0000020D052064A4FF40050FFF787FFF2E73D
:1079D0000520C9E70520C7E73C48002050480020A3
:1079E0004C480020084F002008B5054A137803F0E2
:1079F000FE036FF3410313700120FBF751F808BD3C
:107A0000544E002070B506460D464FF6FF730B80AE
:107A100000240CB1002070BD6309104A52F82330D5
:107A200004F01F02D34013F0010F06D12A884FF64D
:107A3000FF739A420CD12C800AE004EB8400084BBF
:107A400003EB80001022314604300BF063FC08B1D8
:107A50000134DEE72C800120DDE700BF4C48002028
:107A6000084F0020F0B583B04FF6FF73ADF8063035
:107A7000002840D00C461646074600293DD00DF19F
:107A80000601FFF7BFFFBDF8063003F15505ADB2A3
:107A900070B94FF6FF72934231D029463846FFF74E
:107AA00083FB184ABDF806104FF40050FFF74EFE56
:107AB000258086B9BDF80630134A03EB830102EB3B
:107AC0008101C97803EB830302EB83034A1CDA705C
:107AD000002003B0F0BDBDF806300B4A03EB830174
:107AE00002EB8101897803EB830302EB83034A1CD9
:107AF0009A700020EDE70E20EBE70E20E9E7042066
:107B0000E7E700BF4C480020084F002030B583B0A5
:107B100005460C46486820B10DF10601FFF772FFDB
:107B200018B94FF6FF73ADF806300DF1060128467F
:107B3000FEF732FEB0B1BDF8063003EB83030A4A0C
:107B400002EB8303DB7863B1658002232370BDF809
:107B5000063003EB8302044B03EB820304336360C0
:107B600000E0002003B030BD084F002038B50546C6
:107B70004FF6FF730B8000230BE05A09134850F8AF
:107B8000222003F01F00C24012F0010F08D10B8029
:107B90000133542B12D80C884FF6FF729442ECD06C
:107BA0000B4A32F82320AA42F2D1094A02EB83029F
:107BB000D278002AECD00B80012038BDFAF7CCF93E
:107BC0004088A84214BF00200120F6E73C4800206E
:107BD0005048002000B583B0488003230B70002379
:107BE0004B604FF6FE7398420ED007D8031D9BB230
:107BF000012B15D8002003B05DF804FB4FF6FF738E
:107C000098420DD10120F6E701A90120FBF7D6FD2E
:107C100010B99DF80400EEE77846F2F7E3F9F8E7CB
:107C200001A9FFF7A3FFE6E70388012B02D0012B90
:107C30000AD070474288B2F5405FF8D11429F6D1D6
:107C4000A2F5C042428070474388B3F5804FF0D11F
:107C5000242905D01429ECD1A3F5C0434380E8E7DB
:107C6000A3F5A0434380704708B5094B1B7813F078
:107C7000020F0AD113F0010F03D0FFF7D9FD002046
:107C800008BDFFF74DFD0520FAE70B20F8E700BF20
:107C9000544E002008B5002206E0154B03EB82038A
:107CA0000021D97099700132542AF6D90023A3B16A
:107CB0000023104A1360104A1360104A1360104AE0
:107CC0001360104A1360104A1360104A13805380E7
:107CD0000F4A1370FFF788FE08BD03EB8302910083
:107CE0000C4A0A440021D17091700133DFE700BFD4
:107CF00050480020484800203C4800204C480020C4
:107D0000584E0020A4490020D4490020444E0020B1
:107D1000414E0020084F002008B50648064B03607E
:107D2000F5F728FD054A137803F0FD036FF3000310
:107D3000137008BD484E0020D9870300544E002020
:107D400038B5054670B1164B1C6814F0010424D1F7
:107D50006B8823B12888F5F78FFB012806D00B2408
:107D6000204638BD7846F2F73DF9ECE728886B8865
:107D7000184480B2013880B2F5F77EFB0128EED1BD
:107D8000074A136843F0010313602968054B196023
:107D900000210220FFF7DAFCE2E70F24E0E700BF52
:107DA00048480020444E002010B5044618B1044B4A
:107DB0001B68236010BD7846F2F714F9F7E700BF9F
:107DC000444E002008B50122FFF7E6FC08BD000084
:107DD000542809D843091D4A52F8233000F01F02E5
:107DE000D34013F0010F10D1A0F155039BB2FBB9A2
:107DF0005909174A52F8212003F01F0322FA03F30E
:107E000013F0010F16D1002300E00123DBB1542849
:107E100012D955380F4B00EB800203EB82029278A7
:107E200000EB800003EB8000531C83700020704740
:107E30000023EBE70123E9E7074B03EB800083789E
:107E400001338370F2E70520704700BF3C480020F3
:107E50004C480020084F00205048002008B501225F
:107E6000FFF700FE08BD000008B5542812D84309EA
:107E70001A4A52F8233000F01F02D34013F0010FCA
:107E800008D0174B03EB80039A78013A9A70FFF7FA
:107E900053FD08BDA0F155039BB2DBB95909114A46
:107EA00052F8212003F01F0322FA03F313F0010F0D
:107EB00012D0A0F155030C4A03EB830102EB8101C0
:107EC000897803EB830302EB83034A1E9A70FFF762
:107ED00033FDDEE70520DCE70520DAE73C4800203B
:107EE000504800204C480020084F002008B50022D0
:107EF000FFF752FC08BD08B50022FFF7B3FD08BD2F
:107F0000542809D843091D4A52F8233000F01F02B3
:107F1000D34013F0010F10D1A0F155039BB2FBB970
:107F20005909174A52F8212003F01F0322FA03F3DC
:107F300013F0010F16D1002300E00123DBB1542818
:107F400012D955380F4B00EB800203EB8202D27836
:107F500000EB800003EB8000531CC37000207047CF
:107F60000023EBE70123E9E7074B03EB8000C3782D
:107F70000133C370F2E70520704700BF3C48002082
:107F80004C480020084F002050480020002937D0DE
:107F900010B50C46542813D843091C4A52F8233014
:107FA00000F01F02D34013F0010F09D0184B33F833
:107FB00020004880F5F760FA20700020606010BD56
:107FC000A0F155039BB2EBB95909124A52F821208E
:107FD00003F01F0322FA03F313F0010F14D05538F6
:107FE0000D4B00EB800233F82220628000EB800012
:107FF00003EB800004306060022323700020DEE782
:108000000E2070470520DAE70520D8E73C4800201D
:10801000504800204C480020084F002010B582B086
:108020000446542809D843092B4A52F8233000F05B
:108030001F02D34013F0010F10D1A4F155039BB2DE
:1080400023BB5909254A52F8212003F01F0322FAC5
:1080500003F313F0010F1BD1002300E00123BBB396
:1080600069462046FFF792FF70BB9DF80030032B56
:1080700010D0022B2AD1A4F1550303EB8301184A37
:1080800002EB8102D278AAB9052022E00023E6E7BC
:108090000123E4E7134B03EB8403DB780BB90520E2
:1080A00017E0104A02EB8402013BD3702046FFF731
:1080B00043FC0EE00B460A4901EB8303013ADA70F8
:1080C0002046FFF739FC04E0002002E00F2000E02A
:1080D000052002B010BD00BF3C4800204C480020E5
:1080E000084F00205048002070B330B583B00C46D4
:1080F000054659B34088F5F7BFF902280FD0032889
:1081000004D0012802D0102003B030BD2146688879
:10811000FEF770FB08B10020F6E70520F4E74FF604
:10812000FF73ADF80630686850B10DF10601FFF736
:1081300069FC38B1BDF80630553323800020E3E7F1
:108140000E20E1E70520DFE70E2070470E20DBE779
:1081500001464FF6FF7000238BB1002363B17047D7
:1081600098B2012321E04FF6FF72904219D198B2E4
:1081700017E04FF6FF701AE04FF6FF70704710B42B
:108180005A090C4C54F8222003F01F04E24012F06C
:10819000010FE8D0AC2202FB03F2074CA25A914235
:1081A000DED00133002BEBD00023002BE1D05DF8B3
:1081B000044B7047584E00205C4E002018B108B5A3
:1081C000FEF7ACFD08BD4FF6FF70704700B583B0F9
:1081D0000DF10601FEF76EFB20B1BDF8060003B0FD
:1081E0005DF804FB4FF6FF70F9E718B108B5FEF72C
:1081F000CDFD08BD4FF6FF70704700000A4691B1F3
:1082000098B943090B4951F8233000F01F01CB40C6
:1082100013F0010F0BD02A2303FB00F0064B1B5A6F
:108220001380002070470E207047052070470520FE
:10823000704700BFA4490020A8490020292866D81B
:1082400038B504460D46002963D078BB4309344A4B
:1082500052F8233000F01F02D34013F0010F5AD020
:10826000304A2A2303FB00235B88BBB92D4A2A230B
:1082700003FB04235B8859092B4A52F8212003F0A1
:108280001F0322FA03F313F0010F0BD0254B2A2012
:1082900000FB043463882B80002038BD7846F1F75A
:1082A000A1FEE3E77846F1F79DFEEFE7441E620981
:1082B0001E4B53F8223004F01F02D34013F0010F7D
:1082C0002BD01B4A162303FB04235B88BBB9184A37
:1082D000162303FB04235B885909134A52F8212013
:1082E00003F01F0322FA03F313F0010F0BD0104821
:1082F000162303FB040463882B800020CDE7784617
:10830000F1F770FEE3E77846F1F76CFEEFE7052042
:1083100070470E20C1E70520BFE70520BDE700BF7D
:10832000A4490020A8490020584E0020D44900202C
:10833000DC490020002900F08C8070B5C6B00646EC
:1083400014460D46002A00F08680B0F5805F80F06C
:1083500084804FF6FF73138000237BB1002353B357
:108360002088414BAC2202FB00301022294602300B
:108370000AF0D0FF002873D103206FE05A093B496F
:1083800051F8222003F01F01CA4012F0010F0BD058
:10839000AC2202FB03F234498A5A964201D00133DF
:1083A000DBE723800123DAE721884FF6FF72914251
:1083B000F5D12380F3E722884FF6FF739A4251D01C
:1083C00029463046FEF7EAFF284A21884FF44050FC
:1083D000FFF7BCF92388AC2101FB03F18831224B64
:1083E000194404313046F5F7D2F9214B1B6813F4D8
:1083F000802F03D01F4B1B68062B01DC00202DE0D3
:1084000000230F2B0FD8EA5C1B490C681009590098
:10841000265C05A800F8136002F00F020131A25C8F
:1084200042540133EDE705AA00238DF8343003F1FF
:10843000804303F58833D3F8043502920F4A019242
:108440000F4A009240F627120E490720F7F78CFBDF
:10845000D4E70E2070470E2000E0072046B070BD24
:108460000F20FBE70420F9E75C4E0020584E002067
:10847000242E0020202E0020282E0020D459040075
:1084800064390400BA590400034690B942090B4804
:1084900050F8222003F01F00C24012F0010F0AD052
:1084A000074AAC2000FB032393F864300B700020D4
:1084B0007047052070470520704700BF584E0020C8
:1084C0005C4E002000296AD0F8B504460846002C0E
:1084D00067D16309364A52F8233004F01F02D340B3
:1084E00013F0010F5FD0334AAC2303FB042393F84E
:1084F000643073B1012B58D1AC2303FB04F4103466
:1085000014441022A01C0AF005FF00284AD00820BD
:1085100048E02849AC2202FB04F202F110030B44AC
:108520009D1CD0F800E0D0F804C08768C668C3F886
:1085300002E0C3F806C0C3F80A70C3F80E60403208
:1085400011440331F7F7E7F908BBAC2101FB04F153
:108550009031184B194404312846F7F7F1F9D0B996
:108560001448AC2303FB04F3C118012281F86420F2
:1085700003F1A00101440431C05AF4F751FC0C4A44
:1085800021464FF44050FFF7E1F800200AE078461A
:10859000F1F728FDD9E77846F1F724FDE0E70E2052
:1085A00070470520F8BD0520FCE70820FAE700BF6A
:1085B000584E00205C4E002060BB10B504464309B5
:1085C000164A52F8233000F01F02D34013F0010F77
:1085D00022D0134AAC2303FB002393F86430012B11
:1085E00001D0082010BD1046AC2303FB04F3D118C2
:1085F000022281F8642003F1A00101440431C05A31
:10860000F4F70EFC054A21464FF44050FFF79EF860
:108610000020E7E7052070470520E3E7584E0020DB
:108620005C4E0020002840F0A280F8B504464309C3
:10863000514A52F8233000F01F02D34013F0010FCB
:1086400000F097804D4AAC2303FB002393F864307D
:108650000BB90820F8BDAC2101FB00F1501801F165
:108660001003134453F8027F5E689D68DB68C0F80E
:108670000270C0F80660C0F80A50C0F80E3001F170
:108680002003134440311144CA1C023323311768BC
:1086900056689568D0681F605E609D60D860103233
:1086A00010338A42F3D112781A70344EAC2000FB9A
:1086B00004F000F17802324400F19003334453F89F
:1086C000045F5968D3F808C0DF6855609160C2F84C
:1086D0000CC017611D6959695561916133180025F6
:1086E00083F8645000F1880131442A460431305A3D
:1086F000F4F796FB3DB1204A21464FF44050FFF776
:1087000025F80020A6E76B091D4A52F8233005F032
:108710001F02D34013F0010F06D01A4A2A2303FB8D
:1087200005235B88A34201D00135E3E72A2303FB3D
:1087300005239B7D002BF7D013462A2101FB05F171
:108740000A4410310B4453F8077F5E689868D96873
:1087500057609660D06011611B8A938200239375E5
:10876000074AA9B24FF48040FEF7F0FFDCE705208E
:10877000704705206EE700BF584E00205C4E002079
:10878000A4490020A849002070B504460D469DF874
:108790001060FEF7A7FA4FF6FF73984202D020341C
:1087A000AC4200D070BD56B10A4AAC2303FB002393
:1087B00093F86430012BF5D1FFF7FEFEF2E7054A8E
:1087C000AC2303FB002393F86430002BEAD0FFF7BF
:1087D00029FFE7E75C4E00200378042B02D0142B1E
:1087E00010D0704700B583B0037E427E0092003BFC
:1087F00018BF0123426981684068FFF7C5FF03B0D5
:108800005DF804FBC388012B00D07047024A13783F
:1088100043F0020313707047544E002040B108B576
:1088200041B1FEF7A5F808B1002008BD0920FCE71A
:108830000E2070470E20F8E7002A67D0F0B5C7B0C9
:1088400007460C461D461646002B61D0F4F714FE71
:1088500001285FD1002C60D16309344A52F82330DB
:1088600004F01F02D34013F0010F58D00DF58B71A7
:108870003846FDF7EDFF002853D1BDF816314FF60D
:10888000FF7293424FD0324621463846FEF738FCFD
:10889000BDF816110139264A89B24FF4A040FEF7FF
:1088A00055FFBDF816312B80224B186810F480203C
:1088B00031D0214B1B68062B01DC00202BE000236C
:1088C0000F2B0FD8F25C1D490C6810095900255C6C
:1088D00005A800F8135002F00F020131A25C4254C7
:1088E0000133EDE705AA00248DF83440144BD3F88A
:1088F00004350292134A0192134A009240F627224D
:1089000012490720F7F730F9204604E00E2070479F
:108910000E2000E0102047B0F0BD0520FBE7052049
:10892000F9E70F20F7E70420F5E700BF584E0020D5
:10893000D4490020242E0020202E0020282E0020A4
:1089400000100140E459040064390400BA590400DD
:10895000B9B130B583B004460D46F4F78DFD01285A
:1089600002D0102003B030BD0DF106012046FDF706
:108970006FFF20B1BDF806302B800020F2E7052004
:10898000F0E70E2070470000002A6AD0F0B5C7B0AB
:1089900006460C461D461746002B64D0002964D1BC
:1089A0004B09374A52F8233001F01F02D34013F02D
:1089B000010F5CD0B0F5805F5BD22946FDF77AFFEE
:1089C00068B128882F4B2A2202FB0030102239463A
:1089D00006300AF09FFC00284ED103204AE02B8885
:1089E0004FF6FF72934249D03A4621463046FEF791
:1089F000A7FD254A29884FF48040FEF7A7FE234BA8
:108A0000186810F4802035D0214B1B68062B01DC40
:108A100000202FE000230F2B0FD8FA5C1D490C68B3
:108A200010095900255C05A800F8135002F00F0248
:108A30000131A25C42540133EDE705AA00248DF810
:108A40003440154BD3F804350292144A0192144A6B
:108A5000009240F6762213490720F7F785F8204662
:108A600008E00E2070470E2004E0052002E00520FB
:108A700000E0072047B0F0BD0F20FBE70420F9E736
:108A8000584E0020A8490020A4490020242E002090
:108A9000202E0020282E002000100140F459040050
:108AA00064390400BA59040000295AD070B504464C
:108AB0000846002C57D163092E4A52F8233004F09F
:108AC0001F02D34013F0010F4FD02B4A2A2303FB80
:108AD00004235B88294AAC2101FB032393F864300B
:108AE000012B44D1244A2A2303FB04239B7D6BB131
:108AF0002A2303FB04F4103414441022014604F129
:108B000009000AF007FC78B308202DE01A492A234F
:108B100003FB04F3CA180125957510331944066840
:108B200045688268C368C1F80960C1F80D50C1F892
:108B30001120C1F815300831F6F7E2FE68B90E4A87
:108B40002A2303FB04231A79DA750A4A21464FF4D3
:108B50008040FEF7FBFD002006E07846F1F742FA80
:108B6000EDE70E207047052070BD0520FCE70820CA
:108B7000FAE700BFA4490020A84900205C4E00206D
:108B8000A0B908B501464309094A52F8233000F05C
:108B90001F02D34013F0010F01D1052008BD044A84
:108BA0004FF48040FEF79AFE0020F7E7052070475B
:108BB000A4490020002872D138B5044643093B4A35
:108BC00052F8233000F01F02D34013F0010F68D099
:108BD000364B1B6813B90123002014E05A4213409E
:108BE000334A02FB03F3DB0E324AD35CF4E7534211
:108BF0001A402F4B03FB02F2D20E2E4B9B5C03EB71
